:1020000000300020ADE300007124000071240000C6
:1020100000000000000000000000000000000000C0
:10202000000000000000000000000000712400001B
:10203000000000000000000071240000312D0000AD
:10204000712400007124000071240000712400003C
:10205000712400007124000071240000712400002C
:10206000712400007124000071240000712400001C
:10207000713500007124000071240000D12C000093
:1020800071240000712400007124000071240000FC
:1020900071240000712400007124000071240000EC
:1020A00071240000712400007124000071240000DC
:1020B00071240000712400007124000071240000CC
:10240000FFFFFFFFFFFFFFFFFFFFFFFFFFFFFEFFDD
:1024100010B5064C2378002B07D1054B002B02D0BA
:102420000448AFF300800123237010BD90F0FF1F1C
:10243000000000001C000100084B10B5002B03D069
:1024400007490848AFF3008007480368002B00D114
:1024500010BD064B002BFBD09847F9E700000000A9
:1024600094F0FF1F1C00010088F0FF1F0000000017
:1024700000BE704710B5044B044A9A6000F04EF855
:1024800000F082F810BDC04600ED00E00020000022
:1024900020280DDC1F23C217D20E80181840801A86
:1024A0001E3BC0218340034A4900535013607047CC
:1024B000C046FCE700E100E020280BDC1F23C21728
:1024C000D20E80181840801A1E3B83408022024999
:1024D0008B507047C046FCE700E100E070B503296F
:1024E00019DC202817DC03242300FF22C5172B400A
:1024F000AD0F1B18084E401904409B10B4468901CB
:10250000641B134011402240D20091409B00634461
:102510001A681143196070BD00E400E0154B164ABB
:102520009A8001225A7022321A700022134B5A628A
:102530000F23134A51780B4094215370114B19709B
:102540009A238439137013791942FCD10C210C4A57
:1025500013790B40082BFBD1517807330B40102126
:102560000B4353700C2206490B791340082BFBD107
:102570007047C0460020054003E8FFFF008004408C
:1025800000400640005006403F211E4A10B5137817
:102590008B4313D1042413781C4218D0A02080044C
:1025A000194A184B5B78516A5B098900890FD8403A
:1025B000013108F03FFF154B186007E013788B439B
:1025C000402B15D013788B43802B18D010BD137877
:1025D0003E399B065B0F99400D4808F02BFF0D4BD1
:1025E0001B781C4207D043099800C0180002D7E7A7
:1025F00080200002D4E7830018180002D0E70448C6
:10260000CEE7C046004006400080044000F0FF1FB7
:102610000024F4000050064007220C4B10B50120A6
:1026200002211A700824002258709970DA701A7109
:102630005C719A719860D9601A611A755A759A75A9
:10264000DA751A76DA611A6210BDC0464CF9FF1FBE
:10265000FA222D4B120170B51A60DA602B4AFA216A
:102660001A825A820422C900596001209A753A21BF
:102670008022FA24585452010021A4005A620022F8
:102680009C60DC8335242A254E26D9751976597627
:102690009976D976198519873C315A540A391A55D1
:1026A00059640134C3311A55FF3101341A55196484
:1026B0001134C83919539C820234195302345A55C3
:1026C00019539E3518341A771D849C5302369D5336
:1026D000683D5A555B3D1D55023C1953F9395A5412
:1026E00001315A5431315A54802252029A66084AB2
:1026F000084C5A653B229854200007F0E7FA012362
:102700005B42238370BDC046D8F8FF1FE880FFFFFF
:10271000A8610000ACF8FF1F7047C0467047C04674
:102720000A4B0B4A0B495A610B4A0C485A600C4A37
:102730009A6000229A61486148608A6109494A6149
:102740008A618022D2005A607047C04600F00F4074
:10275000132C051840F00F400028050880000004E5
:102760000304001080F00F4070B5584C584B22689D
:1027700000201A60626880255A613A22A15C163AEC
:102780009954E27DA37D12041A431B2107F0B8FB84
:1027900000221721002007F0B3FB4E4A1821002029
:1027A00007F0AEFB4C4A1921002007F0A9FB0722D5
:1027B0001A21002007F0A4FB484A0A21002007F054
:1027C0009FFB474A0421002007F09AFB8022052145
:1027D0005205002007F094FB00220621002007F09C
:1027E0008FFB404A0721002007F08AFB228A6D04F4
:1027F0002A430921002007F083FB628A08212A432B
:10280000002007F07DFB002005F0A4FEE27E2521DC
:102810001203002007F074FB626A2621002007F0F3
:102820006FFB228D29211204002007F069FB4A2347
:10283000E25A023BE15A002007F074FE4E23E25AAE
:10284000023BE15A002007F07DFE50230022E15AAE
:10285000002007F07FFE2368A27D60215A430020FC
:1028600007F04EFB62682021002007F049FBFA22A6
:102870005D21D201002007F043FB1B4A5C210020B0
:1028800007F03EFBE268A18A002007F075FC0022F9
:102890002421002007F034FB00224A21002007F009
:1028A0002FFB00224B21002007F02AFB00222121D0
:1028B000002007F025FB0D4A2021002007F020FB17
:1028C00000224C21002007F01BFB70BDD8F8FF1F31
:1028D000ACF8FF1F9F0F000019190000000100183D
:1028E000100010004E014E01FF7F0000FFFF0000AE
:1028F00080230D4A9B05516910B50B4353613C225F
:102900000A4B0F209A61333A9A6000225A600332D0
:10291000DA601A60013A1A6002321A6041321A60B3
:10292000FFF7B6FD10BDC0460080044000B0034074
:102930007047C0468022024B12059A607047C0461D
:1029400000F00F408022024B12055A607047C046CB
:1029500000F00F40002803D18022024BD2049A607D
:102960007047C04640F00F40002803D18022024B40
:10297000D2045A607047C04640F00F407047C046CE
:102980007047C0467047C0467047C046002803D114
:102990008022024B12019A607047C04600F00F403F
:1029A000002803D18022024B12015A607047C046B2
:1029B00000F00F40002802D18022014B5A6070477E
:1029C00040F00F40002806D1034B1B78002B02D1AA
:1029D0008022024B9A607047ACF0FF1F40F00F401E
:1029E00003000020002B03D1024B18680006C00F23
:1029F0007047C04640F00F40002801D1014B1970CC
:102A00007047C046ACF0FF1F7047C0467047C046D5
:102A10007047C0467047C0467047C0467047C046C2
:102A20007047C0467047C0467047C0467047C046B2
:102A3000002070478022024B52055A607047C04602
:102A400000F00F408022024B52059A607047C0464A
:102A500000F00F40014B00201B68704700F00F4052
:102A600070B5184B18691A69174B4000DC889988B3
:102A7000164BC00FA342A4418B429B4164425B4270
:102A8000DB0024011C438001D20F520104430020CB
:102A9000144307F00FF80500002006F0EBFF0600D6
:102AA000002006F0F7FFFF23AD009B001D40FF2331
:102AB000184004437000FF2676002C43304020432A
:102AC00070BDC04600F00F40ACF0FF1FFF030000D8
:102AD0000A281FD8104B80001B589F460F4B1869BF
:102AE0008000C00F70470E4B0E489B889842804173
:102AF0004042F7E70A4B0B48DB889842804140424E
:102B0000F0E7064B1869C00FECE7044B186940006A
:102B1000C00FE7E70020E5E70CEA000000F00F40F7
:102B2000ACF0FF1FFF030000030010B50020002BD6
:102B300009D1012908D000290BD0022903D1002096
:102B400006F0B8FFC0B210BD002006F093FFC0B27F
:102B5000F9E7002006F09EFFC0B2F4E7002808D095
:102B6000012801D000207047044B1B685B08184007
:102B7000F9E70120014B1B681840F4E700F00F4013
:102B8000002805D0012802D10222034B9A60704729
:102B90000122014B9A60FAE700F00F40002805D0AF
:102BA000012802D10222034B5A6070470122014BD7
:102BB0005A60FAE700F00F4000B583B0082836D815
:102BC0001C4B80001B589F46B9201B4B40001B89A3
:102BD0001A49584308F0B8FC03B000BD164B98885A
:102BE00080B2F9E7144BD88880B2F5E7124B188908
:102BF00080B2F1E7104B588980B2EDE700230193D2
:102C00000F4B0322009302210123002007F0AAFCAE
:102C1000C343DB171840DFE710230193094B03225E
:102C2000009302210123002007F09CFCD4E7002040
:102C3000D2E7C04638EA0000ACF0FF1FFF0F0000EB
:102C4000FFFF00000000FFFF7047C0467047C0460E
:102C50007047C0460E4B82B01B78002B16D0002167
:102C60000C4A0191019B934205D8019B01330193CA
:102C7000019B9342F9D90191019B9342F1D8019BA9
:102C800001330193019B9342F9D9EAE702B07047FF
:102C9000D4F8FF1F3F420F000B4B18691B69400718
:102CA000C00FC0009B0701D504231843064B1B69C6
:102CB000DB0701D502231843044B1B699B0201D596
:102CC000012318437047C04640F00F4000F00F400A
:102CD0000B4B0C4A196989B29180196989B2D1806C
:102CE000196989B21181196989B2518103221A6067
:102CF000013A1A6002321A6041321A607047C046C7
:102D000000B00340ACF0FF1F0221024A53688B431E
:102D10005360704700800440BFF34F8F024A034B5B
:102D2000DA60BFF34F8FFEE70400FA0500ED00E024
:102D300010B5114A114C127823789A4217D863685B
:102D4000013363600E4B1A68002A08D01A68013AF2
:102D50001A601B68002B02D101220A4B1A7000F086
:102D6000ABFC00232370A3680133A36010BD23785C
:102D70000133DBB22370F6E714F0FF1FB8F0FF1F3A
:102D800074F9FF1F70F9FF1FFA22034B52015A60BA
:102D900007221A607047C04610E000E0014B5868F7
:102DA0007047C046B8F0FF1F014B98687047C04697
:102DB000B8F0FF1F802330B5344C1B0265692B43EC
:102DC00001256361324C23782B43237063781D42C5
:102DD000FCD0032365782B4080252B4363700828A3
:102DE00003D82C4B80001B589F468320284B98709B
:102DF0006738D8700020264BCC10E4B2D8721C740F
:102E000007244901C9B259749874D87418755C754F
:102E10009875D875002A0BDDD1105201C9B2D2B213
:102E200019765A769876D87618775C779877D87727
:102E30000121174A13788B43137053781942FCD140
:102E400030BD8120124B98706538D870D2E7B12020
:102E50000F4B98709538D870CCE793200C4B987036
:102E60007738D870C6E78920094B98706D38D870CC
:102E7000C0E78720064B98706B38D870BAE780207F
:102E8000034B98706438D870B4E7C04600800440A3
:102E9000004002405CEA0000F0B5C646012200B5E1
:102EA0002A4B00211C79224229D021241D5D0831A2
:102EB000294028D141702021595C1D5DC9006D0950
:102EC000294341601B5D1B091A40827008210300E1
:102ED000040049421D4D08331034091A1C4ECA180B
:102EE000B446624412781A700133A342F6D12C23FF
:102EF000EA5C1D3B13400370012301212B71080084
:102F000004BC9046F0BD202142702226595C1D5D14
:102F100088461C5D9F5D0136995DFF018C464146E8
:102F200049050F43802109063943E027E403BF0226
:102F30003C4021436446640821436C09A4042143B6
:102F400041609B5D1A408270C0E7C046004002406D
:102F500024400240F0B5C646012200B5364B0021A0
:102F60009C7922423AD09A724668002E3ADB302190
:102F7000F208D2B25A54172201315C5C224074012B
:102F800022430824D2B25A545A5CA2435A54082409
:102F9000294A030005009046644208331035241A7C
:102FA000264FE218BC461978624401331170AB42D7
:102FB000F6D13C2243460F219B5C8B4301780B43A7
:102FC00041468B54002E2FDB31228B5C10218B432A
:102FD00041468B5401220121174B9A71080004BC11
:102FE0009046F0BD3024710DC9B219551821013435
:102FF0001D5DB70C294008257F0129433943B703DC
:103000007F0F39433227C9B21955F109C9B2D955D1
:1030100033215F5C3A4077003A43D2B25A541A5D8A
:103020001543EDB21D55B2E7093A8B5C01218B4384
:1030300041468B54CEE7C046004002403440024037
:103040008023074A1B0351690B435C215361054BE5
:103050001A780A431A7000225A7041329A707047E7
:10306000008004400070074070B50D000400FFF7B9
:1030700061FC2021084AD3781942FCD05471064AD9
:10308000D3785BB2002BFBDA5479E4B2002D01D087
:10309000FFF758FC200070BD0070074010B5040019
:1030A00000210320FFF7E0FF200A0021C0B2FFF754
:1030B000DBFFE0B20021FFF7D7FF01210020FFF77F
:1030C000D3FF10BD70B505000E0006200121FFF7EB
:1030D000CBFF022400210520FFF7C6FF01210020BD
:1030E000FFF7C2FF0442F5D000210220FFF7BCFF2A
:1030F000280A0021C0B2FFF7B7FF0021E8B2FFF7AE
:10310000B3FF01213000FFF7AFFF00210520FFF7DB
:10311000ABFF01210020FFF7A7FFC307F5D470BD67
:10312000F8B58026802702253601FF0101210620FF
:10313000FFF79AFF00210520FFF796FF01210020ED
:10314000FFF792FF0542F5D000210220FFF78CFF28
:10315000300A0021C0B2FFF787FFF0B20021FFF76D
:1031600083FF002421003F394B4259410020C9B25E
:103170000134FFF779FF402CF4D100210520FFF73F
:1031800073FF01210020FFF76FFFC307F5D440361E
:10319000BE42CBD1F8BDC04680231B019C46F0B592
:1031A000C400241A83B064440D0003200021FFF7FB
:1031B0005BFF200A0021C0B2FFF756FFE0B20021FA
:1031C000FFF752FF00210020FFF74EFF002106000D
:1031D0000020FFF749FF002104000020FFF744FF13
:1031E000002107000020FFF73FFF6B460021187108
:1031F0000020FFF739FF6B46002158710020FFF7D0
:1032000033FF6B46012198710020FFF72DFF6B46BD
:103210001E705C70D8711A882B8800209A4201D0E9
:1032200003B0F0BDAB78BB42FAD16B680198C01A0D
:1032300043425841F4E7C046802370B50D00C400F6
:10324000241A1B01E0180978FFF73CFF0F4B69783F
:10325000E018FFF737FF0E4BA978E018FFF732FFB1
:103260000C4B2979E018FFF72DFF0B4B6979E0181B
:10327000FFF728FF094BA979E018FFF723FF084B58
:10328000E979E018FFF71EFF70BDC0460108000095
:103290000208000003080000040800000508000000
:1032A0000608000080231B019C4670B5C400241A48
:1032B00064440D0003200021FFF7D6FE200A002100
:1032C000C0B2FFF7D1FEE0B20021FFF7CDFE002132
:1032D0000020FFF7C9FE002128700020FFF7C4FE80
:1032E000002168700020FFF7BFFE0021A8700020B9
:1032F000FFF7BAFE002128710020FFF7B5FE00217C
:1033000068710020FFF7B0FE0121A8710020FFF7CF
:10331000ABFEE87170BDC046F0B5D6464F46464696
:103320000500C0B58A460620012117000224FFF7D8
:103330009BFE00210520FFF797FE01210020FFF7EB
:1033400093FE0442F5D000210220FFF78DFE280AEB
:103350000021C0B2FFF788FEE8B20021FFF784FE2B
:103360007B1E99463F23002498460226002F0AD14F
:103370003CE04B46191B4B425941C9B2FFF774FE62
:103380000134A74232D05346185D434601352B42E3
:10339000EFD10121FFF768FEA145F1D900210520F9
:1033A000FFF762FE01210020FFF75EFEC307F5D4A0
:1033B00001210620FFF758FE00210520FFF754FEEB
:1033C00001210020FFF750FE0642F5D00021022027
:1033D000FFF74AFE280A0021C0B2FFF745FE01347C
:1033E000E8B20021FFF740FEA742CCD10021052022
:1033F000FFF73AFE01210020FFF736FEC307F5D4A0
:103400001CBC90469946A246F0BDC046F8B50400E3
:1034100015000F0003200021FFF726FE200A0021DF
:10342000C0B2FFF721FEE0B20021FFF71DFE6E1EC5
:103430000024002D0AD0311B4B4259410020C9B253
:10344000FFF712FE38550134A542F4D1F8BDC0464D
:1034500070B51948FFF722FE6D2803D1174B1B7872
:10346000002B26D000211448FFF72CFEFFF758FE52
:10347000134C242221000020FFF74EFF114D402065
:1034800029007022FFF748FF6D210B48FFF71AFE55
:10349000210024220020FFF7B9FF607807F08CFD9F
:1034A000290070224020FFF7B1FF607807F090FDFF
:1034B00070BD034C034DEBE7FF070000D4F8FF1F7E
:1034C0004CF9FF1FD8F8FF1F8022224B5203596985
:1034D00010B50A4380215A61DA680A43DA605A68F3
:1034E0001D490A405A605A681C490A405A605A6885
:1034F0001B490A405A6000221A4BDA709A709A717E
:103500005A71072810D8184B8000C15896231B0207
:10351000994218D9154B48089C46604407F08AFF29
:10352000C204D20EC0B201E0682000221F240D4B5D
:103530001978A1430A431A702C225870DA700C20B3
:10354000FEF7A6FF10BD094807F074FFC204D20EB3
:10355000C0B2EBE700800440FFFCFFFFFFEFFFFF7E
:10356000FF7FFFFF00A0064080EA000040420F00FE
:1035700070B5294B1C79E4B2A30614D5274B1A6801
:103580000132202A3BD059688A423CD0224819682F
:10359000C0795918C0B208721A600A21204A116015
:1035A0009A6A204B1A604025254221D164B2002C32
:1035B00000DB70BD1B4B1D68002DFAD1174CE26A71
:1035C000236B9A4222D0FFF735FA236B5A1C2263F1
:1035D0003422E3189B5C104ADBB2D371236B202B9F
:1035E00000D1256340210C4AD3780B43D370E0E728
:1035F000FFF728FA084AD378AB43D370D6E7002206
:1036000059688A42C2D1044AD279C6E77F23024A66
:10361000D1780B40D370CCE700A00640C4F0FF1F68
:1036200074F9FF1F78F9FF1F0A4A10B5D36A0133F6
:10363000202B0DD0116B8B4209D03424D16A511844
:1036400008558021D362044AD3780B43D37010BD50
:103650000023EFE7C4F0FF1F00A006400A4B5968A3
:103660001A6891420DD05A68511C59609A18127A02
:1036700002705A680120202A00D0704700225A6048
:10368000FBE70020F9E7C046C4F0FF1F014B98623A
:103690007047C046C4F0FF1F034B00201A78002A71
:1036A00001D018700130704770F9FF1F014B186886
:1036B0007047C04678F9FF1F034B1A68002A02D0F2
:1036C0001A68013A1A60704778F9FF1F10B5054B68
:1036D00005491A6888784A604A78052101F0BCFEDD
:1036E00010BDC046C4FAFF1FA8F9FF1F0A4B9A7805
:1036F000002A08D15B78142B09D8084A9B0011686E
:10370000074A995002E00422064B1A7070470322C0
:10371000044B1A70FAE7C046A8F9FF1FC4FAFF1F4E
:10372000B4F9FF1F9CFBFF1F10B5044B09201A685A
:10373000034B5A6003F0ECF910BDC046C4FAFF1FFA
:10374000A8F9FF1F0122054B1A70054B5A78012A70
:1037500002D15A68034B1A607047C0465DFBFF1FD9
:10376000A8F9FF1FF8FAFF1F0222014B1A707047D9
:103770005DFBFF1F0023012000210E4A10B51370CE
:103780000D4A0E4C13700E4A4042E154013301C2FF
:103790002F2BFAD10B4B19700B4B19600B4B196087
:1037A0000B4B19700B4B19600B4B19600B4B1960CD
:1037B00010BDC0469CF9FF1F5CFBFF1F68FBFF1F8D
:1037C00008FAFF1F5DFBFF1FF8FAFF1F64FBFF1FD6
:1037D000A4F9FF1FC4FAFF1FA8FBFF1FB0F9FF1FCA
:1037E0000022014B1A7070475DFBFF1F30B5274A5E
:1037F0005378012B22D0002B15D0022B05D0032BA0
:103800000DD10A22224B5A6030BD0022214B1A6092
:10381000214B1900283104C38B42FCD1F4E7032269
:103820001B4B1A70F0E71B490B68092B27D8581C53
:1038300008605168184A9B009950E5E7154D2868C3
:103840000028E1D0144954680B68A3421BD0002320
:1038500001338342D8D09A008A58A242F8D1421E3E
:1038600093420AD20D4C9B00A44660448000CB18C2
:103870000918586801C38B42FBD12A60C4E70922AA
:10388000034B1A70C0E70023E9E7C046A8F9FF1F01
:103890009CFBFF1F60FBFF1FFCFAFF1FFFFFFF3FAA
:1038A00010B5294A5378092B4BD828499B00CB588F
:1038B0009F46274B1A68D1431960264A08230029DE
:1038C0003BD011689943116010BD5168204B1960BD
:1038D000F3E71F4B51681A68944661441960ECE79E
:1038E0001B4B51681A68511A1960E6E7184B51686A
:1038F0001A6851431960E0E7154C5168206807F0D9
:1039000023FE01002060D8E7114C5168206807F0C1
:1039100001FF2160D1E70E4B51681A681140196010
:10392000CBE70B4B51681A6811431960C5E7084B88
:1039300051681A6851401960BFE711680B43136062
:10394000C2E7034B1968B8E7A8F9FF1FA0EA000017
:10395000C4FAFF1FB0F9FF1F10B5324B5B780A2B7A
:1039600056D8314A9B00D3589F46304B1968304B8C
:103970001960304A0823002950D01168994311601A
:1039800010BD2A4A2A4B1068196818601160F0E7C8
:10399000264B274A11681A68944661441960E8E783
:1039A000224B234A11681A68511A1960E1E71F4B2C
:1039B0001F4A11681A6851431960DAE71B4C1C4B07
:1039C0002068196807F0C0FD01002060D1E7174C9E
:1039D000174B2068196807F09DFE2160C9E7134B5B
:1039E000134A11681A6811401960C2E70F4B104A58
:1039F00011681A6811431960BBE70C4B0C4A116837
:103A00001A6851401960B4E7094A1368DB43136030
:103A1000064B084A196808230029AED111680B43E8
:103A20001360ADE7A8F9FF1FC8EA0000C4FAFF1F42
:103A3000A8FBFF1FB0F9FF1F134B5B78052B08D8BD
:103A4000124A9B00D358124A9F461168114B0B40F3
:103A5000136070478023116899431160F9E70F23C1
:103A600011680B401360F4E710231168994311604B
:103A7000EFE72023116899431160EAE740231168BA
:103A800099431160E5E7C046A8F9FF1FF4EA00007A
:103A9000B0F9FF1FFFFEFFFF154A164B11685B6868
:103AA000154A8B420CDA0323106898430300042064
:103AB0000343136000290ED008218B431360704725
:103AC0008B420CD005231068984303000220034367
:103AD00013600029F0D108310B431360EFE7062390
:103AE000106898430300012003431360E2E7C046D7
:103AF000C4FAFF1FA8F9FF1FB0F9FF1F830703D502
:103B00000822054B1A7070470422044B1A70044BAC
:103B10005A68044B1A60F6E79CFBFF1F5DFBFF1F12
:103B2000A8F9FF1FA0F9FF1F0022014B1A70704770
:103B30005DFBFF1F0A4B0B4A196810B5114203D1F8
:103B4000094A5B68934200D010BD00210748FFF787
:103B5000B9FAFFF7E5FA0120FFF7DEF8F4E7C0460F
:103B6000A8F9FF1F00FFFF00D2040000FF070000BC
:103B7000164B5B78012B1CD0002B0DD0022B06D0EE
:103B8000032B03D1124B1A68124B5A607047124B29
:103B90001A68104B5A60F9E7104A0E4B1278DA7126
:103BA0000F4A12789A710F4A1268110A59711A71E4
:103BB000ECE70A4A074B1278DA71094A12789A71CF
:103BC000094A1268110A59711A71DFE7A8F9FF1F33
:103BD000A8FBFF1F9CFBFF1FC4FAFF1F5DFBFF1F1D
:103BE000A4F9FF1FA0F9FF1FF8FAFF1F0222014BE3
:103BF0001A707047C8FAFF1F024B5A68024B1A60CE
:103C00007047C046A8F9FF1FF8FAFF1F264A5378ED
:103C10000C2B0AD825499B00CB589F46244B1B6888
:103C2000DB0502D55268234B1A607047204B1B6896
:103C30001B06F7D4F9E71E4B1B681B07F2D5F4E708
:103C40001B4B1B68DB07EDD4EFE7194B1B681B0709
:103C5000EBD5E7E7164B1B68DB07E3D5E5E7144B2D
:103C60001B685B07DED4E0E70523114909681942A8
:103C7000D8D1DAE70E4B1B689B07D3D4D5E70C4BA2
:103C80001B689B07CED1D0E7094B1B68DB06C9D464
:103C9000CBE7074B1B689B06C4D4C6E7044B1B68E5
:103CA0005B06BFD4C1E7C046A8F9FF1F0CEB0000BC
:103CB000B0F9FF1FF8FAFF1F074A1368072B09D84E
:103CC000591C1160054A064910689B005850054B65
:103CD0005B6813607047C04664FBFF1FF8FAFF1F64
:103CE000D8FAFF1FA8F9FF1F012210B51D4B1E4C6B
:103CF0001A701E4B20705868802382B01B019842B6
:103D00000CDC01230A420BD00021E21801331170B0
:103D1000082BFAD12378237202B010BD0123F3E7F8
:103D20006946FFF7BFFA6B461978012261705B782C
:103D3000A3706B469B78E3706B46DB7923716B460F
:103D40009B7963716B465B79A3716B461B79E37159
:103D5000002300E0A15CCB18DBB201322372082AF9
:103D6000F8D1D9E7C8FAFF1FCCFAFF1FA8F9FF1F47
:103D7000054A1368002B06D0013B1360034A9B00E1
:103D80009A58034B1A60704764FBFF1FD8FAFF1F55
:103D9000F8FAFF1F30B5124D83B06C78002C0FD0AD
:103DA000012C04D003220F4B1A7003B030BDAB7846
:103DB0002A2BF7D1291D04220B48FFF7ADFAF4E7AF
:103DC000042201A90848FFF721FB6B68019A93427E
:103DD00002D0044B5C60E8E70122024B5A60E4E742
:103DE000A8F9FF1F9CFBFF1FFB0700000022014BEF
:103DF0001A7070475DFBFF1F70B5124D124C2B7887
:103E0000124E63706B683068636080231B019842B8
:103E100005D90723002223700D4B1A7070BD2900AD
:103E2000FFF70AFA29003068FFF7B6F9002805D035
:103E300033680133336065232370EFE70723237072
:103E4000ECE7C046A8F9FF1F9CFBFF1FA0F9FF1F6E
:103E50005DFBFF1F70B5294E294C3378002B0DD127
:103E60006268531C2DD093009B18264A5B00136098
:103E7000FEF794FF244B1860012333706578002D02
:103E800011D0012D0ED1A078802400F069FEE4014C
:103E900004402BD11B4D2B68002B15D11B4A1368F6
:103EA000013B136070BDFEF779FF174B1B68C01A0A
:103EB000C317C0185840134B1B689842EED9357091
:103EC000F0E7134B1A68CEE7FEF768FF0E4B1B684E
:103ED000C01AC317C01858402B689842DED9102367
:103EE0000C4A347011680B431360DBE70023094A66
:103EF00033701168103399431160D3E7A4F9FF1FA1
:103F0000A8F9FF1FACFFFF1F24FBFF1FF8FAFF1FDC
:103F1000C4FAFF1FB0F9FF1F094B9A78002A07D196
:103F20005A78142A08D85968064B9200D15002E0FA
:103F30000422054B1A7070470322034B1A70FAE7EC
:103F4000A8F9FF1FB4F9FF1F9CFBFF1F154B9A78C0
:103F5000002A0CD15A78144B142A1AD8134992000B
:103F600052585A60124A1278002A07D17047042228
:103F70000D4B1A700E4A1278002AF7D00D4A5B6872
:103F800013600D4A002B07D0082311689943116074
:103F9000ECE703221A70EDE7116808330B43136056
:103FA000E4E7C046A8F9FF1F9CFBFF1FB4F9FF1F01
:103FB00029FBFF1FC4FAFF1FB0F9FF1F10B50B4B01
:103FC0009A78002A06D15C78142C07D90322084B72
:103FD0001A7002E00422064B1A7010BD002003F094
:103FE000FDFF044BA400E050F7E7C046A8F9FF1F0F
:103FF0009CFBFF1FB4F9FF1F084B5B782E2B05D9E4
:10400000FF2B07D00322064B1A7070470121054A87
:10401000D154FAE70122044B1A70F6E7A8F9FF1F02
:104020009CFBFF1F68FBFF1F9CF9FF1F084B5B7881
:104030002E2B05D9FF2B07D00322064B1A70704791
:104040000021054AD154FAE70022044B1A70F6E722
:10405000A8F9FF1F9CFBFF1F68FBFF1F9CF9FF1FB8
:10406000064A53782E2B03D90322054B1A7070474A
:104070005168044A9B009950F9E7C046A8F9FF1F10
:104080009CFBFF1F08FAFF1F104B114A19681160B3
:104090005968104A116099680F4A1160D9680F4A2F
:1040A0001160197C0E4A117059690E4A11609969A4
:1040B0000D4A11601B7F0D4AD15C002901D00121FE
:1040C000D15400220A4B1A707047C0467CF9FF1F7A
:1040D000C4FAFF1FA8FBFF1FF8FAFF1FB0F9FF1F6C
:1040E000A4F9FF1F24FBFF1FACFFFF1F68FBFF1F8E
:1040F0005CFBFF1F70B54C4A5368FF2B1ADC5178EC
:104100000B2900D97AE04948890041588F469278B6
:10411000474992009B0052585B589A4200DD71E07B
:1041200000D178E00523434A116899430B0002212E
:104130000B43136070BD91783D4A89009B008858FD
:104140009C588C509850F5E739499B005858937803
:104150009B005850EEE736499B005B589278DB4352
:1041600092005350E6E79278314992009B005B58E9
:10417000505843405350DDE792782D4992009B0000
:104180005B58505803435350D4E792782849920023
:104190009B005B58505803405350CBE79478244D14
:1041A000A4009B005959605907F0B4FA6151C1E766
:1041B00094781F4DA4009B005959605907F0C4F929
:1041C0006051B7E792781A4992009B005B585058AB
:1041D00043435350AEE79278154992009B005B58D9
:1041E0005058C31A5350A5E792781149920050587D
:1041F0009B0084465B58634453509BE703220E4B5D
:104200001A7097E703230B4A116899430B000421A6
:104210000B4313608EE70623064A116899430B008F
:1042200001210B43136085E7A8F9FF1F40EB000055
:10423000ACFBFF1FB0F9FF1F9CFBFF1F70B54A4A84
:1042400053780B2B00D978E048499B00CB589F4608
:1042500093784749474A9B005858146810605C504F
:1042600070BD9378424A9B009A58424B1B689A4211
:1042700067DC6FD00523404A116899430B00022187
:104280000B431360ECE7937839499B005858394A3F
:104290008446126862445A50E2E793783449354ABA
:1042A0009B0058581268821A5A50D9E793783049BF
:1042B000304A9B005858126842435A50D0E79478CD
:1042C0002B4D2C4BA4006059196807F03DF9605143
:1042D000C6E79478264D274BA4006059196807F06B
:1042E00019FA6151BCE793782149224A9B0058583A
:1042F000126802405A50B3E793781D491D4A9B004B
:104300005858126802435A50AAE793781849194A34
:104310009B005858126842405A50A1E79378154ABA
:10432000134912689B00D2435A5099E79378114A77
:104330009B0011680E4A995092E703220F4B1A70A6
:104340008EE703230C4A116899430B0004210B43A9
:10435000136085E70623084A116899430B00012181
:104360000B4313607CE7C046A8F9FF1F70EB000009
:10437000ACFBFF1FC4FAFF1FB0F9FF1F9CFBFF1F20
:1043800010B55C4A53780B2B00D99BE05A499B002F
:10439000CB589F46937859489B001958584A14683F
:1043A0001160584A1C501368002900D186E008218A
:1043B0008B43136010BD9378504A9B009B58504A22
:1043C0001168504A8B4200DA84E000D18AE005236C
:1043D000106898430300022003431360E4E79378D6
:1043E0004649474A9B00595813689C4661441160EE
:1043F000444A1368D8E79378414C404A9B00995847
:104400002368404A591A21601368CDE793783B49E5
:104410003B4A9B005958136859431160394A136845
:10442000C2E79378364C354A9B009958206807F0CC
:104430008BF8344A010020601368B5E79378304C5C
:104440002E4A9B009958206807F064F92D4A216094
:104450001368A9E793782949294A9B00595813689A
:1044600019401160274A13689EE793782349244A2C
:104470009B005958136819431160224A136893E747
:1044800093781E491E4A9B00595813685940116081
:104490001C4A136888E79378184A9B009958184B70
:1044A000C943184A196013687EE79378134A9B0042
:1044B0009958134B134A1960136875E708310B4379
:1044C000136077E70322104B1A700D4B0D4A1968E1
:1044D000136869E70323106898430300042003432B
:1044E000136061E70623106898430300012003432B
:1044F000136059E7A8F9FF1FA0EB0000ACFBFF1FFA
:10450000C4FAFF1FB0F9FF1F9CFBFF1F70B54A4A9A
:1045100053780B2B00D978E048499B00CB589F4635
:1045200093784749474A9B005858146810605C507C
:1045300070BD9378424A9B009A58424B1B689A423E
:1045400067DC6FD00523404A116899430B000221B4
:104550000B431360ECE7937839499B005858394A6C
:104560008446126862445A50E2E793783449354AE7
:104570009B0058581268821A5A50D9E793783049EC
:10458000304A9B005858126842435A50D0E79478FA
:104590002B4D2C4BA4006059196806F0D5FF6051D3
:1045A000C6E79478264D274BA4006059196807F098
:1045B000B1F86151BCE793782149224A9B005858D1
:1045C000126802405A50B3E793781D491D4A9B0078
:1045D0005858126802435A50AAE793781849194A62
:1045E0009B005858126842405A50A1E79378154AE8
:1045F000134912689B00D2435A5099E79378114AA5
:104600009B0011680E4A995092E703220F4B1A70D3
:104610008EE703230C4A116899430B0004210B43D6
:10462000136085E70623084A116899430B000121AE
:104630000B4313607CE7C046A8F9FF1FD0EB0000D6
:10464000ACFBFF1FA8FBFF1FB0F9FF1F9CFBFF1F68
:1046500010B54A4A53780B2B00D978E048499B00A3
:10466000CB589F4693784749474A9B00585814684F
:1046700010605C5010BD9378424A9B009A58424BA0
:104680001B689A4267DB6FD00523404A1168994343
:104690000B0002210B431360ECE793783A49394A47
:1046A0009B009B580A68944663440B60E2E793784A
:1046B0003549344A9B009B580A68D31A0B60D9E7E6
:1046C000937831492F4A9B009B580A6853430B60EB
:1046D000D0E793782C4C2B4A9B002068995806F021
:1046E00033FF2060C6E79378274C264A9B0020685A
:1046F000995807F00FF82160BCE793782249214AC6
:104700009B009B580A6813400B60B3E793781E49DF
:104710001C4A9B009B580A6813430B60AAE79378D6
:104720001949184A9B009B580A6853400B60A1E73F
:104730009378144A9B009B58134ADB43136099E714
:104740009378104A9B009A580F4B1A6092E7032205
:104750000F4B1A708EE703230C4A116899430B0024
:1047600004210B43136085E70623084A1168994327
:104770000B0001210B4313607CE7C046A8F9FF1F23
:1047800000EC0000ACFBFF1FA8FBFF1FB0F9FF1FF0
:104790009CFBFF1F70B53E4A53780B2B64D83D49F4
:1047A0009B00CB589F4693783B499B0059585368D0
:1047B0003A4A994264DC5BD00523116899430B00A7
:1047C00002210B43136007E0937833499B0058584C
:1047D0005268844662445A5070BD93782E499B00BB
:1047E00058585268821A5A50F6E793782A499B0023
:1047F0005858526842435A50EEE79478264DA40028
:104800006059516806F0A0FE6051E5E79478224DAA
:10481000A4006059516806F07DFF6151DCE7937890
:104820001D499B005858526802405A50D4E793786B
:1048300019499B005858526802435A50CCE7937864
:1048400015499B005858526842405A50C4E7937823
:1048500011499B005A58D2435A50BDE7937851688A
:104860000D4A9B009950B7E703220D4B1A70B3E72E
:104870000623116899430B0001210B431360ABE73A
:104880000323116899430B0004210B431360A3E732
:10489000A8F9FF1F30EC0000ACFBFF1FB0F9FF1FB1
:1048A0009CFBFF1F10B5044A044B126898785A60AD
:1048B00000F0F6FC10BDC046C4FAFF1FA8F9FF1FA8
:1048C0000023012000210F4A10B513700E4A0F4C2F
:1048D00013700F4A4042E154013301C22F2BFAD129
:1048E00001220C4B19600C4B19700C4B19600C4BCE
:1048F00019600C4B19600C4B1A700C4B5A680C4B1E
:104900001A6010BD9CF9FF1F5CFBFF1F68FBFF1FB7
:1049100008FAFF1F64FBFF1FA4F9FF1FC4FAFF1F63
:10492000A8FBFF1FB0F9FF1F5DFBFF1FA8F9FF1FCA
:10493000F8FAFF1F06480749427892005358013B96
:104940005350002B02DD4268034B1A607047C0468B
:10495000A8F9FF1FACFBFF1FF8FAFF1F10B5034BB0
:104960001A68034B5A6000F07DFC10BDC4FAFF1FAB
:10497000A8F9FF1F10B5034B1A68034B5A6000F0EB
:104980007BFC10BDC4FAFF1FA8F9FF1F044B1B6876
:10499000FF2B04D8034A9B005168034A9950704783
:1049A000A8FBFF1FA8F9FF1FACFBFF1F0B4B1B68E9
:1049B000FF2B0DD80A4A9B009B580A4A13600A4AEB
:1049C00053600A4A002B04D00823116899431160F0
:1049D0007047116808330B431360F9E7A8FBFF1F0A
:1049E000ACFBFF1FC4FAFF1F9CFBFF1FB0F9FF1FAA
:1049F000044B1B68FF2B04D8034A9B001168034A31
:104A000099507047A8FBFF1FC4FAFF1FACFBFF1FA4
:104A10002B4910B50B68072B14D82A4842780C2A6A
:104A200010D8294C9200A2589746284A12681206BC
:104A300008D55A1C0A60264A264914689B005C5017
:104A40004368136010BD214A12685206FAD5F0E798
:104A50001E4A12689206F5D5EBE71C4A1268D20688
:104A6000F0D5E6E7194A12689207EBD0E1E7174A5A
:104A700012689207E6D5DCE70522144C246814423C
:104A8000E0D0D6E7114A12685207DBD5D1E70F4ACA
:104A90001268D207D6D4CCE70C4A1268D207D1D517
:104AA000C7E70A4A12681207CCD4C2E7074A12685D
:104AB0001207C7D5BDE7054A1268D205B9D4C1E7C8
:104AC00064FBFF1FA8F9FF1F60EC0000B0F9FF1F97
:104AD000F8FAFF1FD8FAFF1F024A800083581943D3
:104AE00081507047BCFFFF1F024B1A6810431860CB
:104AF0007047C046BCFFFF1F024A800083588B43AB
:104B000083507047BCFFFF1F024A13688343136042
:104B10007047C046BCFFFF1F002A05D1054A800030
:104B200083588B4383507047024A8000835819434F
:104B30008150F8E7BCFFFF1F034B8000C0580840BE
:104B4000411E8841C0B27047BCFFFF1F6121034A6C
:104B5000800083588B4383507047C046BCFFFF1FC3
:104B600010B56124034A830098589958A14399507D
:104B700010BDC046BCFFFF1F10B56124044B800070
:104B8000C158C258A243C2506B20084010BDC04655
:104B9000BCFFFF1FF0B5C646002200B5424C82B0F4
:104BA000237865680192052B00D978E03F4A9B0085
:104BB000D3589F46E9B2280E01AA00F08FFB019856
:104BC0002369E5681840237D0121D840A84200DC14
:104BD000002185429241237AC9B25242062B60D805
:104BE000334C9B00E3589F46EAB2280E01AB0621E6
:104BF00000F032FC0198E3E7E9B2280E05F05EF917
:104C0000DEE72E0A2F0EF6B23100380005F056F915
:104C10002A02120E80463100380005F071F9E9B21F
:104C2000380005F04BF9424601903100380005F09C
:104C300067F90198C4E7FEF7B1F8C1E71D4B9C780E
:104C4000002C13D0A8421BD910E01A4B9C78002CE2
:104C50000CD1A84214D809E0164B5C78002C05D181
:104C6000A84203DD0CE00220124B187059709A70B4
:104C700002B004BC9046F0BD0E4B58788842F5D087
:104C800002201870F2E70B4B5C78002CEED0A842A3
:104C9000F6DDEBE7074B98789042F1D1E6E700208C
:104CA0008EE7044BE2E7C046E0FFFF1F94EC0000F4
:104CB000ACEC000018F1FF1F044B10B51B78012B62
:104CC00000D010BDFFF766FFFBE7C04618F1FF1FDD
:104CD000F0B5DE4657464E464546E0B5474C87B0F0
:104CE000E378002B09D02378012B2DD0444A636848
:104CF000126801336360934206D207B03CBC904611
:104D00009946A246AB46F0BD002363602378022B90
:104D1000F3D100233B4D99463B4B2F009A46203759
:104D20002B78002B03D10835AF42F9D1E5E769684C
:104D3000A66888464946721CA2600591052B5AD880
:104D400051469B00CB589F46FFF724FFCEE76A46AB
:104D50004346137143461179180E05AA00F0BEFAB6
:104D6000A2680598B600E368A619F0609342DAD805
:104D7000032323700023E370BFE7FEF70FF8A26858
:104D8000F0E743461B0E9B4643461B0ADBB2190065
:104D90005846019305F092F841460A020290120E1D
:104DA0000199584605F0ACF86A464346D373D17B67
:104DB000584605F083F8029A05900199584605F087
:104DC0009FF8A2680598CDE76A46434613714346AB
:104DD0001179180E05F072F8A268C3E743466A46D7
:104DE000137143461279180E062105AB00F034FB0F
:104DF000A2680598B6E70020B4E7C04618F1FF1F87
:104E000018F0FF1FC0FFFF1FC8EC000001200023A7
:104E10000C490D4A08600121137013619360D3603F
:104E2000D3700A4A4942137053601374536113726A
:104E3000D3601376D361064A137053601161137502
:104E40007047C04618F0FF1F18F1FF1FC0FFFF1F7B
:104E5000E0FFFF1F0022014BDA60704718F1FF1FCF
:104E6000014B18607047C04618F0FF1F70B5002353
:104E700005280DD8094A1278002A09D1084DDC000E
:104E80002A191678002E05D00133042BF7D1002300
:104E9000180070BD285551600123F9E718F1FF1F74
:104EA000C0FFFF1F0023052807D8054A1278002AF3
:104EB00003D1044B18705960012318007047C04695
:104EC00018F1FF1FE0FFFF1F014B186119757047B4
:104ED000E0FFFF1FF0B5CE46474680B5030083B024
:104EE0000020062B2CD8314D2A78002A28D1304CAE
:104EF0002278002B01D0002A22D023720023E16007
:104F000066680193052A4FD82A4B92009B589F460A
:104F1000F1B2300E01AA00F0E1F9E16801982369CD
:104F20001840237DD8400123884200DC00238142C1
:104F300089416B70012301204942A9702B70EB70ED
:104F400003B00CBC90469946F0BD0621F2B2300E7B
:104F500001AB00F081FAE1680198E0E7F1B2300EB0
:104F600004F0ACFFE168DAE7370A330EFFB218004D
:104F70003900984604F0A2FF3202120E8146390031
:104F8000404604F0BDFFF1B2404604F097FF3900FF
:104F900001904A46404604F0B3FFE1680198BEE73D
:104FA000FDF7FCFEE168BAE70020B8E718F1FF1F43
:104FB000E0FFFF1FE0EC0000014B18787047C0468F
:104FC00018F1FF1F064B10B59C680022844204D9DB
:104FD00080001B18DB6801320B60100010BDC0465A
:104FE00018F1FF1F01280FD000280BD0022804D091
:104FF000032804D1054B986870470548FCE7012059
:105000004042F9E70420F7E70020F5E718F1FF1F19
:1050100010270000FF2809D00023032804D8064BDE
:10502000C000C35C0B70012318007047034B1B7852
:105030000B700123F8E7C046C0FFFF1FE0FFFF1F12
:10504000FF280AD00023032805D8064BC0001818F3
:1050500043680B60012318007047034B5B680B60CB
:105060000123F8E7C0FFFF1FE0FFFF1F8023074A6F
:105070001B0351690B435C215361054B1A780A43AA
:105080001A7000225A7011329A70704700800440E2
:105090000070074070B50E0015000024002801D0F4
:1050A000200070BDFDF756FC2021094AD378194233
:1050B000FCD05671064AD3785BB2002BFBDA5479E8
:1050C000E4B2002DECD00020FDF74EFCE8E7C0462E
:1050D000007007407047C046F8B506000D00140088
:1050E0000027FDF753FC0020002C12D020210B4A92
:1050F000D3781942FCD0EF193B785371D3785BB267
:10510000002BFBDA53790130C0B23B700700A0429C
:10511000EED33000FDF744FCF8BDC04600700740F8
:1051200010B50020FDF74EFC72B6084B084A8021EE
:105130001A600022074B00201A60074B013A5A50B0
:105140000131FF315A50FDF7E7FD10BD00F0FF1FA0
:105150007856341210E000E000E100E010B5FFF7EF
:1051600099FF10BD0020704710B5140004F0A6FE92
:10517000206010BD10B504F0C3FE10BD10B51400C2
:1051800005F018FA206010BD10B505F035FA10BD15
:10519000F8B50023254A264E1360264A1360264A96
:1051A0001360264A1360264A13708022D200B11879
:1051B0003300002204C38B42FCD1224D2B7E002BF6
:1051C0000BD1214C214F224B2000E11871180422F1
:1051D0000434FEF71BF9BC42F5D101200023002165
:1051E0001C4A1D4C4042E154013301C22F2BFAD11D
:1051F00000241A4EE0B2FDF76BFC30550134082C48
:10520000F8D101210020FDF78FFC00213072002031
:10521000FDF78AFC30736B7D002B02D1104A1370AE
:10522000F8BD01220E4B1A70FAE7C046F8FAFF1FCC
:10523000ACFBFF1FC4FAFF1FA8FBFF1FB0F9FF1F45
:10524000A4F9FF1F4CF9FF1F1A070000FA0700001E
:10525000E6F8FFFF08FAFF1F68FBFF1F2CF1FF1F96
:105260005DFBFF1F10B5034B5A689878514203F05D
:1052700021F810BDA8F9FF1F10B5034B59689878A5
:1052800003F018F810BDC046A8F9FF1F10B5034B76
:105290000021987803F00EF810BDC046A8F9FF1F52
:1052A00010B50C4B9A78002A08D15A78002A0DD0F4
:1052B000012A07D1596803F053F802E00422064B93
:1052C0001A7010BD0322044B1A70FAE7596803F0F4
:1052D00017F8F6E7A8F9FF1F9CFBFF1F30B5040085
:1052E00083B01500392900D9AFE0594B89005B58CC
:1052F0009F4618226F21200004F002FE6E2120003C
:1053000004F0DCFD2860642003B030BD06212000DD
:1053100004F03EFE200020224E2104F0F1FD2A6818
:1053200020004D2104F0ECFD200021224E2104F04C
:10533000E7FD01224D21200004F0E2FDE3E7152204
:10534000D8E70521E3E71622D4E7042104F020FE84
:1053500020224E21200004F0D3FD2A684D21200098
:1053600004F0CEFD21224E21200004F0C9FD2000D2
:105370000A224D2104F0C4FD6420C5E7242104F075
:105380009DFD28606420BFE71268242104F0B8FD69
:105390006420B9E7002301A90193FFF751FE030040
:1053A0006420002B00D15B38019B2B60ACE700230D
:1053B00001A90193FFF72EFE03006420002BF2D019
:1053C000F2E71068FFF70EFE286064209CE70023D8
:1053D00001A910680193FFF7F5FD03006420002B7D
:1053E000E1D0E1E7FFF7E8FD286064208CE7116871
:1053F000FFF770FD642087E710682100FFF764FD68
:10540000642081E71168FFF74DFD002800D07AE79E
:10541000092079E71168FFF729FD002800D072E71D
:10542000092071E71068FFF71BFD6CE71368042083
:10543000002B00D068E766E71068FFF70BFD6420DB
:1054400062E7FFF7E3FC64205EE703205CE7C04609
:10545000F8EC00007047C046F0B51C0083B000288F
:1054600007D1FF2A01D900F01EFED14B92009B58B4
:105470009F46042006290DD1CE4B1B78002B09D066
:105480002368CD4A1360002B21D00823CB4A116832
:105490009943116003B0F0BD062926D133260225B9
:1054A000C74FBB5D1D4201D101F04CFA0121002024
:1054B000FDF73AFB012801D100F03CFD0023BD4A75
:1054C00023601278002A10D06420BB4A136008239E
:1054D000BA4A11680B431360DCE7052901D100F0DB
:1054E000ECFD062901D100F0E1FD6420D2E7062998
:1054F000FBD100220339100004F002FD022100203C
:1055000004F0DCFC80B220606420B5E70629ECD111
:1055100000220339100004F0F3FC0221002004F003
:10552000CDFC000C20606420A6E70629DDD10C31FB
:10553000002004F0C3FC00B2206064209CE7062930
:10554000D3D10D31F4E7052901D101F079F806290D
:1055500001D101F0C9F8072901D101F033F9082977
:10556000C3D1502002229749FDF750FF642091E7F4
:10557000052901D100F0C6FF062901D101F0D7F8B5
:10558000072901D101F016F90829AED152200222D3
:105590008D49FDF73BFF64207CE7052901D100F030
:1055A00096FD062901D101F089F9072901D101F001
:1055B0007DF9082999D1562001228449FDF726FF5B
:1055C000642067E7052901D100F09CFD062901D17F
:1055D00001F010F9072901D101F0FCF8082984D164
:1055E0004C2004227A49FDF711FF642052E7062976
:1055F00000D07AE70C31002004F060FC754B0014F9
:10560000C218754B9A4200D900202060642033E70D
:10561000052901D100F033FE062901D100F024FF55
:10562000072901D101F0F3F9082900D05DE74820EE
:1056300004226A49FDF7EAFE64202BE7062900D020
:1056400053E7002002F07AFF0500002002F070FF0F
:105650002D1A2DB2256064200EE7052901D100F036
:10566000A8FF062901D101F05BF8072901D101F05B
:1056700081F8082900D038E7592001225849FDF760
:10568000C5FE642006E7052901D100F07CFF06294C
:1056900000D02AE7002002F0EFFB20606420EBE658
:1056A000062900D021E7002002F042FF206064209C
:1056B000E2E6062900D018E7002002F0AFFB2060E8
:1056C000A4E7052901D100F069FF062900D00CE705
:1056D000002002F0AFFB20606420CDE6062900D058
:1056E00003E7002002F0A0FB20606420C4E6052947
:1056F00001D100F076FF062901D101F00AF807294F
:1057000001D101F03FF8082900D0EEE65720012230
:105710003449FDF77BFE6420BCE6052901D100F089
:1057200083FF062901D100F0D8FF072901D101F03C
:1057300019F8082900D0D8E6582001222A49FDF797
:1057400065FE6420A6E6052901D100F03EFF06298A
:1057500001D100F0D7FF072901D101F023F8082972
:1057600000D0C2E6A52001222049FDF74FFE6420AB
:1057700090E6052901D100F040FF062901D100F093
:10578000BAFF072901D101F005F8082900D0ACE6DD
:105790005A2001221649FDF739FE64207AE60629CF
:1057A00000D0A2E6002002F0C9FE2060642063E67B
:1057B000E0ED000029FBFF1FC4FAFF1FB0F9FF1F37
:1057C000D8F8FF1FE8F8FF1FEAF8FF1FEEF8FF1FE9
:1057D000E4F8FF1FFF7C0000FEF90000E0F8FF1F67
:1057E000F1F8FF1FEFF8FF1FF0F8FF1F3DF9FF1F53
:1057F000F2F8FF1F062900D077E6002002F0A4FE91
:105800002060642038E6052901D100F002FF062956
:1058100000D06AE6002002F033FB206064202BE613
:10582000062900D061E6002002F08EFE0CE7062972
:1058300000D05AE6002002F029FB206064201BE61D
:10584000062900D051E6002002F026FB20606420EB
:1058500012E6052901D100F041FE062901D100F030
:10586000A1FD072901D101F040F8082900D03CE64C
:1058700040200422D849FDF7C9FD64200AE6052925
:1058800001D100F000FF062901D100F07CFD0729BD
:1058900001D100F0EEFF082900D026E644200422C2
:1058A000CE49FDF7B3FD6420F4E5052901D100F0F0
:1058B000F5FE062901D100F06CFD072901D100F0A9
:1058C000E0FF082900D010E67A200122C449FDF744
:1058D0009DFD6420DEE5052901D100F0EAFE0629E0
:1058E00000D002E6002002F037FB20606420C3E510
:1058F000062900D0F9E5002002F04EFB206064206C
:10590000BAE5052901D100F0A3FC062901D100F078
:10591000B8FD072901D101F024F8082900D0E4E5F9
:105920005C200122AF49FDF771FD6420B2E5062934
:1059300000D0DAE52A23A84A6420D35C23609BE5E3
:10594000052901D100F0D3FC062901D100F079FD31
:10595000072901D101F072F8082900D0C5E55E20C1
:105960000222A149FDF752FD642093E5052900D1EB
:10597000D2E3062901D100F021FD072901D101F070
:1059800036F8082900D0B0E5602002229749FDF7DB
:105990003DFD64207EE5052901D100F08DFC06293E
:1059A00001D100F047FD072901D101F04FF8082986
:1059B00000D09AE58E2002228D49FDF727FD642054
:1059C00068E5062900D090E5012300205B420093A2
:1059D000019005336D22663104F0C4FD206015E6A8
:1059E000062900D081E5012300205B42009301904D
:1059F0000633EFE76420052900D03BE521686038D5
:105A0000072900D946E50020C9B2FDF71DF9642039
:105A100040E5062900D068E502F0B0F92060642076
:105A20002AE5062900D060E5002002F0D9F92060BF
:105A3000642021E5062900D057E505F017FA20601B
:105A4000642019E5062900D04FE51231002004F04A
:105A500035FA81B20131674805F076FD2060642097
:105A60000AE5062900D040E505F05CFA20606420D4
:105A700002E5052901D100F02AFE062900D034E50F
:105A800005F064FA20606420F6E4052901D100F0F5
:105A900019FD062900D028E505F064FA206064208D
:105AA000EAE4052901D100F055FD062900D01CE5E6
:105AB00005F064FA20606420DEE4052901D100F0DD
:105AC0005BFD062900D010E5002002F087FA206077
:105AD0006420D1E4052900D14BE3062901D100F06F
:105AE0009DFC072901D100F0C8FF082900D0FCE483
:105AF000942004224049FDF789FC6420CAE4062969
:105B000000D0F2E4012300205B42009301900433B3
:105B100060E7052900D1E2E3062901D100F0B9FED2
:105B2000072901D100F05EFE082900D0DDE47520D0
:105B300001223249FDF76AFC6420ABE4052900D15B
:105B400072E3062901D100F0D8FE072901D100F047
:105B5000E1FE082900D0C8E4772001222849FDF79A
:105B600055FC642096E4052901D100F074FD062956
:105B700000D0BAE405F032FA206064207CE4052904
:105B800001D100F06EFD062900D0AEE405F03EFA2A
:105B90002060642070E4052901D100F06EFD062923
:105BA00000D0A2E405F03EFA2060642064E40529F8
:105BB00000D158E3062901D100F069FC072901D181
:105BC00000F06BFF082900D08FE47B2001220D49F3
:105BD000FDF71CFC64205DE4D8F8FF1FDCF8FF1F14
:105BE00012F9FF1FF4F8FF1FF6F8FF1FF8F8FF1F68
:105BF00026F9FF1F00E1F5052CF9FF1F0EF9FF1F25
:105C00000FF9FF1F13F9FF1F052900D17BE30629B8
:105C100001D100F01CFC072901D100F0AAFE0829DF
:105C200000D062E468200222E649FDF7EFFB642021
:105C300030E4052900D172E3062900D055E43C2365
:105C4000E14A6420D35C5B07DB0F2360FFF714FCA1
:105C5000062900D049E47031002004F02FF9072311
:105C6000184020606420FFF707FC062900D03CE4C0
:105C7000012300205B420093019007336D226631BF
:105C800004F070FCD04B997D05F05EFC2060642030
:105C9000FFF7F2FB062900D027E4012300205B4236
:105CA00000930190030095E6062900D01DE401232E
:105CB00000205B420093019002338BE6062900D05E
:105CC00013E4012300205B42009301900333D5E7E6
:105CD000052900D164E2062900D176E3072901D124
:105CE00000F065FE082901D0FFF7FFFB902002229B
:105CF000B649FDF78BFB6420FFF7CCFB052901D1EA
:105D000000F0F7FB062900D136E3072901D100F0A6
:105D1000DCFD082901D0FFF7E8FB78200222AC491E
:105D2000FDF774FB6420FFF7B5FB052900D101E204
:105D3000062901D100F07EFD072901D100F0CDFD3B
:105D4000082901D0FFF7D1FB64200422A149FDF707
:105D50005DFB6420FFF79EFB052900D1E2E30629E5
:105D600001D100F0EBFC072901D100F0F3FC082978
:105D700001D0FFF7BAFB5B2001229749FDF746FBF4
:105D80006420FFF787FB052900D1E3E1062901D153
:105D900000F05AFD072901D100F063FD082901D068
:105DA000FFF7A3FB752001228C49FDF72FFB642030
:105DB000FFF770FB062901D0FFF797FB7031002039
:105DC00004F07CF843055B0F23606420FFF754FB6D
:105DD000052900D1B0E2062900D125E3072901D128
:105DE00000F00DFE082901D0FFF77FFBA820042258
:105DF0007B49FDF70BFB6420FFF74CFB052900D125
:105E0000F3E1062900D14FE3072901D100F0DFFDBE
:105E1000082901D0FFF769FB882002227149FDF7AC
:105E2000F5FA6420FFF736FB052900D1CAE10629FF
:105E300000D1D1E2072901D100F0D1FD082901D01C
:105E4000FFF753FB8A2002226749FDF7DFFA64203F
:105E5000FFF720FB052900D11BE2062900D109E349
:105E6000072901D100F011FE082901D0FFF73DFB01
:105E70008C2002225D49FDF7C9FA6420FFF70AFB76
:105E8000052900D124E3062901D0FFF72EFB05F0F8
:105E90008DF820606420FFF7EFFA052900D1E6E3D2
:105EA000062901D0FFF721FB05F074F8206064207B
:105EB000FFF7E2FA052900D1BEE1062900D1EDE2A3
:105EC000072901D100F02EFD082901D0FFF70DFBB5
:105ED000802004224649FDF799FA6420FFF7DAFA98
:105EE000052900D194E1062900D1E4E2072901D176
:105EF00000F020FD082901D0FFF7F7FA73200122F6
:105F00003C49FDF783FA6420FFF7C4FA062901D063
:105F1000FFF7EBFA332604252B4FBB5D1D4201D161
:105F200000F09CFD02210020FCF7FEFD012801D0BD
:105F3000FFF7C4FA0123304A23601278002A01D106
:105F4000FFF7D3FA2D4A64201360FFF79EFA052964
:105F500000D105E2062900D12AE2072901D100F08B
:105F60002EFD082901D0FFF7C0FA8420042224491D
:105F7000FDF74CFA6420FFF78DFA062901D0FFF7F0
:105F8000B4FA002002F060FB20606420FFF774FA8E
:105F9000052900D1E4E2062901D0FFF7A6FA05F0B1
:105FA00029F820606420FFF767FA052900D1DDE2B7
:105FB000062901D0FFF799FA05F004F82060642063
:105FC000FFF75AFA00F9FF1FD8F8FF1F28F9FF1F43
:105FD00010F9FF1FFCF8FF1FF3F8FF1F0DF9FF1F5B
:105FE00040F9FF1F20F9FF1F22F9FF1F24F9FF1FAF
:105FF00018F9FF1F0BF9FF1F29FBFF1FC4FAFF1F32
:106000001CF9FF1F05296FD0062901D0FFF76DFA93
:106010003C23F54A6420D25C3B3B13402360FFF7EE
:106020002BFA062901D0FFF760FA0020FEF798FD51
:1060300020606420FFF720FA062901D0FFF755FA07
:1060400033260125E84FBB5D1D4201D100F0E7FC7E
:1060500000210020FCF768FD012801D0FFF72EFA8F
:1060600068E7062901D0FFF740FA2131002003F04C
:1060700025FF20606420FFF7FFF9052900D166E1C4
:10608000062900D1E9E1072901D100F07AFC0829AD
:1060900001D0FFF72AFA74200122D449FDF7B6F99E
:1060A0006420FFF7F7F90320FFF7E4F90020FCF77D
:1060B00097FC20606420FFF7DFF923680020002BA5
:1060C00000D02AE2FCF77EFC6420FFF7E3F92168A8
:1060D0004B1EFE2B02D90420FFF7DCF9002002F052
:1060E00071F96420FFF7D6F92368002B01D000F086
:1060F00050FC3C220120BC498B5C83438B546330B1
:10610000FFF7C8F92168BA4B9942E4D8002002F0A1
:1061100067F96420FFF7BEF9B64A2368042099188E
:10612000B54A914201D9FFF7B5F9AF4A60301384FF
:10613000FFF7B0F92268B14B04209A4201D9FFF76A
:10614000A9F9A94B00205A62213103F0D9FE64203D
:10615000FFF7A0F9236804203522012B01D9FFF7AE
:1061600099F9A14900208B5402F0F4F96420FFF75B
:1061700091F9A34A236804209918A24A914201D9AF
:10618000FFF788F9984AA0485365216805F0DCF9C3
:106190001821421E002003F0B3FE6420FFF77AF9B5
:1061A00021689A4B0420994201D9FFF773F95023D3
:1061B0008D4A89B2D1520022100004F0CBF964203C
:1061C000FFF768F92268914B04209A4201D9FFF742
:1061D00061F9854B92B245315A5202390020595A21
:1061E00004F0A0F96420FFF755F92168874B0420DB
:1061F000994201D9FFF74EF948227B4B89B2995257
:10620000023200209A5A04F08DF96420FFF742F917
:1062100023680420072B01D9FFF73CF93322724988
:1062200060308B54FFF736F9236804203722012BA6
:1062300001D9FFF72FF994E723686E4A04209342AF
:1062400001D9FFF727F9684A60301364FFF722F994
:1062500023680420022B01D9FFF71CF9624A603041
:106260001377FFF717F923680420082B01D9FFF7EC
:1062700011F93B225C4960308B54FFF70BF923681E
:106280005B4A934200D926E7574A64209360FFF7A0
:1062900001F921685D4B0420994201D9FFF7FAF812
:1062A0004C22514B89B29952023200209A5A04F082
:1062B00049F96420FFF7EEF82268544B04209A4213
:1062C00001D9FFF7E7F8484B92B249315A520239E7
:1062D0000020595A04F036F96420FFF7DBF82368F0
:1062E0000420012B01D9FFF7D5F8362239E72368BE
:1062F000474A0420934201D9FFF7CCF83A4A60306C
:10630000D383FFF7C7F82368424A0420934201D998
:10631000FFF7C0F8344A60301385FFF7BBF82368F5
:1063200031493C22002B00D1CAE10423885C03439D
:106330008B546420FFF7AEF823680420052B01DCA2
:10634000FFF7A8F8284A60309366FFF7A3F8072301
:10635000226825491340342264208B54FFF79AF8B1
:1063600023682D4A0420934201D9FFF793F81E4A6F
:1063700060305364FFF78EF81B4B642038229B5E1D
:106380002360FFF779F8184B64205B682360FFF700
:1063900073F83A23144A6420D35C5A1E9341236055
:1063A000FFF76AF8104B64201B682360FFF764F85E
:1063B0000D4B64205B6C2360FFF75EF80A4B642092
:1063C00020229B5E2360FFF757F85023064A642083
:1063D000D35A2360FFF750F84A23034A6420D35A64
:1063E0002360FFF749F8C046D8F8FF1F0CF9FF1FDC
:1063F00088130000400D0300801A0600FFFFFF0015
:10640000589EFFFFF824010000E1F505FF7F000022
:1064100010270000FFFF0000A0860100F94B642058
:106420005B6D2360FFF728F8F64B64209B6E2360BA
:10643000FFF722F84E23F34A6420D35A2360FFF774
:106440001BF8F04B6420DB8B2360FFF715F8ED4B56
:1064500064201B8D2360FFF70FF83423E94A642082
:10646000D35C2360FFF708F8E64B64209B68236049
:10647000FFF702F84C23E34A6420D35A2360FEF767
:10648000FBFFE04B64201B7F2360FEF7F5FF3B23FF
:10649000DC4A6420D35C2360FEF7EEFFD94B642016
:1064A0001B6C2360FEF7E8FF4823D64A6420D35ACA
:1064B0002360FEF7E1FF3323D24A6420D35C2360DC
:1064C000FEF7DAFF206804F047FD6420FEF7E2FFE4
:1064D000206804F065FD6420FEF7DCFF21680020E1
:1064E00001F0E8FC002801D0FEF7FFFF0420FEF7D2
:1064F000D1FF2268C34B00201A8702F02BF86420DA
:10650000FEF7C8FF2168002002F08EFF002801D0AE
:10651000FEF7EBFF0420FEF7BDFFFCF74BFA64200B
:10652000FEF7B8FF2368B74D5A1E93412031EB7632
:10653000002003F0C3FC8023EA7E5B0112031A40B3
:10654000B14B252118400243002003F0D9FC642000
:10655000FEF7A0FF206804F00BFD6420FEF79AFF11
:10656000206804F041FD6420FEF794FF206804F0E9
:1065700023FD6420FEF78EFF0020216801F04EFD10
:106580006420FEF787FF2168002001F039FE002813
:1065900001D0FEF7AAFF0420FEF77CFF216800204F
:1065A00001F060FE002801D0FEF79FFF0420FEF7F7
:1065B00071FF21680020C9B201F08AFF002801D0D4
:1065C000FEF793FF0420FEF765FF21680020C9B2A3
:1065D00001F03EFF002801D0FEF787FF0420FEF700
:1065E00059FF21680020C9B201F012FF002801D034
:1065F000FEF77BFF0420FEF74DFF21680020C9B2A3
:1066000001F07EFF002801D0FEF76FFF0420FEF7A7
:1066100041FF2168002001F04DFE002801D0FEF767
:1066200064FF0420FEF736FF21680020C9B201F0A4
:1066300029FF002801D0FEF758FF0420FEF72AFFAB
:106640002168002002F0CCFE002801D0FEF74DFFAB
:106650000420FEF71FFF206804F0BAFC6420FEF758
:1066600019FF206804F0CCFC6420FEF713FF2068BB
:1066700004F08AFC6420FEF70DFF206804F0CCFCD7
:106680006420FEF707FF2168002001F031FC00289C
:1066900001D0FEF72AFF0420FEF7FCFE216800204F
:1066A00001F040FC002801D0FEF71FFF0420FEF798
:1066B000F1FE0020216801F023FE6420FEF7EAFECF
:1066C00004208B5C83438B546030FEF7E3FE20682C
:1066D00004F036FC6420FEF7DDFE002001F0EEFE43
:1066E00020606420FEF7C8FE002002F06BFE2060F0
:1066F0006420FEF7C1FE002001F010FF206064203E
:10670000FEF7BAFE002001F0B3FE20606420FEF721
:10671000B3FE002001F08EFE20606420FEF7ACFE88
:10672000002001F0E3FE20606420FEF7A5FE0020BB
:1067300002F06CFE20606420FEF79EFE1F310020F8
:1067400003F0BCFB2F4AC304DB0FD3766420236025
:10675000FEF792FE5B2001222C49FCF7DDFD642050
:10676000FEF798FE582001222949FCF7D5FD642048
:10677000FEF790FE592001222649FCF7CDFD64204A
:10678000FEF788FE572001222349FCF7C5FD64204F
:10679000FEF780FE5A2001222049FCF7BDFD64204F
:1067A000FEF778FEA52001221D49FCF7B5FD642007
:1067B000FEF770FE522002221A49FCF7ADFD64205C
:1067C000FEF768FE502002221749FCF7A5FD642061
:1067D000FEF760FE4C2004221449FCF79DFD642066
:1067E000FEF758FE762001221149FCF795FD642042
:1067F000FEF750FE002001F001FE20606420FEF74D
:106800003BFEC046D8F8FF1FFFEFFFFFF3F8FF1F66
:10681000F0F8FF1FF1F8FF1FEFF8FF1FF2F8FF1F5E
:106820003DF9FF1FEAF8FF1FE8F8FF1FE4F8FF1F1C
:106830000EF9FF1F2031002003F040FB9B4B5862F4
:1068400020606420FEF718FE2D31002003F036FB97
:106850000123964A18403433D05420606420FEF758
:106860000BFE752001229249FCF756FD6420FEF7CD
:1068700011FE442004228F49FCF74EFD6420FEF7F0
:1068800009FE7A2001228C49FCF746FD6420FEF7C0
:1068900001FE2D31002003F011FB3622C304834991
:1068A000DB0F8B5464202360FEF7E6FD56200122A7
:1068B0008249FCF731FD6420FEF7ECFD002001F079
:1068C00073FD20606420FEF7D7FD782002227C490A
:1068D000FCF722FD6420FEF7DDFD642004227949E7
:1068E000FCF71AFD6420FEF7D5FD402004226F4915
:1068F000FCF712FD6420FEF7CDFD2D31002003F0E2
:10690000DDFA3722C3056949DB0F8B54642023600D
:10691000FEF7B2FD772001226B49FCF7FDFC6420F5
:10692000FEF7B8FD802004226849FCF7F5FC6420DE
:10693000FEF7B0FD732001226549FCF7EDFC6420F1
:10694000FEF7A8FD01210020FCF7EEF8002801D198
:10695000FFF7F0FABB5D2B4201D1FEF7AFFDFEF76A
:10696000A5FD5C2001225B49FCF7D6FC6420FEF704
:1069700091FD682002225849FCF7CEFC6420FEF706
:1069800089FD742001225549FCF7C6FC6420FEF7FE
:1069900081FD00222331100003F0B2FA3C220123D2
:1069A0004249885C03438B546420FEF773FD9020BA
:1069B00002224B49FCF7B0FC6420FEF76BFD8420FB
:1069C00004224849FCF7A8FC6420FEF763FD8820F8
:1069D00002224549FCF7A0FC6420FEF75BFD8A20FB
:1069E00002224249FCF798FC6420FEF753FD602028
:1069F00002223F49FCF790FC6420FEF74BFDA820E3
:106A000004223C49FCF788FC6420FEF743FD482043
:106A100004223949FCF780FC6420FEF73BFD00218D
:106A20000800FCF781F8002801D1FFF783FABB5D6D
:106A30002B4201D1FEF742FDFFF70AFB5E20022246
:106A40002E49FCF769FC6420FEF724FD8E2002220B
:106A50002B49FCF761FC6420FEF71CFD022100209D
:106A6000FCF762F8002801D1FFF764FABB5D2B4206
:106A700001D1FEF723FDFFF755FA942004222149A6
:106A8000FCF74AFC6420FEF705FD8C2002221E491B
:106A9000FCF742FC6420FEF7FDFC7B2001221B4931
:106AA000FCF73AFC6420FEF7F5FCC046D8F8FF1F5F
:106AB0000DF9FF1FDCF8FF1F12F9FF1FEEF8FF1F93
:106AC00010F9FF1FFCF8FF1F0FF9FF1F18F9FF1F38
:106AD0000BF9FF1FF4F8FF1F00F9FF1F0CF9FF1F50
:106AE00028F9FF1F1CF9FF1F20F9FF1F22F9FF1FC4
:106AF000F8F8FF1F40F9FF1FE0F8FF1FF6F8FF1F2F
:106B000026F9FF1F2CF9FF1F24F9FF1F13F9FF1FA0
:106B100070B5BE4CA378002B09D16378403BDBB243
:106B2000BF2B00D96DE1BA4A9B00D3589F46022B78
:106B300015D0032B2ED00422B64B1A700A280DD183
:106B4000B54A1278002A09D0B44A5B681360B44A87
:106B5000002B1AD0082311689943116070BD627828
:106B6000372A1FD80A2800D114E209281FD00B2881
:106B700000D16EE20C28F1D1AA4BAB49920051181A
:106B8000D0180422FCF742FCE8E7116808330B43F5
:106B90001360E3E763782E2B00D932E1A34A9B0010
:106BA000D3589F460A2800D1F4E10928D6D161685C
:106BB0009D4B9200D150D1E70A28CFD19C4A954BEA
:106BC00012785A60BCE70A2800D14BE20928C5D1E7
:106BD00021799848FCF776FAC0E70A2800D1E4E169
:106BE0000928BBD1636894490422CB6003300C317F
:106BF000FCF792FBFBF792FDB0E70A2800D1F6E123
:106C00000928ABD121798C4B00201970FCF75AFA76
:106C1000A4E70A2800D1D2E109289FD1864D042299
:106C20002900636810312B610730FCF775FBFBF717
:106C300075FD2A69A9686879FCF7BCF88EE70A280F
:106C400000D1FCE1092800D088E77B4963681C314A
:106C50000B6004221330FCF75FFB7FE70A2800D1AA
:106C6000A8E1092800D079E72179734B073899709A
:106C7000FCF728FA72E70A2800D1C2E1092800D0FF
:106C80006CE720796C4C607004F0AEF961780120FB
:106C9000FCF718FA62E70A2800D05FE7674A5D4B05
:106CA00012685A604CE70A2800D194E1092800D004
:106CB00054E72179604B04385971FCF703FAFBF76C
:106CC0002DFD4BE70A2800D18AE1092800D045E7CD
:106CD0002179002900D0CBE1574BD9751720FCF75B
:106CE000F1F93BE70A2800D038E7554A494B1278BA
:106CF0005A6025E70A2800D030E7514A454B127800
:106D0000043A5042504158601AE70A2800D147E13E
:106D1000092800D022E70123474D21792A7D13421B
:106D200002D00B4200D1FEE114202975FCF7CAF90C
:106D300014E70A2800D187E1092800D00EE73E4970
:106D4000636820310B6004221730FCF7E5FA05E791
:106D50000A2800D15FE1092800D0FFE62179364BEF
:106D60000C305975FCF7AEF9F8E60A2800D15CE161
:106D7000092800D0F2E6274B5A68324B1A60EDE63C
:106D80000A2800D138E1092800D0E7E62A4D6368D7
:106D90002900AB6008310422013846E70A2800D1F7
:106DA00048E1092800D0D9E66368012B00D8B1E199
:106DB0000422184B1A70D1E60A2800D126E10928CE
:106DC00000D0CBE621791C4C0638E170FCF77AF94B
:106DD000E078FCF75BFCC1E60A2800D120E1092835
:106DE00000D0BBE60B4B5A68174B1A60B6E60A2870
:106DF00000D1E9E0092800D0B0E62279134B1A70DF
:106E0000ACE60322034B1A7098E6C046A8F9FF1FB0
:106E1000E0F100009CFBFF1F29FBFF1FC4FAFF1FCE
:106E2000B0F9FF1F1A070000ACFBFF1FE0F40000E1
:106E300048F9FF1FFF0700004CF9FF1FF8FAFF1F7A
:106E40005DFBFF1FF8FFFF1FFCFFFF1F28FBFF1F5D
:106E50000A2800D127E1092800D07FE66268B44BF8
:106E60009A627BE60A2800D122E1092800D075E663
:106E70006268AF4B5A6271E60A2800D11DE1092809
:106E800000D06BE66268AA4B1A6267E60A2800D156
:106E9000F5E0092800D061E66268A54BDA615DE69D
:106EA0000A2800D1F5E0092800D057E6FBF776FF65
:106EB000A04B626858609E4B5A604FE60A2800D18A
:106EC00000E1092800D049E66268994BDA6245E69C
:106ED0000A2800D1D8E0092800D03FE66268944B28
:106EE0009A613BE60A2800D100E1092800D035E686
:106EF000FBF754FF8F4B626818608D4B1A602DE6CC
:106F00000A2800D1E8E0092800D027E62279884B3A
:106F10005A7323E60A2800D1F2E0092800D01DE6C2
:106F20006268834B1A6119E60A2800D1CFE009286C
:106F300000D013E622797E4B1A730FE60A2800D19F
:106F4000D9E0092800D009E66268794B5A6105E664
:106F50000A2800D1C5E0092800D0FFE52279744B4A
:106F60009A73FBE50A2800D1CFE0092800D0F5E5A7
:106F700022796F4BDA73F1E50A2800D18EE00928F7
:106F800000D0EBE5FBF70AFF6A4B62689860684B3C
:106F90009A60E3E568499200684B52585A60CFE521
:106FA000674A664B127D5A60CAE5654A634BD268F0
:106FB0005A60C5E5624A614B92785A60C0E5604A02
:106FC0005E4B12695A60BBE55E4A5C4B1278511EFB
:106FD0008A415A60B4E55A4A584B52795A60AFE533
:106FE000574A564BD27D511E8A415A60A8E5544AF1
:106FF000524B12785A60A3E5514A504B92685A603E
:107000009EE54F4A4D4B52785A6099E54C4A4B4B9E
:10701000D2785A6094E54A4A484B527D5A608FE5CF
:10702000494A464B12685A608AE5484B1A68434BF6
:107030005A6085E5424A414B127E5A6080E5404ADB
:107040003E4BD2695A607BE53D4A3C4B126A5A601E
:1070500076E53F4B384992005118D0180422FCF7CE
:107060005BF97BE53B48FCF719F8344B586067E562
:107070000123334A0121D375304A53602EE62C4B4D
:10708000DA692E4B5A605BE5294B9A692B4B5A60A3
:1070900056E5274B5A68294B5A6051E5244B9A68AC
:1070A000264B5A604CE5224B9A6A244B5A6047E5BE
:1070B0001F4B5A6A214B5A6042E51D4B1A6A1F4BFF
:1070C0005A603DE51A4BDA6A1C4B5A6038E5184B9A
:1070D0001A7B1A4B5A6033E5154B5A7B174B5A6093
:1070E0002EE5134B9A7B154B5A6029E5104B1A6815
:1070F000124B5A6024E50E4B5A69104B5A601FE53B
:107100000B4B1A690D4B5A601AE5094BDA7B0B4B96
:107110005A6015E522790A4B0F491A760F30012281
:10712000FCF7FAF81AE5FBF7FBFF2179FCE5C0460E
:107130002CFBFF1FB0FFFF1FACFBFF1F9CFBFF1FC3
:107140004CF9FF1F28FBFF1FFCFFFF1FF8FFFF1F6D
:107150001A070000FF07000064F9FF1F10B5094B74
:107160009A78022A06D15A685878002A06D1FBF785
:1071700007FD02E00422044B1A7010BDFBF70EFD60
:10718000FBE7C046A8F9FF1F9CFBFF1F10B51F4C73
:10719000A378012B29D0002B1FD0022B06D004226C
:1071A0001B4B1A7022780F2A08D010BD6078FBF7AD
:1071B000D5FC174B227858600F2AF6D1154A127861
:1071C000002AF2D0144A5B681360144A002B12D0D4
:1071D0000823116899431160E7E76078FF280FD012
:1071E000FBF776FC0A4B5860DCE76078FBF7E4FCC1
:1071F000074B5860D6E7116808330B431360D4E798
:10720000FBF72EFC024B5860CCE7C046A8F9FF1FE5
:107210009CFBFF1F29FBFF1FC4FAFF1FB0F9FF1FD4
:1072200010B52C4B5B78002B10D101222A4B2B4838
:107230001A702B4B9B7803702A4B1A680023117825
:107240000133C1540132082BF9D110BD012B11D0EB
:10725000022B18D0052B28D0062B30D0072BF4D1C9
:107260000A22214BDA7101329A7101325A710132CC
:107270001A71EAE706211C4AD17153715F31083354
:1072800091711371E1E701228024134B13481A70A6
:10729000134BA4019B780370144B154A19789A1864
:1072A00001338154A342F8D1CFE714220E4BDA7197
:1072B000023A9A71073A5A7112321A71C5E70022DE
:1072C000094BDA7111329A71033A5A7118321A71F4
:1072D000BBE7C046A8F9FF1FC8FAFF1FCCFAFF1F83
:1072E0004CF9FF1F10F0FF1F9CFBFF1FF81F000051
:1072F00009E0FFFF642230B57C4B7D4C18787D4D52
:107300008100227069585A6883B0607062608F464D
:1073100079491B680B4079498B4204D1784B9A42DA
:1073200001D1FDF7FDFE03B030BD764B9A42FAD194
:107330000122754B5A73F6E75978987802F0BEFD32
:107340006060F0E75978987802F0DAFDEBE7019297
:107350005978987801AAFDF7C1FF2070019B6360FE
:10736000E1E7FCF743FADEE7FCF714FDDBE7FCF7A7
:10737000E1FBD8E7FFF754FFD5E7FCF7F9FBD2E7CD
:10738000624B197D9878FCF7AFFCCCE7FCF7CCFB9F
:107390000020FBF70FFB0021002000F031FFC2E7C7
:1073A0005A4B187DFCF7AAFBBDE7FCF7E3F9BAE7F7
:1073B000FCF7DAF9B7E7FCF7C5F9B4E7FCF710FA20
:1073C000B1E7FDF725FBAEE7FDF712FBABE7FDF7F5
:1073D000EDFAA8E7FDF7DAFAA5E7FDF7CBFAA2E7A1
:1073E000FDF7BCFA9FE7FDF7A5FA9CE7FDF768FA01
:1073F00099E7FDF757FA96E7FDF7CCF993E7FDF724
:1074000027F990E7FDF782F88DE7FCF7B9FF8AE7E7
:10741000FCF714FF87E7FCF76DFE84E7FCF766F9DD
:1074200081E7FCF731FE7EE7FCF71AFE7BE7FCF70D
:1074300003FB78E7FCF778F975E7FCF747F972E7A3
:10744000FCF78AFA6FE7FCF7B9FD6CE7FCF77EFD05
:1074500069E7FCF761FD66E7FCF7C8FC63E7FCF74A
:10746000F9FC60E7FCF7E2FD5DE7FCF7C5FD5AE7D4
:10747000FCF77EFC57E7FCF71FFC54E7FCF7BCFB6E
:1074800051E7FCF7C3FB4EE7FCF706FB4BE7FCF7C5
:1074900007FA48E7FFF77AFE45E7FFF75FFE42E7A6
:1074A000FFF736FB3FE701929D785A78010001AB68
:1074B0002800FDF7D1FF2070019B636033E79878C7
:1074C000FDF7EEFE2FE79878002100F0F3FE2AE7A3
:1074D0005142987800F0EEFE25E79878110000F010
:1074E000E9FE20E7022323701DE7C046A8F9FF1F2D
:1074F0009CFBFF1F9CF5000000FFFF000081920035
:10750000D6C5B4A3D20400002CF1FF1F4CF9FF1F15
:10751000F0B5DE4657464E464546E0B5A94B87B026
:107520001B78002B5CD0FB22A74E3378991F1142A9
:1075300056D0EB3A93430F2B52D00023A34CA44ECA
:10754000A3733370637B02AD002B5CD00120FBF78B
:10755000E3FB2800FBF7A0FC002859D003F08CFCCB
:107560002B7A994E33706B7A7370AB7AB370EB7A77
:10757000F3712B7BB3716B7B7371AB7B33716B7866
:10758000E3732B78072B00D1BEE00223A373914F46
:107590003B785A1E012A00D8E7E1052B00D1E4E12F
:1075A00001228D4B1A706B46DD1D2800FCF756F842
:1075B000002800D0E6E03A78A37B04211800884335
:1075C0000100042A39D1804E32787F2A35D800292B
:1075D0003CD0FD22063B134238D0FCF70DFC35E0D1
:1075E0007A4C02ADA27B531ED9B2012945D9784EFF
:1075F000032A32D0042A00D10AE20023A373337095
:10760000637B002BA2D12800FBF746FC0028A5D104
:107610006B46DD1D2800FCF721F8002800D066E14C
:107620006C4F3A78531E012B00D8BCE0A37B042199
:10763000180088430100042AC5D0002904D0FD2188
:107640009A1F0A4200D0D5E0092B3CD007B03CBCC1
:1076500090469946A246AB46F0BD3378002B56D0F3
:10766000012BCAD15D4B002798464346D85D0137B0
:10767000FBF7DAFF092FF8D1BFE75949544ECA6822
:107680006A605A1E934107332B70E37B32786B702C
:107690000023AB70002A30D18B682B72514B1978C4
:1076A00069725978A972D979E972997929735979E6
:1076B00069731B79EA73AB732800FBF74BFC002856
:1076C000C4D0A27B94E73B78022B13D0464A1168C2
:1076D0000029BBD0012BB9D1444B454C1868236815
:1076E000834207D0002301338B42AFD09A00A258C7
:1076F0008242F8D105233B70A8E7012A00D1BDE101
:10770000022A00D179E7D7E7063BA3733FE7344B62
:10771000987899465F78334BC71998461B78FF18BD
:1077200043465B78FF184346DB79FF1843469B7955
:10773000FF1843465B79FF1843461B79FF18FBF798
:1077400073FF4B465878FBF76FFF43461878FBF7FB
:107750006BFF43465878FBF767FF4346D879FBF742
:1077600063FF43469879FBF75FFF43465879FBF781
:107770005BFF4346FFB21879FBF756FF3800FBF773
:1077800053FF3AE701239846FBF786FF061E00D118
:10779000B5E0012323742B7823754346002B00D1D9
:1077A0003FE73A7808E78022104B120118689042B0
:1077B00000D86EE100233B70A37B042219009143A3
:1077C0003BE7C04628FBFF1FA8F9FF1F2CF1FF1F56
:1077D000C8FAFF1F5DFBFF1F29FBFF1FCCFAFF1F2D
:1077E0004CF9FF1F9CFBFF1F60FBFF1FF8FAFF1FF8
:1077F000FCFAFF1FFFF77EFDA37B092B00D025E7D6
:10780000FBF7CCFAC54DC64B2A689846801AC217BA
:107810001B6880185040984207D9C2480378012B52
:1078200000D128E1FBF7BAFA2860FBF7B7FA434624
:107830006A685B68801AC21780185040984207D95E
:10784000B8484378012B00D112E1FBF7A7FA686032
:10785000FBF7A4FA4346AA689B68801AC2178018EF
:107860005040984207D9AF488378012B00D1FCE003
:10787000FBF794FAA860002000F0E6FE2023E25C0B
:10788000002A08D1002806D00132A648E254C37865
:10789000012B00D1E6E0002000F0D6FE002801D147
:1078A0002023E0549F4B2726002599469A469B4665
:1078B00007E0032B47D0012B4DD001350136082DB1
:1078C00057D0E8B2FBF704F9635D8342F5D0424636
:1078D0002B1D9B00D3586055022BEAD10028ECD118
:1078E0004A46925D012AE8D14A469355E5E70023CE
:1078F0008D4F9846FBF7D0FE061E00D049E7227C4C
:107900002978531CDBB2A21823741175092B00D0FF
:1079100043E7207403F0B0FA844B227D5B789342F6
:1079200000D048E621000023143100E0725CD31837
:107930000136DBB2082EF9D1227F9A4200D115E13F
:107940000423A37382E653469B5D012BB5D15246B7
:1079500001339355B1E70028AFD05B469B5D012B07
:10796000ABD15A4601339355A7E70022704B1A70EA
:1079700019E601210020FBF7D7F8237A834212D0C1
:10798000434620701B7BDBB2022B00D194E0032B1B
:1079900003D0012B07D1002805D06248C37E012BFC
:1079A00001D10133C37600210020FBF7BDF8237B12
:1079B000834212D0434620709B7BDBB2022B00D166
:1079C00084E0032B03D0012B07D1002805D05548B4
:1079D000037F012B01D101330377564B1B78002B1A
:1079E00014D0554B98461B78002B0FD1534A4D4865
:1079F000002503E0013304322F2B07D0C15C02299C
:107A0000F8D111684E1C69D1C554F3E7A37B1BE67E
:107A100000234B4F033A7B707B60444B3A7099468E
:107A200098785B78C3180133DBB29846FBF7FCFD0E
:107A30004B465878FBF7F8FD3878FBF7F5FD78787A
:107A4000FBF7F2FDF879FBF7EFFDB879FBF7ECFDFA
:107A50007879FBF7E9FD3879FBF7E6FD4046FBF75F
:107A6000E3FDCAE50133C37015E701338370FFE618
:107A700001334370E9E601330370D3E6314A002352
:107A8000904641460133C95CEA18D171082BF8D100
:107A900012E62D4E421C31001A60FBF703FC09234D
:107AA000A3730122224B1A703A78042A00D0A1E66F
:107AB000A37B1900914387E5002800D073E719489C
:107AC000C27E012A00D06EE7C3766CE7002884D11D
:107AD0001448027F012A80D103777EE71B481C4AA5
:107AE0000068137710601B480023006850601A4834
:107AF000056801609560194D2D68D560184D2E7888
:107B00002B701661174E013336685661164E366873
:107B1000966142461370A37B96E5C046B0FFFF1FF7
:107B20002CFBFF1F68FBFF1F5DFBFF1F4CF9FF1FB6
:107B300029FBFF1F9CF9FF1F5CFBFF1F08FAFF1FBB
:107B40009CFBFF1FCCFAFF1FA8F9FF1FC4FAFF1F01
:107B50007CF9FF1FA8FBFF1FF8FAFF1FB0F9FF1FFA
:107B6000A4F9FF1F24FBFF1FACFFFF1F637D114E15
:107B70003370A37D7370E37DB370237EF371637EF6
:107B8000B371A37E7371E37E3371FBF707F90022B3
:107B9000094B1860094B1A700323A3733B785A1ED4
:107BA000012A02D9052B00D07BE70022044B1A7072
:107BB0007AE7C046A8F9FF1F98FBFF1FA4FBFF1F31
:107BC00029FBFF1FF0B51F4C83B06B4622000E004F
:107BD00082CA82C31C4B42786D461A7082785A70F2
:107BE000C2789A700279DA7142799A7182795A71FF
:107BF000C2791A710022154B1A70FFF77BFB144BE8
:107C00001B78002B0ED0012B03D00CCD0CC403B07D
:107C1000F0BD00230F49CA185278F2540133082BE3
:107C2000F9D1F2E7337073702378B3706378F3702F
:107C3000E3793371A37973716379B3712379F37144
:107C4000E3E7C0469CFBFF1FA8F9FF1F29FBFF1FAE
:107C5000C8FAFF1FCCFAFF1F0123802207495B42AD
:107C60008B500132FF328B50002000231A00C032AB
:107C7000920001335050082BF8D1704700E100E02A
:107C8000074A084B116810B50B4007498B4200D0DA
:107C900010BD064B52689A42FAD1FDF741FAF7E758
:107CA000A8F9FF1F00FFFF0000819200D6C5B4A312
:107CB000044A054B52689A4202D10122034B5A737F
:107CC0007047C046A8F9FF1FD20400002CF1FF1F27
:107CD00010B50024174B184A1C70FF231370174A65
:107CE00017491370174A1370002200230A604B6073
:107CF00015490C6015490C6015490C6015490A605E
:107D00004B60154B1C60154B1C60154B1C60154BD4
:107D10001C60154B1C60154B1C60154B1C601548F6
:107D200003F066F88021144B490000201C80FCF70A
:107D3000D3FE10BD340000203C0000207400002061
:107D400028000020180000200C0000201400002053
:107D50001C0000200000002008000020100000206F
:107D60002000002068000020700000203800002063
:107D7000400000204800002050F1FF1F014B186810
:107D80007047C0463000002010B5124B1878FAF743
:107D900013FFB9235B0058430F4903F04BFB0F4B14
:107DA00018601823FF3398420FD83C2806D90420C6
:107DB000FCF7AAFE0220FCF7A7FE10BD0220FCF78C
:107DC00093FE0420FCF7A0FEF7E70420FCF78CFEEE
:107DD000F3E7C04605F0FF1FFF0F00003000002052
:107DE000014B8000C05870476C00002010B50400A3
:107DF000FAF7F6FD002800D010BD2000FCF7BCFE0D
:107E00000028F9D1802120004900FCF795FE0028C8
:107E1000F2D12000FAF7CEFDEEE7C046014B80001C
:107E2000C05870470C000020014B8000C0587047BC
:107E30000C000020C3000F491A1A12018A1810B54D
:107E4000147E012C0FD01B1A1B01CB181A006532AF
:107E50001278998A002A02D002F004F910BD02F0CB
:107E600001F94042FAE7D47D012CECD0918A02F06E
:107E7000F9F8F3E7D8F8FF1F10B5FFF7DBFF10BDE7
:107E8000014B8000C058704710000020014B80005B
:107E9000C058704768000020014B8000C0587047F0
:107EA00008000020C300181A014B0001C058704799
:107EB000D8F8FF1F0B4A70B50023914210D8C300B9
:107EC000094C1B1A82001B011218084D1951D200CF
:107ED000E31851519A7D4A43602102F011F80123C1
:107EE000180070BD400D0300D8F8FF1FACF8FF1F4D
:107EF000094A002391420CD8C3001B1A074A1B01F0
:107F0000D318596083001818054BC00018180123B6
:107F1000416118007047C046A0860100D8F8FF1FD5
:107F2000ACF8FF1F0300002001290FD8D800C01AA9
:107F3000074A000112189800C018064BC0001B1811
:107F40000120C9B23A322433117019707047C0460B
:107F5000D8F8FF1FACF8FF1F0D4B820070B504006E
:107F6000D05804F03BFA051CE0000A4B001B00014E
:107F70001818806E04F032FA011C281C03F052FF1E
:107F8000DE21890503F04EFF04F008FA70BDC046FB
:107F900070000020D8F8FF1F83000E4A1B18DB007A
:107FA000D31870B50400986804F018FA051CE000B6
:107FB000094B001B00011818806E04F00FFA011C19
:107FC000281C03F02FFFDE21890503F02BFF04F0AE
:107FD000E5F970BDACF8FF1FD8F8FF1F0D4B82000C
:107FE00070B50400D05804F0F9F9051CE0000A4B04
:107FF000001B00011818806E04F0F0F9011C281C09
:1080000003F010FFDE21890503F00CFF04F0C6F930
:1080100070BDC04638000020D8F8FF1F70B50400BE
:10802000080004F0DBF98F21C90503F0FBFEE60030
:10803000194B361B36019E19051CB06E04F0CEF9A3
:10804000011C281C03F0A6FD04F0A8F933006533D9
:108050001B780500002B16D0B27D6B214243200017
:1080600001F04EFF80212000C901FCF745FD0B4BBC
:10807000A000C5500A4BC55000190A4BC000181883
:108080008560456070BDB27D43425A436B2120003C
:1080900001F036FFE6E7C046D8F8FF1F38000020A1
:1080A00070000020ACF8FF1F802310B59B00040077
:1080B000994235D025DD8023DB00994212D0802300
:1080C0001B0199420DD1FCF707FD8E212000C9014B
:1080D000FCF712FD0122174B012120001A5501F077
:1080E00057FF10BDFCF7F8FC96212000C901FCF7F2
:1080F00003FD03220F4B022120001A5501F048FF17
:10810000EFE7013BFF3B9942EBD1FCF7E5FC9C21FB
:108110002000C901FCF7F0FC0022064B1A55E0E7ED
:10812000FCF7DAFC9A212000C901FCF7E5FC0222E9
:10813000E0E7C0463400002010B5274B1878FAF766
:108140003BFD04F09BF905F04FFF02000B002348B4
:10815000234904F0E9FC214A224B05F099FB05F084
:1081600095FF214903F016FD05F03EFF06F0B6F934
:1081700000221E4B05F00CF900221D4B04F0C4F93F
:1081800002000B0000201B4904F0CEFC1A4B002219
:1081900005F07EFB05F07AFF04F000F9174B18603C
:1081A000772802DC642811DD10BD08210020FCF7CF
:1081B00093FC802100204900FFF776FF002100207A
:1081C000FAF71AFC0020FAF7FDFBEDE70821002082
:1081D000FCF792FCE8E7C04604F0FF1F9A999999D2
:1081E0009999C140999901400000204100A0724036
:1081F00000D4AA40C83A2F41001071406C00002002
:10820000C3001B1A124A1B01D3181A7E10B50400B2
:108210000020002A07D0012A15D00E4B0E4ACB1899
:108220000020934200D910BD0C4AA3009950802130
:108230000B4A090198502000FFF736FF2000FFF796
:10824000D5FD0120EFE7DB7D012BECD1E5E7C04652
:10825000D8F8FF1F8813000010270000140000202A
:108260001C000020C3001B1A0D4A1B01D3181B7EE3
:1082700010B5012B12D90B4B0B4CCB180022A3428B
:1082800001D9100010BD094C83001A51084A9950B9
:1082900080210901FFF708FF0122F2E70022F0E741
:1082A000D8F8FF1F881300001027000014000020DA
:1082B0001C000020C3001B1A0D4A1B01D3181B7E93
:1082C00010B504000020002B04D00A4B0A4ACB183A
:1082D000934200D910BD094BA200D150802120004B
:1082E0008900FFF7E1FE2000FFF780FD0120F1E7A4
:1082F000D8F8FF1F400D0300801A06001000002070
:10830000C30070B51B1A144D1B01ED182B7E040021
:10831000002B20D0080004F061F88F21C90503F07C
:1083200081FD061CA86E04F059F8011C301C03F0F6
:1083300031FC04F033F88021084BA500E850C90156
:108340002000FCF7D9FB80212000C900FFF7ACFE1C
:108350002000FFF74BFD70BDD8F8FF1F7000002014
:1083600070B504000E4B8200D0580D0004F036F8B2
:10837000E3000C4A1B1B1B01D318061C986E04F06B
:108380002DF8011C301C03F04DFDDE21890503F0A2
:1083900049FD04F003F841192000FFF7B1FF70BD5B
:1083A00038000020D8F8FF1F10B5040002F07EF856
:1083B000E3001B1B024A1B01D318987510BDC04671
:1083C000D8F8FF1F10B5C3001B1A044A1B01C9B21D
:1083D000D318997502F070F810BDC046D8F8FF1F89
:1083E00010B5C3001B1A044C1B01E3180A00D96026
:1083F000998A01F0C1FE10BDD8F8FF1FC300181AFA
:10840000024B00011818C0687047C046D8F8FF1F1B
:1084100010B50023032908D8C3001B1A044A1B0106
:10842000D318D97502F030F80123180010BDC046EA
:10843000D8F8FF1F10B5040002F01EF8E3001B1B64
:10844000024A1B01D318D87510BDC046D8F8FF1FCB
:108450000023012907D8C3001B1A04481B01C018B8
:1084600001236530017018007047C046D8F8FF1F1F
:10847000C3001B1A02481B01C01865300078704702
:10848000D8F8FF1F10B50024042911D8C3001B1A07
:10849000084A1B01D31819760134012908D000219C
:1084A000054B8200D15000230022643101F056FDBB
:1084B000200010BDD8F8FF1F1C000020C300181AB0
:1084C000024B00011818007E7047C046D8F8FF1F05
:1084D0000023022906D8C300181A034B00011818FC
:1084E0000123417618007047D8F8FF1FC300181AFF
:1084F000024B00011818407E7047C046D8F8FF1F95
:108500000023022906D8C300181A034B00011818CB
:108510000123817618007047D8F8FF1FC300181A8E
:10852000024B00011818807E7047C046D8F8FF1F24
:1085300010B5232101F0C2FC00B210BD10B53921E5
:1085400001F0BCFC00B210BD10B52A2101F0B6FC50
:10855000001410BDF8B5C6001C4F331A1B01FB18E0
:108560001A003532157836336A1E95411B7804009F
:10857000ADB2002B02D080235B011D43331B1B01D6
:10858000FB1837331B78002B02D080235B001D4380
:108590003321200001F092FC020C12042A43200037
:1085A000332101F0ADFC3721200001F087FC361BA0
:1085B0003601BE193823F25E0004000C1204024397
:1085C0003721200001F09CFCF8BDC046D8F8FF1F01
:1085D000C3001B1A03481B01C0183C3003788B43AF
:1085E00003707047D8F8FF1FC200121A044B120123
:1085F0009B183C3318780840411E8841C0B2704730
:10860000D8F8FF1F70B50125C3001B1A074C1B01CA
:10861000E4183C3423781D4207D00021FFF7FEFC0C
:1086200023785A0701D5AB43237070BDD8F8FF1FDC
:1086300010B52821040001F041FC002802D02000E0
:10864000FFF7E0FF10BDC04610B5FCF789FA400403
:10865000C00F10BDC2003B49131A1B01CB181B7E73
:1086600010B50400042B19D837489B00C3589F4607
:10867000121B12018A18D37D0322012B4CD05221E8
:10868000200001F03DFC802120000901FCF754FA94
:10869000414241412000013101F07AFC10BD121B22
:1086A00012018A18D37D0122012BE8D1200000227B
:1086B000522101F053FC0023200000221C2101F074
:1086C0004DFC20000122512101F01AFC0122502111
:1086D000200001F015FCE1E720000022242101F038
:1086E0000FFC01222000522101F00AFC2000082189
:1086F00001F04EFC00222121200001F001FCCDE719
:1087000020000222522101F0FBFB0121200001F098
:108710003FFCC3E70522B2E720000022522101F00E
:108720001DFC0023200000221C2101F017FC20006A
:108730000322512101F0E4FB03225021200001F02B
:10874000DFFBABE7D8F8FF1F9CF90000C3001B1A42
:108750000C4A1B01D3185B7E10B5012B0DD0002BEA
:1087600006D0022B03D10122502101F0C9FB10BD1C
:108770000022502101F0C4FBF9E70322502101F04F
:10878000BFFBF4E7D8F8FF1FC3001B1A0C4A1B01FC
:10879000D3189B7E10B5012B0DD0002B06D0022BD9
:1087A00003D10122512101F0ABFB10BD0022512168
:1087B00001F0A6FBF9E70322512101F0A1FBF4E748
:1087C000D8F8FF1FF0B54F464646D6460400C0B560
:1087D0005A4BE5009946185C594E2B1B1B01F318A8
:1087E0001A7E584F90425BD0032A5FD02B1B1B018F
:1087F000F3189B7E9C46002398466346012B6ED05F
:10880000042A29D02B1B1B01F3189B7E022B23D09B
:108810004B461A5563463B554346002B2BD120004F
:10882000FFF718FF802120000902FCF755F920000E
:10883000FFF7AAFF2D1B444F2D0175193A5D6B7E82
:108840009A4204D02000FFF781FF6B7E3B551CBC91
:1088500090469946A246F0BD0428D9D03B5D022B34
:10886000D6D001202B1B1B01F318313318704B4657
:108870001A5563463B550021344A630099528021C2
:1088800020000901FCF758F9414241412000013123
:1088900001F07EFB802120000902FCF72DF9C6E7DC
:1088A000395D9B7E9942C5D0032A9FD103281ED0F3
:1088B0003B5D012B33D02B1B1B019A46B244534620
:1088C000D97D01291FD92A218C4629398846D444CB
:1088D000614643460B7053469B7E9C4690E70328B7
:1088E000E6D1042A03D13B5D022BBAD106E02B1B53
:1088F0001B01F3189B7E9C46022B18D04B461A5541
:1089000063463B558BE72A239C4600239846D44474
:1089100063464146197053469B7E9C4670E72B1B6D
:108920001B01F3189B7E9C460023984668E73B5D3D
:10893000022B96D149463B550A5570E73C00002072
:10894000D8F8FF1F180000207400002050F1FF1F0E
:10895000F0B54F464646D646C0B51F000B7804001A
:108960000D001600012B42D0002B3CD0022B06D06C
:1089700000230B701CBC90469946A246F0BDFAF746
:108980002FF800286DD0654B9946630098464B46FA
:10899000424641469B5A4A4601339BB25352632B8F
:1089A00065D9C72B00D896E02C22FF32934200D81D
:1089B000A1E09022FF32934200D8A0E0F422FF32DF
:1089C000934200D89EE0564A934200D89EE0554A12
:1089D000934200D89DE00021534A8A46934249D8E9
:1089E000524B9A4646E04D4A4400A352C2E7002348
:1089F0000122292101F0B2FA012300225221200094
:108A000001F0ACFA002300221C21200001F0A6FA9C
:108A10000121200001F0BCFA6421200001F04EFA8F
:108A20000204120C6421200001F06AFA6421200083
:108A300001F044FAE3003E4A1B1B1B01D3189A685D
:108A4000998A0600100202F07FFD360C0204120C17
:108A5000360432436421200001F052FA02232B70C5
:108A600088E701232B702D4B6400E05282E78023BE
:108A7000DB019A461C21200001F020FA5346020C2B
:108A800012041A431C21200001F03AFA4B464246D8
:108A90009B5AB34200D26DE7002F1FD1244EE30052
:108AA0001B1B1B01F618B18A0022200001F0AEFA50
:108AB0000022B18A200001F039FB80212000090149
:108AC000FCF73AF8414241412000013101F060FADF
:108AD00003232B704EE7174B9A46CBE70022272142
:108AE000200001F00DFA0021E300114E1A1B1201C3
:108AF000B2181185D4E780239B019A46BAE70E4B42
:108B00009A46B7E780235B019A46B3E70B4B9A4638
:108B1000B0E780231B019A46ACE7C04650F1FF1F27
:108B200057020000BB0200001F030000FFF7000017
:108B3000D8F8FF1FFFBF0000FFDF0000FFEF0000BD
:108B4000401A00B27047C046F0B5D6464F4646467A
:108B5000C0B50B7804000D00012B35D0002B2BD0B5
:108B6000022B2ED1644B1B5C9A1E012A53D9012B78
:108B700067D000223921200001F0E2F95F4F022284
:108B8000BB5E02B29A4217D09BB2C01A00B2C60FA7
:108B9000361801222A21761020009E1901F0D0F902
:108BA000BB88B6B2C31AF31A9BB201222921200056
:108BB00001F0D4F900232B701CBC90469946A246C4
:108BC000F0BD00230B70F7E7332101F077F94C4A31
:108BD00033210240200001F093F9002301222921D2
:108BE000200001F0BBF900223921200001F0A8F992
:108BF000424F0600788001222A21200001F0A0F9CE
:108C0000331A9BB2012229212000BB8001F0A6F972
:108C100002232B70D0E7C6003A4F331A1B01FB1812
:108C200065331B788200002B54D0374BD258361B4B
:108C30003601BF19BB7D66215A43200001F060F95F
:108C400097E7C6002F4F331A1B01FB1865331B78BB
:108C5000002B43D0830099464A462C4B9B5898469C
:108C60006421200001F02AF9434682461802331B92
:108C70001B019846B8444346998A02F065FC534666
:108C800002041804000C02436421200001F038F9AA
:108C9000434665331B78002B28D14A461C4B985815
:108CA000434299466421200001F008F94B46804672
:108CB000361B3601BE19B18A180202F045FC434644
:108CC0000204180C0004120C02436421200001F07D
:108CD00017F94EE70C4BD2585242A8E78300994649
:108CE0004A460A4B985843429846B9E74A46084BC9
:108CF0009B589946D6E7C0463400002050F1FF1F2C
:108D0000FFFEFFFFD8F8FF1F6800002014000020BE
:108D10001C000020F0B5C6461C000026C300194DFB
:108D20001B1A00B51B01E818503000888A1A84B05D
:108D30005D5966612260D3172061002102F052FD67
:108D400002900391CB17FF2198468C46414660461E
:108D500001400A00029803990023801859416E428D
:108D60000B060095F717ED17000A1843019532001E
:108D70003B00091202F01CFBA06104B004BC904649
:108D8000F0BDC046D8F8FF1FF0B5DE464E4645465A
:108D90005746E0B58BB0FAF701F80600FAF704F889
:108DA000C54D0400AB68984202D0FBF791FFAC6060
:108DB000EB68F31ADA179B185340C04A934200DD60
:108DC00055E12B699E4200D14AE102F0A3F8002050
:108DD000FFF7F8FC6A21002001F070F8B84CA17D83
:108DE00002F0B2FB6523E35C0100002B00D141429D
:108DF000237E012B00D15CE1B24B082219609A4618
:108E00003B23B14FE35C00923A68B04800F040FF6A
:108E10003860002001F008FAA17D02F095FBAC4B10
:108E2000186098466523E35C002B02D1434640421C
:108E300018606921002001F041F8E37D020C012B4C
:108E400000D118E1A34BA449D3189BB28B4205D89B
:108E5000A04BC3189BB28B4200D895E23427002167
:108E60000122E35D03911A420CD03323E35C1A42E2
:108E700000D1B9E10020F9F757FE431E9841C3B273
:108E80000393E35D022200271A420BD03323E35CF5
:108E9000012100201A4200D1A0E1F9F745FE471E4A
:108EA000B841C7B280210020C900FBF745FE002869
:108EB0005BD03A23E35C002B00D023E1874B424692
:108EC0009B465946864B126809680020FFF722FF2F
:108ED000844B994618605B4642461B6812689B1A91
:108EE000DA179B185340626C934208DC53461B68A8
:108EF000DA179B185340226C934200DCACE1002F40
:108F000003D04B461B68002B06DB039B002B33D0A2
:108F10004B461B68002B2FDD00210020FFF720FAB5
:108F2000802100208900FBF707FE00282BD06E4B24
:108F300099466E4B4846984642464B461268DA6060
:108F400000F0D2FE4B46674A1B691360002F01D028
:108F5000002B04DB039A002A15D0002B13DD00231D
:108F6000424613604A4613610DE043461A685B4B64
:108F70001A605D4B9A601862802100208900FBF71F
:108F8000DBFD0028D3D1802100200901FBF7D4FDAF
:108F900000280DD05346544A1B68D3601361514AD0
:108FA0001360002F00D032E1039B002B00D03AE188
:108FB000802100204900FBF7BFFD00284DD1237E12
:108FC000012B00D14EE1023B022B46D8802100202C
:108FD0000902FBF7B1FD002800D12AE1444B1B78C0
:108FE0009A1E012A00D8A8E1012B36D16433E35C34
:108FF000002B00D0C4E13F4B1868434298466421DF
:10900000002000F05BFF43460700A18A180202F02F
:109010009BFA64213F0402043F0C3A43002000F015
:109020006FFF6523E35C002B00D095E1324B18689D
:10903000434298466421002000F040FF4346070069
:10904000A18A180202F080FA3F0C0204120C3F04BD
:109050003A436421002000F053FFFEF795FE2E6195
:109060000BB03CBC90469946A246AB46F0BDFFF71C
:1090700063F8EE60A5E6174B1749D3189BB28B42F5
:1090800000D9EBE6A18A12B24A43FF21D317194057
:10909000891809126523E35C002B00D1494208239B
:1090A000164F00933A68073B154800F0F1FD386011
:1090B000D4E60D4B19699FE650F1FF1FE70300004E
:1090C000D8F8FF1F2000002008000020000000202A
:1090D00038000020FF7C0000FEF900007000002036
:1090E0004800002068000020ACF8FF1F100000209E
:1090F00034000020140000201C0000200C00002080
:1091000028000020A74B9946A74B48469B465A4645
:109110004B4612685A6000F02BFE42464946A34B6C
:10912000126889680020FFF7F5FDA14B42461860E0
:109130004B46216812689B68C8179B1A07906068A5
:10914000DA1704930592069178220023C11702F0E2
:1091500049FB049B08900991D8171A184240D3176D
:109160000898099902F03EFB924A002302F016FB90
:10917000079B0890099106990A000800190002F05F
:1091800031FB00220090019108980999002300F01A
:10919000D3FC00F0E7FC059A002A30D1049B002B99
:1091A0002DD0236859421A0000F0BCFCC317C21826
:1091B0005A4051427E4B1B681800049302F0E4F8B9
:1091C0007B4B22681860236859424B461B69C018C4
:1091D00002F0DAF8784B994618607CE6F9F7A4FCBF
:1091E00047424741FFB25DE600210020F9F79CFCB1
:1091F000030058425841C3B20393E35D42E6049B27
:10920000059A134300D0A3E000210022D2E70020FA
:10921000FEF710FE002800DBC6E60023674A136055
:10922000674A1360C4E60020FEF704FE0028F4DC61
:10923000BEE62A23E35C002B05D0237E032B4BD014
:10924000A37E012B48D00020FFF704FA80210020E4
:109250000902FBF741FC00E780210020C901FBF770
:109260003BFC4CE6012100F093FEE37D012B3FD057
:10927000514B99461B689846002B02D0A3681B02ED
:1092800098466421002000F019FEA18A070040469C
:1092900002F05AF93F0C0204120C3F043A436421D5
:1092A000002000F02DFE6421002000F007FE0204E3
:1092B000120C6421002000F023FE6523E35C002BE8
:1092C00007D14B461A6852422121002000F018FEB7
:1092D000C3E64B461A68F7E7237F002B47D0022BE3
:1092E00000D0BAE6210000202A31FFF72DFCB4E6B9
:1092F0006433E35C002B33D1304B1868434298460B
:109300006421002000F0DAFD4346A18A070018021C
:1093100002F01AF93F0402043F0C3A436421002092
:1093200000F0EEFD6421002000F0C8FD020C1204E4
:109330006421002000F0E4FD8FE66523E35C002B50
:1093400012D11D4B1A685242A37D66215A4365E62D
:1093500023684042594226E7194B1B68984669E644
:10936000164B1B689846CBE7134B1A68ECE72100B5
:10937000E28B2A31009300200123FFF7E9FA6CE623
:109380000E4B1B6898463AE6A18A00B212B28218C8
:109390004A43D117C9B2237E89180912012B00D084
:1093A00078E67CE6ACF8FF1F700000204800002043
:1093B00040000020FFFF0000680000201400002093
:1093C0001C00002010B5040001F084F8E3001B1B12
:1093D000024A1B01D318188210BDC046D8F8FF1FDF
:1093E000084A10B50023914209D8C3001B1A064A47
:1093F0001B01D31889B2198201F072F801231800F9
:1094000010BDC046FFFF0000D8F8FF1F10B50400D4
:1094100001F074F8E3001B1B024A1B01D3185882A9
:1094200010BDC046D8F8FF1F084A10B5002391426E
:1094300009D8C3001B1A064A1B01D31889B25982E6
:1094400001F062F80123180010BDC046FFFF0000C4
:10945000D8F8FF1F7047C04610B5F9F79FFC014BC5
:10946000186010BD6CF1FF1FF8B55F4E84005F4BB4
:1094700032599A423CD837197A689A4238D8BA6831
:109480009A4235D8FA689A4232D83A699A422FD825
:10949000A6253300AD00454314335D190021280093
:1094A00001F01EF90223020000219A43280001F076
:1094B00007F9325928009200282101F001F97B6850
:1094C00028009A00292101F0FBF8BB6828009A00C7
:1094D0002A2101F0F5F8FB6828009A002B2101F001
:1094E000EFF83A692C219200280001F0E9F879E0C0
:1094F000A62335009B00584314352D180021280061
:1095000001F0EEF8022200210243280001F0D8F811
:10951000305902F0B3FF04F067FD0022344B03F032
:1095200037FFA222334B120603F0FEFA04F0E6FCEA
:10953000341902002821280001F0C2F8606802F006
:109540009DFF04F051FD0022294B03F021FFA222D0
:10955000284B120603F0E8FA04F0D0FC292102009F
:10956000280001F0ADF8A06802F088FF04F03CFD8F
:1095700000221F4B03F00CFFA2221E4B120603F029
:10958000D3FA04F0BBFC2A210200280001F098F86D
:10959000E06802F073FF04F027FD0022144B03F093
:1095A000F7FEA222134B120603F0BEFA04F0A6FC4B
:1095B0002B210200280001F083F8206902F05EFFF1
:1095C00004F012FD00220A4B03F0E2FEA222094B36
:1095D000120603F0A9FA04F091FC2C2102002800E5
:1095E00001F06EF8F8BDC04670F1FF1FFFFF3F00AD
:1095F00000004042941AED4270B5294D294B2C00D1
:10960000294A14342C3320002C32002101F020F997
:1096100020000022002101F053F82000234A1021ED
:1096200001F04EF820000022042101F049F820004A
:109630001F4A312101F044F820000422202101F0CA
:109640003FF820000022372101F03AF820000022E4
:10965000212101F035F8C826C822B60220001204E4
:10966000242101F02DF832002000282101F028F8F3
:1096700032002000292101F023F8C8230D4A1B02E3
:109680001364C0222000920201212B606B6001F064
:1096900017F8094A3521200001F012F870BDC046C4
:1096A00070F1FF1FF0F3FF1FF0F5FF1F050005002D
:1096B00040787D01F0F7FF1FFFFFFF7FA622920099
:1096C000424310B502481430801801F059F910BD1A
:1096D00070F1FF1F10B5A624A40044431100054BF0
:1096E000820005489B1814301A6C001901F08EF99D
:1096F00010BDC046F0F7FF1F70F1FF1FA6229200B9
:10970000424310B502481430801801F079F910BDB9
:1097100070F1FF1F2839C9B270B515290CD8634BF9
:1097200089005B589F46A621890041436048143058
:109730004018302100F0C4FF002070BDA621890030
:1097400041435B48143040182F2100F0B9FFF3E784
:10975000A62189004143564814304018372100F0B3
:10976000AFFFE9E7A6218900414351481430401872
:10977000212100F0A5FFDFE7A621890041434C48E5
:10978000120214304018242100F09AFFD4E7A621D9
:10979000890041434648120214304018222100F04B
:1097A0008FFFC9E7A624A40083006043404C414DCD
:1097B00014342418ED181202202120002A6400F02D
:1097C0008FFF4307B8D52A6C24211202200000F035
:1097D00077FFB1E7364B8100CA50FFF745FEABE794
:1097E000A62189004143324814304018332100F04B
:1097F00067FFA1E7A621890041432D481430401896
:10980000342100F05DFF97E7A621890041432848F5
:10981000120214304018252100F052FF8CE7244B2F
:1098200081005B189A60FFF71FFE85E7204B8100DF
:109830005B185A60FFF718FE7EE7A62189004143B6
:109840001B48120214304018272100F039FF73E73B
:10985000174B81005B18DA60FFF706FE6CE7A62164
:10986000890041431248120214304018262100F0AA
:1098700027FF61E70E4B81005B181A61FFF7F4FDCB
:109880005AE7A621890041430948143040182D2188
:1098900000F016FF50E7A621890041430448143028
:1098A00040182E2100F00CFF46E7C046B0F900003A
:1098B00070F1FF1FF0F7FF1F2839C9B210B514006F
:1098C0001A2900D9CEE0684B89005B589F46A62232
:1098D00092004243654833211430801800F000FFA5
:1098E0002060642010BD614B8000C3586420136069
:1098F000F8E75F4B80001818036C64201B1213609C
:10990000F0E7A622920042435848222114308018E2
:1099100000F0E6FE001220606420E3E7A622920039
:109920004243524824211430801800F0D9FE00121E
:1099300020606420D6E7A622920042434B482121B2
:109940001430801800F0CCFE20606420CAE7A62204
:1099500092004243454837211430801800F0C0FE81
:1099600020606420BEE7A622920042433F48302197
:109970001430801800F0B4FE20606420B2E7A62204
:109980009200424339482F211430801800F0A8FE7D
:1099900020606420A6E7A6229200424333482E218D
:1099A0001430801800F09CFE206064209AE7A62204
:1099B000920042432D482D211430801800F090FE73
:1099C000206064208EE7294B80001818036964200A
:1099D000136087E7A62292004243244826211430D0
:1099E000801800F07DFE0012206064207AE71F4B93
:1099F00080001818C3686420136073E7A6229200E1
:109A000042431A4827211430801800F069FE0012E2
:109A10002060642066E7154B8000181843686420B6
:109A200013605FE7114B800018188368642013608F
:109A300058E7A622920042430C4825211430801892
:109A400000F04EFE0012206064204BE7A622920038
:109A50004243064834211430801800F041FE206053
:109A600064203FE703203DE708FA000070F1FF1F84
:109A7000F0F7FF1FA62292004243054810B51430AC
:109A800080180F2100F02CFE0006C00F10BDC0464C
:109A900070F1FF1FA62292004243054810B5143012
:109AA00080180F2100F01CFEC005C00F10BDC0467D
:109AB00070F1FF1F10B5A624A4006043164C2221AC
:109AC00014342418200000F00BFE2121002812DBA2
:109AD000200000F005FE114B3521C218200000F0D7
:109AE000EFFD0F21200000F0FBFD80235B011840FB
:109AF0004342584110BD200000F0F2FD084B3521D3
:109B0000C218200000F0DCFD0F21200000F0E8FD6D
:109B1000C004C00FEEE7C04670F1FF1FFFFFFF7FDC
:109B200001000080904202DC0200884201DB10004C
:109B300070470A00FBE7C04630B5049C039DA14274
:109B40000CDC09D08B4202DD1000190030BD8B42C5
:109B5000FCD18242FAD9F7E7A842F3D928002100C4
:109B6000F4E7C04670B5041E00DA76E0FF2820DD79
:109B70003B4B98420DDD3B4B98421EDD3A4B9842E1
:109B80002FDD3A4B98425EDD394A0316D15C09025B
:109B90002EE0384B98421BDD374B98423DDD344A6E
:109BA0000312D05C0130030043439C4204DA0138C5
:109BB00002E02F4B185C000970BD304B98421EDD4F
:109BC0002F4B984244DD2A4A0314D15C09011DE061
:109BD0002C4B984227DD264A0311D05C80080130C7
:109BE000E1E7294B984229DC214A8314D15C4901E1
:109BF00020004D1C01F0A8FC2918491006E0234B59
:109C0000984216DC1A4A8312D15C490020004D1C90
:109C100001F09AFC28184010C5E7154A8311D05C62
:109C200040080130BFE7124A8310D05CC008013001
:109C3000B9E70F4A0313D15C8900E7E70C4A031523
:109C4000D15C8901D4E70A4A8315D15CC901CFE709
:109C5000074A8313D15CC900D8E701204042ABE733
:109C6000FFFF0000FFFFFF00FFFFFF0FFFFFFF3FB1
:109C700074FA0000FF0F0000FF3F0000FFFF0F001D
:109C8000FFFF3F00FF030000FFFFFF03FFFF030094
:109C9000D0B504AC24788A1AE31A9A401600D71774
:109CA00002684368B6185F4120235B420660476044
:109CB000E31802D438001841D0BD20233A00300008
:109CC0001B1B9A40E0401043F6E7C04601220023E8
:109CD00052420283253203604360C36003614361E3
:109CE000C361036283547047F0B5C646242300B5B0
:109CF000C35C0400002B24D0FA21C36805694669BF
:109D00005F1B9846FB17FF18890030005F4001F089
:109D10001BFC874202DAFA26B6007E43E369FA2189
:109D20009C4666448900300001F0F4FCE161A845DE
:109D300013DC08DA0D49300001F006FC2D1825610E
:109D400001E0C56805612368280059421A00FFF741
:109D5000E9FE206104BC9046F0BDFA213000890084
:109D600001F0F2FB2D182561EDE7C04618FCFFFF5E
:109D7000F0B5C646242300B5C35C82B00600002BB4
:109D800005D14368836002B004BC9046F0BD4368CF
:109D900082689F1A03687822984643694069D917F8
:109DA000002301F01FFDFB17FA185A40D31701F0EA
:109DB00019FD328B002301F0F1FC424604000D0036
:109DC00000234046002101F00DFD0022009001918A
:109DD000002320002900FFF7AFFEFFF7C3FE002F8E
:109DE00056DD32680021FFF79DFE0700FA21336936
:109DF0007469FD1A9846EB17ED18890020005D4044
:109E000001F0A2FB854202DAFA24A4006C43F36954
:109E1000FA219C4664448900200001F07BFCF1613A
:109E200047453FDDFA218900200001F08DFB804489
:109E300043463361FA22B3689200D917B068002311
:109E400001F0D0FC434604000D00DB174246308B86
:109E5000002101F0C7FC3C22002301F09FFC326A84
:109E6000D3178018594124184D41FA21E317E018FF
:109E700058408900002D19DB01F04CFC3162FA22B8
:109E8000002392002000290001F088FCB0607AE7EE
:109E9000002FABD03368404259420022FFF742FE08
:109EA0000700A3E74745C5DA0349BDE701F032FCE7
:109EB00049423162E3E7C04618FCFFFF7F2370B5DB
:109EC000050019400022FBF749F928000022002173
:109ED000FBF744F90022060200212800FBF73EF9B7
:109EE00030430402002228000021FBF737F9012249
:109EF000044300212800FBF731F92402204370BD00
:109F0000802370B50500140019430022FBF726F9E1
:109F1000210E28000022FBF721F921142800C9B2E4
:109F20000022FBF71BF921122800C9B20022FBF71F
:109F300015F92800E1B20122FBF710F970BDC04607
:109F400010B51400FFF7BAFF002C05D0000C012C4F
:109F500000D110BD0020FCE780B2FAE7F8B5170089
:109F600004000D001E00FFF7A9FF002F0BD0012FEA
:109F700003D10004000C3604304302002900200005
:109F8000FFF7BEFFF8BD000C00043043F5E7C04604
:109F900070B50C0063210500FFF790FFFF2302005E
:109FA0009A43280022436321FFF7AAFF70BDC046F1
:109FB00070B505000C000121FFF7EAFF2800A3B2ED
:109FC00001226421FFF7CAFF70BDC04670B56F2142
:109FD0000400FFF773FF002206006F212000FFF747
:109FE0008FFF6E212000FFF769FF0500320020007F
:109FF0006F21FFF785FF280070BDC04610B56921AD
:10A00000FFF75CFF001410BD0020704770B514000E
:10A010000E0001210500FFF7BBFF3100200201F017
:10A0200093FA012283B264212800FFF797FF70BDE5
:10A0300010B50C00FFF7CAFF4443FF20E317184098
:10A040000019001210BDC04610B50C006921FFF7C1
:10A0500035FF00144443FF20E31718400019001295
:10A0600010BDC046F0B5C6460D0000B56F21040016
:10A07000FFF724FF002280466F212000FFF740FFFA
:10A080006E212000FFF71AFF012206006F21200039
:10A09000FFF736FF6E212000FFF710FF0700424652
:10A0A00020006F21FFF72CFFFF20F6197543EB17F7
:10A0B00018404019001204BC9046F0BD10B50C00C9
:10A0C0006921FFF7FBFE011400B208184443FF208A
:10A0D000E31718400019001210BDC0460020704759
:10A0E00010B58BB200226421FFF738FF10BDC046C7
:10A0F00070B56F210400FFF7E1FE012206006F2119
:10A100002000FFF7FDFE6E212000FFF7D7FE0500BF
:10A11000320020006F21FFF7F3FE280070BDC0461B
:10A1200010B56921FFF7CAFE00B210BD10B50400DA
:10A13000100201F009FA002283B264212000FFF727
:10A140000DFF10BD10B50C00FFF7D2FF4443FF20F8
:10A15000E31718400019001210BDC04610B50C00DE
:10A160006921FFF7ABFE00B24443FF20E31718401C
:10A170000019001210BDC04610B50400100201F015
:10A18000E3F9002283B25E212000FFF7E7FE10BD55
:10A1900010B50C005E21FFF791FE0004000C604337
:10A1A000001210BD70B50D0004000221FFF7F0FE93
:10A1B0002A0066212000FFF7A3FE70BD10B56621BE
:10A1C000FFF77CFE10BDC04610B56A21FFF776FE92
:10A1D00010BDC0460020704770B50D00040003217B
:10A1E000FFF7D6FE2A0068212000FFF789FE70BD28
:10A1F00070B504000D000321FFF7CAFE6B2120009B
:10A20000FFF75CFE682142192000FFF779FE70BD60
:10A2100010B56821FFF752FE10BDC04610B50A0008
:10A220006B21FFF76DFE10BD10B56B21FFF746FEE9
:10A2300010BDC04600207047F8B50D0006A90E8875
:10A2400029780400012927D0002923D0022902D02F
:10A2500000232B70F8BD1988013189B21980914211
:10A26000F8D300222721FFF74BFE234E24217268EA
:10A270002000FFF745FE338900221C212000FFF754
:10A280006DFE3388002252212000FFF767FE032372
:10A290002B70DFE71980DDE75221FFF70FFE164F25
:10A2A000242138802000FFF709FE1C21786020005F
:10A2B000FFF704FE00233881012229212000FFF747
:10A2C0004DFE0123002252212000FFF747FE00230C
:10A2D000012224212000FFF741FE33000022242127
:10A2E0002000FFF73BFE002300221C212000FFF787
:10A2F00035FE02232B70ADE734F8FF1F401A00B281
:10A300007047C046F8B50B7804000D00012B2AD029
:10A31000002B26D0022B02D000230B70F8BD392170
:10A32000FFF7CCFD234F0A22BB5E02B29A42F5D062
:10A330009BB2C01A00B2C60F36182A217610200030
:10A340009E19FFF7BBFDBB89000CC31AB6B2F31A06
:10A350009BB2012229212000FFF700FE00232B7071
:10A36000DCE71380DAE73321FFF7A8FD124A332137
:10A3700002402000FFF7C4FD002301222921200014
:10A38000FFF7ECFD39212000FFF798FD094F06008B
:10A3900078812A212000FFF791FD000C331A9BB22F
:10A3A000012229212000BB81FFF7D8FD02232B7059
:10A3B000B4E7C04634F8FF1FFFFEFFFFF0B5C64606
:10A3C00000B5114D82B00E009846296908AB140003
:10A3D0001A880AAB07001B88B14202D0002C06D0B5
:10A3E0002E61022C09D002B004BC9046F0BD00934F
:10A3F0004146099BFFF720FFF2E7099A41463800E2
:10A40000FFF780FFEFE7C04634F8FF1F30B585B097
:10A410000AAD2D8808AC24880295099D0094019509
:10A42000FFF7CCFF05B030BD1378002B03D1002817
:10A4300002D0022800D07047012308701370FAE799
:10A4400070B514001D00914208D05221FFF758FD4D
:10A45000032C03D1049B1B78002B00D070BD02336A
:10A460009D43FBD1049A013B1370F7E710B500221E
:10A470001A21FFF745FD10BD10B51B21FFF71EFD8A
:10A480000014C0B210BDC04670B50C001B21050001
:10A49000FFF714FD044A24040240224328001B2134
:10A4A000FFF72EFD70BDC046FFFF00FF10B51B215A
:10A4B000FFF704FDC0B210BD70B50D001B210400F4
:10A4C000FFF7FCFC020C12042A431B212000FFF7BB
:10A4D00017FD70BD10B50921FFF7F0FC80B210BD6B
:10A4E00070B50D0009210400FFF7E8FC020C12040E
:10A4F0002A4309212000FFF703FD70BD10B5082194
:10A50000FFF7DCFC80B210BD70B50D00082104001F
:10A51000FFF7D4FC020C12042A4308212000FFF7A5
:10A52000EFFC70BD0904114370B505000C000A0072
:10A530005421FFF7E5FC280022005621FFF7E0FC3C
:10A5400070BDC04610B509040A435821FFF7D8FC76
:10A5500010BDC04610B509040A435A21FFF7D0FCCC
:10A5600010BDC046F0B5D6464F464646C0B59A46E1
:10A5700008AB10CB89461B781100050016009846E1
:10A58000FFF79CFC5246070031002800FFF7B8FC9B
:10A5900049462800FFF792FC43460440DC4028006F
:10A5A0003A003100FFF7ACFC20001CBC90469946F5
:10A5B000A246F0BD7F2370B5050019400022FAF7CE
:10A5C000D1FD280000220021FAF7CCFD002206026E
:10A5D00000212800FAF7C6FD3043040200222800BB
:10A5E0000021FAF7BFFD0122044300212800FAF7F9
:10A5F000B9FD2402204370BD802370B5050014000E
:10A6000019430022FAF7AEFD210E28000022FAF7C6
:10A61000A9FD21142800C9B20022FAF7A3FD2112D6
:10A620002800C9B20022FAF79DFD2800E1B20122FC
:10A63000FAF798FD70BDC046F0B5CE46474680B5E6
:10A6400083B01F000AAB1C780BAB1B781600984632
:10A6500080236A465B420B43137056709770D47028
:10A660006B4642461A71842302689B0005008946A6
:10A67000D05C69460522FAF72FFD6B461A78A423B1
:10A680009B00EA542A684B4694467F2142462402A6
:10A69000194014433F048B003C4336066344344363
:10A6A0005C6084239B009C4608226D1865442B78CF
:10A6B00013432B7003B00CBC90469946F0BDC046C6
:10A6C00030B5131483B0150ED4B212120194D4B263
:10A6D000DBB200942A00FFF7AFFF03B030BDC046E5
:10A6E00070B584267F24B600B4460C400319634439
:10A6F0001B7882B00500DB0705D40168A4000C19A3
:10A70000606802B070BD6B461C7003680522985DDE
:10A710006946FAF7E1FC6B461C702B680522985DD0
:10A720006946FAF7D9FC6B461A78A4239B00EA54D1
:10A730006B4658789B7800061B0418436B461B79C0
:10A7400018436B46DB781B021843DAE7F0B5464640
:10A75000D6464F46C0B5541E86B080460E0092467F
:10A76000072C57D8DC22036852009F58043A9B58A4
:10A7700004ADAD3AFF3A341900212800994603F0A0
:10A78000A5FE23002A00013E1978013B1170013219
:10A790009E42F9D153460393042B41D86978287817
:10A7A000AB78EA780190009140466C21FFF744FFB6
:10A7B000002303930133039A03930133652BFAD1EA
:10A7C0005346042B37D86E214046FFF789FF030A12
:10A7D0006B70030CAB700023C2B2000E2A70E870DD
:10A7E000039300E02A782270013C0135A642F9D19A
:10A7F0003A0EF9B23B143F12FFB2DBB2019100975F
:10A800006D214046FFF718FF43461A68DA23494690
:10A810005B00D15006B01CBC90469946A246F0BDE4
:10A820002979AB79EA7901916979404600916D21E6
:10A83000FFF702FFB2E76F214046FFF751FF030A1F
:10A8400028716B71030C000EAB71E871BBE7C04659
:10A8500030B583250024AD004460C460846002608C
:10A860005451043551554119084D5470147010302D
:10A870006A1C4334803501E0147801320C7010CB2F
:10A88000013110C0AA42F7D130BDC0468CFB000098
:10A89000F0B54746CE4680B51D4F00240021BC468A
:10A8A00002E0013180292AD084239B00CB18C35CAD
:10A8B000422BF6D126000E2C25D8E300FD5CB846CD
:10A8C0008D420FDA0134E3B2DA00BA1805E01578E8
:10A8D0001E00083201338D4204DADCB20F2CF6D1AF
:10A8E00000250F26A942DCD10268F60091464644B5
:10A8F0008B0072684B4401315A608029D4D10CBC62
:10A9000090469946F0BD6246E300E046D55CE9E733
:10A910000CFC000010B5046800232278002A12D134
:10A92000A42284239200944608219B00C31860440B
:10A930001A788A431A7001338342F9D101232370B4
:10A94000002363700133180010BDC0460368002067
:10A950001A78002A03D1023258701A7001307047F9
:10A9600080239B001030CA1808C908C09142FBD14F
:10A970007047C046832302689B00D1507047C04691
:10A9800030B50C0083B020210500FFF7A9FE042399
:10A990009843020EC1B203140012C0B2DBB201919F
:10A9A000009020212800FFF747FEE317E2185A40E5
:10A9B0000D4B9A420DDD002C12DB002412237A226B
:10A9C00000210094019128002431FFF735FE03B0E7
:10A9D00030BD24022314220E2412DBB2E4B2EFE7CE
:10A9E0000024EE238522EBE700127A0010B5FFF772
:10A9F000C7FF10BD10B54942FFF7C2FF10BDC046EA
:10AA000010B50021FFF7BCFF10BDC04670B50C00AB
:10AA100082B0202116000500FFF762FE04231843D0
:10AA2000020EC1B203140012C0B2DBB20191009059
:10AA300020212800FFF700FEF317F2185A40144BAC
:10AA40009A4219DD002E1EDB002612237A220021F5
:10AA50002800019100962431FFF7EEFD220EE1B2AD
:10AA600023142412E4B20191DBB2009437212800B0
:10AA7000FFF7E2FD02B070BD36023314320E36121B
:10AA8000DBB2F6B2E3E70026EE238522DFE7C0461D
:10AA900000127A0070B50D00212116000400FFF7A6
:10AAA0001FFE2B683200C11829602000FFF7AEFF9F
:10AAB00070BDC046C317C2185A40054B9A4203DD09
:10AAC000002803DB034870470002FCE70248FAE76E
:10AAD00000127A000000127A0000EE85F0B5884D71
:10AAE00083B004002B7800294BD0002B49D10133CF
:10AAF0002B7028212000FFF7F3FD292107002000FB
:10AB0000FFF7EEFD202106002000FFF7E9FD0423FA
:10AB10006860019300232000009300222021FFF7AA
:10AB20008BFDFA2338009B009F4200D2D3E0C1B2D4
:10AB30000314020E0012C0B2DBB201910090282172
:10AB40002000FFF779FDFA2330009B009E4200D2DF
:10AB50001800020EC1B203140012C0B2DBB20191A0
:10AB6000009029212000FFF767FD002320000193BA
:10AB7000009300222421FFF75FFD022300202B70A9
:10AB800050E0052B4DD85F4A9B00D3589F460721C4
:10AB90002000FFF7A5FD5C4B1840020EC1B2031464
:10ABA0000012C0B2DBB20191009007212000FFF734
:10ABB00043FD07212000FFF793FD544B0340802005
:10ABC000C0031843020EC1B203140012C0B2DBB2BC
:10ABD0000191009007212000FFF72EFD2221200087
:10ABE000FFF77EFD061E1CD1042300900193002276
:10ABF000002320212000FFF71FFD10230196009362
:10AC00000022173324212000FFF716FD79212000B0
:10AC1000FF26FFF765FD30407F3E361A5DD10323E6
:10AC20002B70002003B0F0BD002301202B70F9E74A
:10AC300007212000FFF754FD80235B041843C1B2B5
:10AC40000314020E0012C0B2DBB201910090072182
:10AC50002000FFF7F1FC042300202B70E2E700291D
:10AC6000DFD107312000FFF73BFD274B1840020ED4
:10AC7000C1B203140012C0B2DBB2019100900721EF
:10AC80002000FFF7D9FC07212000FFF729FD1F4B0B
:10AC900003408020C0031843020EC1B20314001207
:10ACA000C0B2DBB20191009007212000FFF7C4FC85
:10ACB00004216B681943C8B20B140A0E0912C9B2F9
:10ACC000DBB20190009120002021FFF7B5FC0523A5
:10ACD00000202B70A6E7180029E721212000FFF7AC
:10ACE000FFFC3618F1B23314320E3612F6B201916F
:10ACF0002000DBB200963721FFF79EFC002091E791
:10AD000048F8FF1F74FB0000FFFFFFFEFFFF3FFF3F
:10AD100070B5056882B02B7804000E00002B08D1B6
:10AD2000C3688B4203D00021FFF7D8FEE66002B073
:10AD300070BD022B2BD069784BB2002B1BDB842219
:10AD400092009446431863441A7842231340022B1E
:10AD500035D0422208E08420800084466318634492
:10AD60001B781340022B2AD00131C9B24BB2697053
:10AD7000002BF0DA256883239B00EB58002B03D0CF
:10AD8000297820009847256800232B70CFE76B783F
:10AD900002215AB24820002AEDDB8426B600B446D0
:10ADA000E21862441278114202D00240402A19D1BE
:10ADB0000133DBB25AB26B70002AEEDADAE7230015
:10ADC00010338A00D0580314020EC6B20012C0B26B
:10ADD000DBB2009001962000FFF72EFC6B78013368
:10ADE0006B70A4E769784BB2002BC3DB2B1DE8E73F
:10ADF00030B500230025002403608460C5608361B2
:10AE000030BDC046104B1A68821AD11752184A40FA
:10AE10000E498A4216DD9A6819695A600022D96083
:10AE200099699A605961196A1A61D961996A9A6136
:10AE30005962196B1A62D962996B9A621A635963E3
:10AE40009A6318607047C04650F8FF1FE703000080
:10AE5000024A9368013393607047C04650F8FF1F61
:10AE6000014B98687047C04650F8FF1F014B586867
:10AE70007047C04650F8FF1F024A1369013313613F
:10AE80007047C04650F8FF1F014BD8687047C04656
:10AE900050F8FF1F024A9369013393617047C0461F
:10AEA00050F8FF1F014B58697047C04650F8FF1F0C
:10AEB000024A136A013313627047C04650F8FF1FFD
:10AEC000014BD8697047C04650F8FF1F024A936A89
:10AED000013393627047C04650F8FF1F014B586A18
:10AEE0007047C04650F8FF1F024A136B01331363CB
:10AEF0007047C04650F8FF1F014BD86A7047C046E4
:10AF000050F8FF1F024B1B6B9800C01840007047A1
:10AF100050F8FF1F024A936B013393637047C0469A
:10AF200050F8FF1F014B586B7047C04650F8FF1F89
:10AF3000024B9B6B9800C0184000704750F8FF1FF1
:10AF4000014B18607047C0469C000020014B1868F8
:10AF50007047C0469C000020014B18607047C046F7
:10AF600094000020014B18687047C04694000020F0
:10AF7000014B18607047C04690000020014B1868D4
:10AF80007047C04690000020014B18607047C046D3
:10AF900088000020014B18687047C04688000020D8
:10AFA000014B18607047C04698000020014B18689C
:10AFB0007047C04698000020014B18607047C0469B
:10AFC0007C000020014B18687047C0467C000020C0
:10AFD000014B18607047C04684000020014B186880
:10AFE0007047C04684000020014B18607047C0467F
:10AFF00080000020014B18687047C0468000002088
:10B00000014B18607047C0468C000020014B186847
:10B010007047C0468C000020014B18607047C04646
:10B0200078000020014B18687047C0467800002067
:10B03000044B00225960012118701A725972DA60AB
:10B040007047C04694F8FF1F0022024B5A721A72D2
:10B05000DA60704794F8FF1F014B187A7047C046BA
:10B0600094F8FF1F014B587A7047C04694F8FF1FB1
:10B07000014BD8687047C04694F8FF1F0021064B6B
:10B080000068DA6819610132DA60824202D15972CD
:10B090001972D9607047C04694F8FF1F84B030B56C
:10B0A00083B00892154A07911549099313690968F5
:10B0B000013313618B4218DB137A002B15D004681F
:10B0C000D3689C4211DD41681D0107984919086049
:10B0D0000898013348600998D360886001900A9805
:10B0E000C860002111619C4204D003B030BC08BC90
:10B0F00004B0184751721172D160F6E794F8FF1F3F
:10B100001CF0FF1F00687047006800017047C046D0
:10B110000420704730B50400256801208D4202DD0F
:10B120000130032A00DD30BD6068920082180901F9
:10B13000525800201A60F6E70A2803D80B4A830009
:10B14000D3589F4600220A4B5A6170470322084B8E
:10B150005A61FAE7064B5861F7E70122044B5A613E
:10B16000F3E70222024B5A61EFE7C04684FC00007D
:10B1700094F8FF1F014B58697047C04694F8FF1FB1
:10B18000014B18607047C0461CF0FF1F014B186848
:10B190007047C0461CF0FF1F30B5134C2378062BB8
:10B1A00006D8124D9B00EB589F466368984207DD16
:10B1B000012323720023637230BD63688342F7DC8E
:10B1C000237A002BF8D0F5E763689342F8DDEFE7C8
:10B1D00063689A42ECDCF3E763688B42E8DCEFE7F4
:10B1E00063689942E4DCEBE794F8FF1FB0FC0000D1
:10B1F00070B50500414885421EDD414B9D4233DD5F
:10B20000404B9D423BDC404B9D4254DD3F4A2B1559
:10B21000D15C890128004C1C00F096F921184910D6
:10B2200028004C1C00F090F9201840100300434304
:10B230009D4208DA013806E0FF2D05DC002D5ADBBF
:10B24000324B585D000970BD314B9D422ADD314BB8
:10B250009D424ADD2D4A2B12D05C0130030043434E
:10B260009D42F0DA0138EEE72B4B9D4212DD2B4B6D
:10B270009D4230DD254A2B14D15C0901D0E7284BD3
:10B280009D421DDD274B9D42DDDC204A2B16D15C03
:10B290000902BFE7244B9D4222DD1C4A2B13D15CDF
:10B2A0008900BDE7214B9D420FDD184A2B11D05C70
:10B2B00080080130D2E7154AAB14D15C4901A9E7F7
:10B2C000124AAB15D15CC901A4E7104AAB10D05C9F
:10B2D000C0080130C2E70D4AAB13D15CC9009FE73B
:10B2E0000A4AAB12D15C49009AE7084AAB11D05C1C
:10B2F00040080130B2E701204042A4E7FFFF000010
:10B30000FFFFFF00FFFFFF0FFFFFFF03CCFC00006C
:10B31000FF0F0000FF3F0000FFFF0F00FFFF3F0097
:10B32000FFFFFF3F0080FE7FFFFF0300FF030000E1
:10B33000104A03000020934206D80F48834204D8E5
:10B34000FF2B0AD80D4AD05C70470D498B4208D9B3
:10B35000D31A0A4AD05C4042F6E7C01A074B185C81
:10B36000F2E7084A05489446C318634418784042F7
:10B37000EAE7C046FF030000FF010000CCFD00002B
:10B38000FF02000000FEFFFF904202DC0200884244
:10B3900001DB100070470A00FBE7C046904202D86C
:10B3A0000200884201D3100070470A00FBE7C04644
:10B3B00030B5049C039DA1420CDC09D08B4202DD18
:10B3C0001000190030BD8B42FCD18242FAD9F7E758
:10B3D000A842F3D928002100F4E7C04670B5140054
:10B3E0000E0000F0FBFF051C200001F047F8041CD4
:10B3F000011C281C00F0CEFB011C281C00F032FEB2
:10B40000051C300000F0EAFF211C00F0C3FB011C0A
:10B41000281C00F02DFA00F0C1FF70BD10B5029C91
:10B420008A1AE31A9A4003689C46624402602241E9
:10B43000100010BD002243088B4274D303098B42D5
:10B440005FD3030A8B4244D3030B8B4228D3030CF4
:10B450008B420DD3FF22090212BA030C8B4202D396
:10B460001212090265D0030B8B4219D300E0090ABE
:10B47000C30B8B4201D3CB03C01A5241830B8B42C7
:10B4800001D38B03C01A5241430B8B4201D34B03B0
:10B49000C01A5241030B8B4201D30B03C01A524115
:10B4A000C30A8B4201D3CB02C01A5241830A8B429A
:10B4B00001D38B02C01A5241430A8B4201D34B0283
:10B4C000C01A5241030A8B4201D30B02C01A5241E7
:10B4D000CDD2C3098B4201D3CB01C01A524183099B
:10B4E0008B4201D38B01C01A524143098B4201D3D5
:10B4F0004B01C01A524103098B4201D30B01C01A00
:10B500005241C3088B4201D3CB00C01A5241830879
:10B510008B4201D38B00C01A524143088B4201D3A6
:10B520004B00C01A5241411A00D201465241104606
:10B530007047FFE701B5002000F0F0F802BDC046FB
:10B540000029F7D076E7704703460B437FD40022EB
:10B5500043088B4274D303098B425FD3030A8B42A7
:10B5600044D3030B8B4228D3030C8B420DD3FF2211
:10B57000090212BA030C8B4202D31212090265D0DF
:10B58000030B8B4219D300E0090AC30B8B4201D392
:10B59000CB03C01A5241830B8B4201D38B03C01AD9
:10B5A0005241430B8B4201D34B03C01A5241030B50
:10B5B0008B4201D30B03C01A5241C30A8B4201D301
:10B5C000CB02C01A5241830A8B4201D38B02C01AAC
:10B5D0005241430A8B4201D34B02C01A5241030A23
:10B5E0008B4201D30B02C01A5241CDD2C3098B4208
:10B5F00001D3CB01C01A524183098B4201D38B0185
:10B60000C01A524143098B4201D34B01C01A524127
:10B6100003098B4201D30B01C01A5241C3088B426C
:10B6200001D3CB00C01A524183088B4201D38B0057
:10B63000C01A524143088B4201D34B00C01A5241F9
:10B64000411A00D201465241104670475DE0CA0FD0
:10B6500000D04942031000D34042534000229C4690
:10B6600003098B422DD3030A8B4212D3FC2289019A
:10B6700012BA030A8B420CD3890192118B4208D370
:10B68000890192118B4204D389013AD0921100E0D2
:10B690008909C3098B4201D3CB01C01A52418309E6
:10B6A0008B4201D38B01C01A524143098B4201D313
:10B6B0004B01C01A524103098B4201D30B01C01A3E
:10B6C0005241C3088B4201D3CB00C01A52418308B8
:10B6D0008B4201D38B00C01A5241D9D243088B420E
:10B6E00001D34B00C01A5241411A00D201466346B1
:10B6F00052415B10104601D34042002B00D5494215
:10B70000704763465B1000D3404201B5002000F053
:10B7100005F802BD0029F8D016E770477047C0460B
:10B720008446101C62468C46191C634600E0C046E5
:10B730001FB501F0CBFD002801D40021C8421FBD78
:10B7400010B501F025FD4042013010BD10B501F0EB
:10B75000BDFD002801DB002010BD012010BDC0464A
:10B7600010B501F0B3FD002801DD002010BD01205F
:10B7700010BDC04610B501F045FD002801DC0020D9
:10B7800010BD012010BDC04610B501F03BFD0028E2
:10B7900001DA002010BD012010BDC046002B15D1DC
:10B7A000002A13D1002906DB01DC002806D0002086
:10B7B000C043410802E080210906002007B4024886
:10B7C00001A14018029003BD55FFFFFF03B4684676
:10B7D00001B5029800F030F8019B9E4602B00CBC07
:10B7E0007047C046F0B5CE46474615042D0C2E00D6
:10B7F00080B50704140C3F0C9946030C7E435D434F
:10B80000674363437F19340CE4199C46A54203D96E
:10B8100080235B029846C4444B465143434336045D
:10B82000360C250C24046544A41959184919200024
:10B830000CBC90469946F0BDF0B583B016001F00D1
:10B840000090019102F0CAFC04000D0002000B0000
:10B8500030003900FFF7C6FF009A019B121A8B4196
:10B86000089920000A604B60290003B0F0BDC04673
:10B87000F0B5C6464E024702760A7B0A4400C50F61
:10B88000F7004800984600B5240E2A00DB00000EA1
:10B89000C90FBC468D4267D0221A002A00DCA5E001
:10B8A00000283AD1002F00D193E0511E002900D08A
:10B8B000BCE00124DB1B5A0146D59B019E093000E8
:10B8C00002F06EFC05388640844200DD9DE0041BDA
:10B8D000320020200134E240041BA64033005E1EEB
:10B8E000B341002413435A0704D00F221A40042AFC
:10B8F00000D004335A0129D50134FF2C00D181E056
:10B900002A009B015B0AE4B25B02E405580AD207F5
:10B910002043104304BC9046F0BDFF2CE3D08021AF
:10B920003800C904084384461B2A00DD82E0202039
:10B930006146D140821A604690400200501E82410A
:10B940000A439B1A5A01B8D45A07CED1DE082A00FE
:10B95000FF2C3AD1002E00D1AEE08023DB0333432D
:10B960005B025B0AFF24CFE7211A002952DD002881
:10B9700031D0FF2CB7D080203E00C0040643B4462F
:10B980001B2900DDAAE020266046C840711A6646E1
:10B990008E4031004E1EB14101435B185901D3D591
:10B9A0000134FF2C00D187E0012278491A405B085E
:10B9B0000B40134397E7002C00D0A7E0002B00D0EA
:10B9C000B6E03B1E62D10026002273025B0AE4B29D
:10B9D0009AE7140087E7002F4DD0481E002857D162
:10B9E000634401245A01AFD50224DDE7002A24D1A3
:10B9F000621CD2B2012ADEDDDE1B720135D5FE1AD1
:10BA00000D005CE72A0000237EE73300604A241A19
:10BA1000134068E7002963D1611CC8B201284EDDDC
:10BA2000FF2949D063445B080C005CE7FF2A41D042
:10BA30000A0079E701229B1A84E7002C1DD0FF2819
:10BA400022D08024E404524223431B2A00DD8AE0F2
:10BA50001C002025D440AA1A93405A1E9341234328
:10BA600062460400D31A0D0025E7002E00D026E719
:10BA700000220024A9E70C0035E7002B4DD0D2436B
:10BA8000002AEDD0FF28E0D16346FF240D002AE70D
:10BA9000FF290FD0010073E7002B61D0FF24002F96
:10BAA00000D120E780224146D203114202D0164243
:10BAB00000D13B00FF2416E7FF24002324E7002CDD
:10BAC000EAD1002B58D0002F00D10CE763445A0173
:10BAD00000D439E72E4A0C00134004E701215CE74B
:10BAE000002C1ED1002B40D0C94300290BD0FF28C9
:10BAF00036D01B2947DC1C002026CC40711A8B4015
:10BB0000591E8B4123436344040047E7002B18D19F
:10BB10003B1E2DD00D00FF24E5E63B0004000D0088
:10BB2000E1E6FF281CD08024E40449422343E0E7F7
:10BB3000002F00D1D7E6DE1B72011FD5FB1A0D00C6
:10BB4000D1E6FF24002F00D1CDE680224046D2036B
:10BB50001042AFD01642ADD13B000D00FF24C2E62B
:10BB60006346FF24BFE601237AE73B000400BAE600
:10BB700080260022F603F0E63B00B4E6331E00D038
:10BB8000E2E6002221E70123BDE7C046FFFFFF7D7B
:10BB9000FFFFFFFBF0B557464E46DE464546E0B593
:10BBA00044024300C60F83B00F1C640A1B0EB2464A
:10BBB00053D0FF2B27D08022E400D20414437F22ED
:10BBC000524290469844002399469B467D02780055
:10BBD000FB0F6D0A000E009324D0FF2846D080236F
:10BBE0000021ED00DB041D437F384746381A4F46DD
:10BBF0000F43BF00B9463300009A874F53404A466F
:10BC0000BA5801939746002C4ED108239946F73332
:10BC10009846FD3B9B467D027800FB0F6D0A000EA7
:10BC20000093DAD1002D26D1002001213300009AA3
:10BC30007A4F53404246101A4A460A439200BA5875
:10BC40001D009746009B2C009A468B465B46022BB4
:10BC500031D15346FF21002438E0002C17D10423B2
:10BC600099460023984601339B46AFE7FF20002DFD
:10BC70000BD10221DAE7280002F092FA431F9D401F
:10BC800076235B42181A0021AFE70321ADE72000BD
:10BC900002F086FA431F9C4076235B421B1A9846AB
:10BCA000002399469B4691E70C239946F333984627
:10BCB000FC3B9B468AE7032B00D1A5E05546012BB0
:10BCC00000D081E00123002100242B406402C9053B
:10BCD000600ADB070843184303B03CBC9046994612
:10BCE000A246AB46F0BD80240023E403FF21EDE72C
:10BCF000FF210024EAE70123591A1B2966DD019A76
:10BD0000134000210024E1E78023DB031C4238D0EC
:10BD10001D4251D01C436402640A3300FF21D5E761
:10BD200063016C01A3423BD21B260021013801258F
:10BD30001F0049005B00002F01DB9C4201D81B1B48
:10BD40002943013E002EF3D11C00631E9C410C438D
:10BD500001007F310029CEDD630704D00F2323408B
:10BD6000042B00D00434230103D501002C4B803177
:10BD70001C40FE290DDD0123019AFF211340002400
:10BD8000A4E78023DB031C436402640A3300FF2121
:10BD90009CE70123019AA401640AC9B2134095E704
:10BDA0001B1B1A260121C2E7009B8B469A460024E2
:10BDB0004CE76302E5D500258024E4032C436402AC
:10BDC000640A009BFF2181E70195C1E72300202041
:10BDD000CB40411A8C40611E8C411C43630704D048
:10BDE0000F232340042B00D00434630105D5012325
:10BDF000019A01211340002468E70123019AA4015C
:10BE0000640A1340002161E78023DB031C436402C2
:10BE1000640A5346FF2159E7CCFE00000CFF0000E6
:10BE2000FFFFFFF7F8B557464E464546DE46E0B5FC
:10BE30004702460088467F0A360EC40F002E47D0C0
:10BE4000FF2E24D0FB008027FF041F4300239946C8
:10BE50009A467F3E43465D025800DB0F6D0A000E96
:10BE6000984643D0FF283BD0EB0080250022ED040C
:10BE70001D437F383618731C41469B464B46614034
:10BE800013430F2B64D875489B00C3589F46002F5F
:10BE900042D108239946063BFF269A46DAE74146F7
:10BEA000022A28D0032A00D1CEE0012A00D0ACE03B
:10BEB000114000200022CCB24002D205400AE40723
:10BEC000104320433CBC90469946A246AB46F8BD81
:10BED000002F15D104239946033B00269A46B9E763
:10BEE000FF200222002DC5D00322C3E7002D19D167
:10BEF00000200122BEE70124FF220C400020DBE7E6
:10BF0000380002F04DF97626431F9F400023764209
:10BF1000361A99469A469DE70C239946093BFF2617
:10BF20009A4697E7280002F03BF9431F9D4076238D
:10BF30005B42181A00229DE780200024C003FF22E4
:10BF4000BAE73D005246ABE73D0021005246A7E765
:10BF50003B0C9C462A04120C2B0C140060466546D0
:10BF60003F043F0C7C4342435D437B43270C9B18BB
:10BF7000FF18BA4203D980235B029C46654424041F
:10BF80003A04240C121993015C1EA3413F0C920E3B
:10BF90007D191A43AD0115432B0104D501235E46DB
:10BFA0006A081D40154332007F32002A25DD6B07E9
:10BFB00004D00F232B40042B00D004352B0103D5D4
:10BFC0003200274B80321D40FE2A94DC0124A80158
:10BFD000400AD2B20C406FE78020C003074207D06E
:10BFE000054205D128434002400A4446FF2263E748
:10BFF00038434002400AFF225EE70124A31A1B2BAC
:10C0000005DD0C400022002056E75E46CBE72A0003
:10C010002020DA40C31A9D402B005D1EAB41134324
:10C020005A0704D00F221A40042A00D004335A01C0
:10C0300004D5012401220C4000203DE701249B018E
:10C04000580A0C40002237E780200124C00328430F
:10C050004002400A0C40FF222EE7C0464CFF000081
:10C06000FFFFFFF7F0B54F46D64646464400C0B541
:10C07000C20F47024802400A844666467B0A4800CF
:10C08000C90F9A46240E1500DB00000E8946F60003
:10C09000FF2800D18FE001214F464F4039009142E7
:10C0A00066D0221A002A00DC9DE000283DD1002E37
:10C0B00000D18BE0511E002900D0B5E001249B1B6C
:10C0C0005A0144D59B019F09380002F069F80538F0
:10C0D0008740844200DD96E0041B3A0020200134B2
:10C0E000E240041BA7403B005F1EBB4100241343FA
:10C0F0005A0704D00F221A40042A00D004335A01F0
:10C1000027D50134FF2C00D179E001229B015B0A85
:10C11000E4B22A405B02E405580AD20720431043E8
:10C120001CBC90469946A246F0BDFF2CE0D0802171
:10C13000C9040E431B2A7BDC31002020D140821A27
:10C140009640721E96410E439B1B5A01BAD45A0761
:10C15000D0D10122DF082A40FF2C33D1002F00D19B
:10C16000A8E08023DB033B435B025B0AFF24D1E7AB
:10C17000211A00294CDD00282AD0FF2CB8D08020BD
:10C18000C00406431B2900DDAFE030002027C84073
:10C19000791A8E40711E8E4106439B195901D6D5DE
:10C1A0000134FF2C00D185E001227A491A405B0856
:10C1B0000B4013439CE7002E00D070E76BE73B1E5B
:10C1C000C5D100227B025B0AE4B2A3E714008FE72B
:10C1D000002E4DD0481E002857D19B1901245A012A
:10C1E000B5D50224E0E7002A25D1621CD2B2012A8B
:10C1F00072DD9F1B7A0135D5F71A0D0064E7012225
:10C2000000232A4086E73B00634A241A13406FE765
:10C2100000296CD1611CC8B201284EDDFF2949D02C
:10C220009B195B080C0063E7FF2A41D00A0081E7F5
:10C2300001269B1B89E7002C1CD0FF2821D08024DD
:10C24000E404524223431B2A00DD96E01C00202513
:10C25000D440AA1A93405A1E93412343F31A040070
:10C260000D002DE7002F00D02EE700220024A9E7C3
:10C270000C003DE7002B58D0D243002AEED0FF2817
:10C28000E1D13300FF240D0032E7FF2910D0010077
:10C2900078E7002B6ED0FF24002E00D128E7802203
:10C2A0005146D203114203D06146114200D13300FE
:10C2B000FF241DE7FF2400232CE7002CE9D1002BED
:10C2C00063D0002E00D113E79B195A0100D43EE73A
:10C2D000314A0C0013400BE7002C1ED1002B2FD14C
:10C2E000002E4FD033000D0002E7012655E7002C49
:10C2F0001FD1002B43D0C94300290BD0FF2839D0D0
:10C300001B2944DC1C002027CC40791A8B40591E85
:10C310008B4123439B19040040E7002B1AD1002EC8
:10C3200024D180270022FF031BE7330004000D0007
:10C33000DEE6FF281ED08024E40449422343DFE7E1
:10C34000002E00D1D4E69F1B7A0100D437E7F31A00
:10C350000D00CDE6FF24002E00D1C9E68022504614
:10C36000D2031042A4D060461042A1D133000D0088
:10C37000FF24BDE63300FF24BAE601236EE7330055
:10C380000400B5E6002700221CE73300B0E60123D5
:10C39000C0E7C046FFFFFF7DFFFFFFFB41024300F8
:10C3A000C20F490A1B0E00207E2B0DDD9D2B0CDCDD
:10C3B000802000040143952B0ADC9620C31AD94043
:10C3C0004842002A00D108007047034BD018FBE711
:10C3D000963B9940F4E7C046FFFFFF7F70B5002809
:10C3E00030D0C317C4185C40C50F200001F0D8FE40
:10C3F0009E231B1A962B0DDC9622D21A94402A00FB
:10C400006402640ADBB26402DB05600AD2071843E7
:10C41000104370BD992B19DC9922D21A002A29DD0C
:10C4200094402200144C1440510704D00F210A40BC
:10C43000042A00D00434620113D4A401640ADBB2DC
:10C440002A00E0E7002200230024DCE70522210087
:10C45000121AD140B922D21A9440621E94410C4360
:10C46000DAE7054B2A001C409F23A4011B1A640A2B
:10C47000DBB2C8E72200D5E7FFFFFFFB10B5041EC3
:10C4800027D001F08DFE9E231B1A962B0ADC9622E4
:10C49000D21A94406402640ADBB26402DB05600ACB
:10C4A000184310BD992B17DC9922D21A002A27DDD8
:10C4B00094402200134C1440510704D00F210A402D
:10C4C000042A00D00434620112D4A401640ADBB24D
:10C4D000E3E700230024E0E7B9222100D21A9140CB
:10C4E0000A00511E8A410521091ACC401443DBE79A
:10C4F000044B1C409F23A4011B1A640ADBB2CCE747
:10C500002200D7E7FFFFFFFBF8B54546DE4657465A
:10C510004E460C03E0B54E00C90F88460D00610A77
:10C52000440F0C43C70019035800DB0F9B464B0A0E
:10C53000510F0B43760D400D1900D200D84500D1A4
:10C54000AEE0351A002D00DCF6E000280FD11343D1
:10C5500000D1DBE06B1E002B00D037E1BA1A974206
:10C56000BF41641A7F42E41B0126170024E0C64B3A
:10C570009E424DD080231B041943382D00DD07E176
:10C580001F2D00DD38E12020431B9A460B0050464A
:10C590008340994613004846EB4018430300504639
:10C5A0008240501E8241E9401A43BA1A611A9742EA
:10C5B000A441170064420C1B230262D56402650A81
:10C5C000002D00D1DFE0280001F0EAFD0300083B68
:10C5D0001F2B00DDD2E020223C00D21A9D40D44027
:10C5E0009F4025439E4200DDC4E09E1B731C1F2B11
:10C5F00000DDF1E0202238002900D21AD840914015
:10C6000097402C000143781E8741DC4000260F43F1
:10C610007B0709D00F233B40042B05D03B1DBB42B9
:10C62000BF417F42E4191F0023022CD5964B0136EF
:10C630009E4200D19AE04546944BFF081C4060079B
:10C64000760564020743240B760D00212403230B97
:10C650000C0D8F4A24051C431440330523435B0013
:10C66000ED075B082B43380019003CBC9046994607
:10C67000A246AB46F8BD6446044300D111E2040073
:10C6800067467B07C6D145466007FF080743E408B5
:10C690007D4B9E4230D024037605240B760DD4E7E3
:10C6A000331A9A46002B78DD002831D0764886422E
:10C6B000AED08020000401435346382B00DCE9E073
:10C6C0000A43511E8A410021D219BA42BF410919B9
:10C6D0007C4217000C192302D3D56B4B01369E42C6
:10C6E00000D13AE10120694B1C407B0807401F4301
:10C6F000E007074364088BE723003B4300D1CBE10D
:10C700008022120314432403240B9EE72E007FE7AC
:10C710000800104300D1B4E0581E002800D0DEE02D
:10C72000BA18BA429B4164185B42E418170001260C
:10C730002302A6D50226D5E7002D6ED1701C400538
:10C74000400D012800DCF9E0B81A84468742804198
:10C75000E51A40422D1A280200D489E0D71BBA42BC
:10C7600092411C1B5242A51AD84629E7454600248F
:10C7700000276AE7454CF61A2C4049E73D00283867
:10C78000854000272EE7380001F00AFD20301DE724
:10C790000A43511E8A41002107E7002B00D0F3E035
:10C7A000701C43055B0D012B00DCADE0364B98425D
:10C7B00000D1D1E0BA18BA42BF4164187F42E419EF
:10C7C000E707520817436408060021E72E48854210
:10C7D00000D193E01D00D0E629001F3EF140202B40
:10C7E00000D18DE04022D31A9D402F437D1EAF41E2
:10C7F00000240F43002644E72B000800203BD840CC
:10C800000300202D00D17DE04020451BA9400A43B4
:10C81000511E8A4100211A43C7E6002E50D01A4EFD
:10C82000B04257D080266B429946360434434B467B
:10C83000382B00DDD6E01F2B00DD35E12026F51A70
:10C840002600AE40B2463E00DE40AC4635005646BD
:10C850002E436546AF407D1EAF41DC403743D71BBA
:10C86000BA4292410C1B5242A41A0600D846A3E6D3
:10C87000644667462C4300D0A2E600250026002728
:10C8800006E71E00C4E6C046FF070000FFFF7FFF6B
:10C89000FFFF0F801F2B63DC2020C31A0800984085
:10C8A0009C46834653461000D84003005846184320
:10C8B00063469A40531E9A4153460243D94003E7C8
:10C8C00026003E4306D0EB439946002BC7D0944E3A
:10C8D000B042ACD10C0017000600D84698E6904B49
:10C8E0009A450BD08246E7E6002800D09EE018006B
:10C8F000104300D1E9E01C001700D846884E87E6B7
:10C90000002572E7002182E723003B43002E00D080
:10C91000ABE0002B00D1E7E00B00134300D177E63A
:10C92000BA18BA42BF4164187F42E419230200D406
:10C93000F2E07C4B17001C40060069E620003843FB
:10C94000002ED1D100285BD11C00144300D1A8E0F7
:10C950001C001700D8465BE606000024002797E677
:10C9600050460B002038C34099465346202B00D137
:10C9700095E0402350461B1A99400A43511E8A41B4
:10C980004B4600211A439FE6002E30D126003E433D
:10C9900067D0DB439A46002B1CD0614EB04260D07A
:10C9A0005346382B00DD96E01F2B00DD9FE020264C
:10C9B000F31A26009E409C46B34653463E00DE4096
:10C9C00033005E461E4363469F407B1E9F41534695
:10C9D000DC403743BF189742924164185242A41872
:10C9E000060078E627437C1EA741002437E74C4E1B
:10C9F000B04236D080265B4236049A463443CFE7B5
:10CA00001800104300D103E6B81A84466745AD41CB
:10CA1000E01A6D42401B050200D42CE6D71BBA4237
:10CA200092411C1B5242A41AD846F1E5180010434B
:10CA300000D163E7F808670707438020E408000394
:10CA4000044208D0DD08054205D1D2085907114338
:10CA50000F002C00D8467B0FE4001C43FF00304E33
:10CA6000D6E50C0017000600D2E5002B38D00B00ED
:10CA7000134300D142E7F808670707438020E40822
:10CA800000030442E7D0CB080342E4D1D2084907AF
:10CA900011430F001C00DEE700270024D5E500212C
:10CAA0006BE700250027F3E54E462500203EF540C4
:10CAB0004B462E00202B2DD04025ED1AAC402743AD
:10CAC0007C1EA74100243743C9E6802400252403A7
:10CAD000134E0027DCE527437C1EA741002479E79D
:10CAE0000C0017000E4E93E50C00170090E556461B
:10CAF0002300203EF34099465346202B0ED040237E
:10CB000056469B1B9C4027437C1EA7414B46002456
:10CB10001F435FE70024D2E71700B2E50024F2E7E5
:10CB2000FF070000FFFF7FFFF0B557464546DE4692
:10CB30004E46E0B54C000E0387B0834692461D007A
:10CB40008046360B640DCF0F002C4FD06F4B9C42AC
:10CB500035D08023420F1B04F6001343334399461C
:10CB6000C30098466A4B00269C4600236444039306
:10CB70002B031B0B9B466B00ED0F50465B0D019585
:10CB80005ED0624A934253D05A46D1008022400F71
:10CB9000120402430A4393465246D1005C4A94462B
:10CBA000002263443800684084460290E41A164329
:10CBB0000F2E00D9B4E0574BB6009B599F46030097
:10CBC000334399466CD100239846023308260393D9
:10CBD000CEE7CB464146039A0197022A65D1019BD5
:10CBE0004A4C9C460023002298466BE003003343E6
:10CBF00099464ED0002E00D1BCE1300001F0D0FAB1
:10CC000003000B3B1C2B00DDACE11D22D31A5A465E
:10CC10000100DA4008398E401300334399465B46E1
:10CC20008B40984600233C4C0026241A03939FE730
:10CC300051465A46114329D1002293460232B1E7A8
:10CC4000594601431ED05B46002B00D19EE1584659
:10CC500001F0A6FA03000B3B1C2B00DD8FE1020064
:10CC60005946083A91408B461D21CB1A5146D9406E
:10CC70000B0059460B4351469B469140264B0022E0
:10CC80001B1A8FE7002301229B468BE751460322A4
:10CC900088E700239846013304260024039367E7BE
:10CCA0000323B14603930C2662E7032A00D15CE21A
:10CCB000019B012A00D0E4E113409C46002300249C
:10CCC0000022984600211203130B0A0D12051A4385
:10CCD0002305124C40462240134362465B00D207B4
:10CCE0005B081343190007B03CBC90469946A24626
:10CCF000AB46F0BD002380229C4612039846034CAD
:10CD0000E0E70023014C00229846DBE7FF07000024
:10CD100001FCFFFF8CFF00000DFCFFFFFFFF0F80F9
:10CD2000D94500D939E100D134E1002346464D46CA
:10CD30009A46013C5B460A0E1B021A430B02170C73
:10CD4000039313041B0C3900280090460193FEF74F
:10CD500071FB0200019B83465A432800390091462B
:10CD6000FEF7EEFB350C09040D43A9450DD95B46D2
:10CD70004544013BA84500D93AE1A94500D837E12F
:10CD800002235B429C464544E3444B46EB1A390080
:10CD900018000493FEF74EFB019B05004343390046
:10CDA00004989946FEF7CCFB330409041B0C0B4393
:10CDB000994509D943446A1E984500D91AE1994515
:10CDC00000D817E1023D43444A469B1A5A461204D2
:10CDD0002A4303999346100C0A0C914609045A46BB
:10CDE000090C4E460D001204120C454305915143A7
:10CDF0007243704352190E0CB218954203D9802524
:10CE00006D02AC466044150C09041204090C281884
:10CE10005218834200D2CEE000D1C8E01D1A53461A
:10CE20009E1AB24592415242AB1A9A46984500D199
:10CE300017E139001800FEF7FDFA019B0500434396
:10CE4000390050460493FEF77BFB04980B04310C29
:10CE50001943884209D941446B1E884500D907E12E
:10CE6000884200D804E1023D4144049BCB1A1800DB
:10CE700039000493FEF7DEFA019B824643433900F2
:10CE800004980193FEF75CFB01980B043104090C34
:10CE9000194388420DD953464144013B884500D986
:10CEA000E8E0884200D8E5E002235B429C4641442A
:10CEB000E244019B2D04CE1A51462943059D4F465D
:10CEC0002A000B04080C1B0C5A4345437B43784350
:10CED0005B19170CFB189D4203D980256D02AC46E7
:10CEE00060441D0C12041B04120C28189B18864267
:10CEF00000D293E000D18EE001231943A04BE31848
:10CF0000002B00DC99E04A0700D09EE05A46D2018F
:10CF100006D55A469B4B1A4080239346DB00E31804
:10CF2000994A934268DD0123029A984C1A400023E3
:10CF3000944698460022C5E680224B4612031342CF
:10CF40000AD05B46134206D11A431203120BAC46B9
:10CF500088468E4CB6E64B461A431203120BBC466B
:10CF60008A4CAFE603005A46283B9A40002391467C
:10CF7000984657E6584601F013F9203040E6030082
:10CF80005246283B9A400021934677E601F008F983
:10CF900020305FE6884500D2C7E64B46DE075D08D5
:10CFA00043465B081E434346DB079A46C2E600251C
:10CFB000924500D333E7039E5946B446E244B24556
:10CFC000AD416D424544EB180139984507D298426E
:10CFD00000D97FE000D1BCE01D1A8B461FE79845C1
:10CFE000FAD1039D5545F2D943468B461D1A16E7E3
:10CFF0009B46CAE61500E7E65A46C90852070A43A7
:10D000005B0590465C0D5A46012302995202194075
:10D01000120B8C4656E6002B00D16FE746444A1EA1
:10D02000B04529D91100864200D065E7039A9342A2
:10D0300000D061E762E7012149420120C21A382A83
:10D0400021DD029B03409C4638E60F220A40042A59
:10D0500000D15BE70A00111D914292415242934474
:10D0600054E7474BE318002BE5DD01225242F2E77B
:10D070001D00FAE69A461CE7B04239D86ED011007E
:10D080003AE702933AE71F2A3CDC20239B1A0C0064
:10D090005846994098404B1E99415B46D440D34036
:10D0A000204308431A00430709D00F230340042BF1
:10D0B00005D00100081D88429B415B42D218130233
:10D0C0003AD50123029A01241A4000239446984637
:10D0D0000022F7E5022149428C46039DE344AC4619
:10D0E000E244AA45AD416D424544ED182D1A96E63D
:10D0F0008A1E03994D008D42894149424144761868
:10D1000003958FE71F204042C31A5846D8400300BA
:10D11000202A28D040205D46821A954029434A1E85
:10D1200091411943072300220B4009D00F2300220D
:10D130000B400800042BBDD1010053075202120B13
:10D14000C9081943012388460299002419408C46D6
:10D15000B8E55245BED88B46002560E6039D9D424A
:10D16000C6D3110062E70025D8E780225B46120390
:10D170001A43019B1203120B9C468846034CA1E5FF
:10D18000FF030000FFFFFFFEFE070000FF07000097
:10D19000F0B54F464646D6465C00C0B51F03DB0FD0
:10D1A0009A46174B0E034D0084468046360B6D0D94
:10D1B000C90F91463F0B640D01209D4208D09C424F
:10D1C00001D0A5420BD01CBC90469946A246F0BDAA
:10D1D00063463343F7D1AC42F5D13A43F3D1012052
:10D1E000BE42F0D1C845EED1514507D0002DEAD15D
:10D1F00063461E433000461EB041E4E70020E2E7EC
:10D20000FF070000F0B54546DE4657464E46E0B5FE
:10D210001F033D0B2C4F0E034C00AB465D008446B4
:10D22000360B640DC90F90466D0DDB0FBC422AD042
:10D23000254FBD422DD0002C0FD130430700814631
:10D2400078427841C0B2002D17D15F463A4314D1DD
:10D250004B460020002B0AD006E0002D02D1584694
:10D26000024301D0994218D04842012108433CBCF6
:10D2700090469946A246AB46F0BD0028F2D0012068
:10D28000013B1843F3E737000743D1D00220404267
:10D29000EDE75F461743CED0F8E7AC42E4DC03DAB3
:10D2A000481E01210843E2E75E45DDD806D0002094
:10D2B0005E45DCD20123481E1843D8E7C445D3D8C5
:10D2C0000020C445F6D3D2E7FF070000F0B54E4674
:10D2D0004546DE4657465C00E0B51F03DB0F994626
:10D2E0002A4B0E034D00C90F8446360B6D0D8B463D
:10D2F00090463F0B640D9D4220D0244B9C4222D08F
:10D30000002D12D1304343424341DBB2002C1FD0E9
:10D31000002B0CD04B460120013B034318003CBCC2
:10D3200090469946A246AB46F0BD002C16D0CB45A0
:10D3300017D05B46594201230B43EFE7310002232C
:10D340000143EBD1D9E7390002231143E6D1D7E7F6
:10D350003A43DDD100230028E0D0EAE73A43E6D1A2
:10D36000E7E7A542E5DC05DBBE42E2D807D00023B3
:10D37000BE42D3D25946012301390B43CEE7C445FF
:10D38000D7D80023C445F5D3C8E7C046FF0700003F
:10D39000F0B557464546DE464E46E0B50C03984686
:10D3A0004E00230B87B0070092469B46760DCD0FAB
:10D3B000002E6BD06D4B9E4235D080245B46420FD1
:10D3C0002404DB0014431C43C3009946684BA34666
:10D3D0009C46002300276644029343461C035A00E0
:10D3E000DB0F5046240B520D984600D176E05F4B80
:10D3F0009A426DD08023410F1B040B435C49E4002B
:10D400008C461C43C300002062444146B618694064
:10D41000721C0191944607430F2F00D9B0E0554A82
:10D42000BF00D25997465B460343994600D087E038
:10D4300000239B46023308270293CEE7424601921F
:10D44000022867D0032800D10EE2012800D062E153
:10D45000002300240022994601990140CDB2002109
:10D4600012030B0D120B1B051343434A24051340F3
:10D470001C436400ED0764082C434846210007B0B4
:10D480003CBC90469946A246AB46F0BD0343994644
:10D490004FD05B46002B00D189E1584600F080FE5A
:10D4A00003000B3B1C2B00DD7AE11D22D31A3A004E
:10D4B00001005C46DA4008398C4013008F4023435A
:10D4C0009B46B94600232D4E0027361A029384E767
:10D4D000534623432AD10024022096E75346234390
:10D4E00020D0002C00D157E1200000F059FE0300AD
:10D4F0000B3B1C2B00DD49E11D21CB1A51460200DC
:10D50000D9405346083A944093400C431B4A121AA0
:10D5100000207AE70125019B144C1D4000230022C6
:10D5200099469CE70024002201206EE75346032021
:10D530006BE700239B4601330427002602934CE748
:10D54000032381460C27029347E78022002300250E
:10D5500012039946054C82E75C464B4602986FE7FA
:10D560005C464B46019502986AE7C046FF070000FB
:10D5700001FCFFFFCCFF0000FFFF0F800DFCFFFF51
:10D580004A464946170C1A0C1B041B0C08041900C8
:10D59000000C41431500884619007D4379430395EB
:10D5A00089462900150045434D44029545462D0CFA
:10D5B000AA46029D5544A94506D98A4680214902BA
:10D5C0008946CA4451460391290C049141460904F5
:10D5D0002D04090C88462900250C24044144240C00
:10D5E0000591210041438846210079438A466843DA
:10D5F000414650448146080C48446F43824503D954
:10D600008021490289464F44010C8946390049442A
:10D61000029141460F0404993F0C88460004C0194A
:10D6200080444146049159460F0C0904090C884670
:10D6300059438A4639005143894641464A43514637
:10D64000090C8B467B43D2185A44934203D980235A
:10D650005B029B46D94451460904090C8A4641465F
:10D6600061437C43130C12044B445244A1468A4646
:10D670003C0041466C434D4351464D440F0C7D19CF
:10D68000A94503D98021490288464444049F03994F
:10D69000B84641448B4683458041414288465146C5
:10D6A00008042F04000C3F185846029910188946A8
:10D6B000904292414F44BA46524299469346C244E0
:10D6C000D144CB448F42BF41C245894199459B41DA
:10D6D000934592417F4249422D0C52420F435B4297
:10D6E00013437F19FF185B463C19DB0D059A640252
:10D6F0001C43430213435D1EAB415A46C00D034316
:10D7000052021343E20156D501205A080340134345
:10D71000E207134364085A48604400284DDD5A0765
:10D7200009D00F221A40042A05D01A1D9A429B41A3
:10D730005B42E4181300E20104D58020514AC00086
:10D7400014406044504A904200DDE3E60125DB08C6
:10D7500062071A436402019B9146220B4405640D43
:10D760001D407CE6802259461203114208D0144223
:10D7700006D122431203120B45469946434C6EE6EE
:10D780005B461A431203120B404C68E603005446F2
:10D79000283B9C400023B9E600F002FD2030A6E6BD
:10D7A0000300283B9F400023BB4699468AE600F0D1
:10D7B000F7FC203074E6B446ADE701252A1A382A72
:10D7C00006DD019B00241D4000230022994646E609
:10D7D0001F2A21DC20252000AD1A1E00AB40A840E6
:10D7E000D6405D1EAB4130431843D440430709D0B7
:10D7F0000F230340042B05D00300181D98429B41C2
:10D800005B42E418230221D50125019B01241D4020
:10D8100000230022994622E61F2521006D42281A86
:10D82000C1400800202A1DD05F35AA1A9440234326
:10D830005C1EA341072503431D400022002D09D093
:10D840000F2200241A401800042AD6D103006507CD
:10D850006402220BDB082B4301259946019B00241F
:10D860001D40FCE50024E2E780220125120322434B
:10D8700001991203120B0D409946044CEFE5C04686
:10D88000FF030000FFFFFFFEFE070000FF07000090
:10D89000F0B54646D6464F460C03C0B5CD0F4E00F8
:10D8A000610A440F0C43C1005800400D84468A466B
:10D8B0000F001903500F490A0143C648760DA846C8
:10D8C000DB0FD200844500D1D8E001204340AB42B9
:10D8D00000D1A6E06046351A002D00DC05E10028E5
:10D8E00010D10B00134300D1D7E06B1E002B00D0EA
:10D8F0004BE153469F1ABA458041641A4042241AAC
:10D9000001261EE0B34B9E4248D080231B041943DE
:10D91000382D00DD19E11F2D00DD4CE120230F0023
:10D920005B1B10009A409F40E840531E9A41E9401B
:10D93000074317435346DF1B611ABA45A4416442AB
:10D940000C1B230200D4C5E06402650A002D00D13F
:10D95000F6E0280000F024FC0300083B1F2B00DD4C
:10D96000E9E020223C00D21A9D40D4409F4025434C
:10D970009E4200DDDBE09E1B731C1F2B00DD0AE1D5
:10D9800020223800D21A290097402C009140D8401C
:10D990007A1E9741DC40002601430F437B0709D0E4
:10D9A0000F233B40042B05D03B1DBB42BF417F42B0
:10D9B000E4191F00230225D5864B01369E4200D173
:10D9C000AFE0854B01251C4043466207FF08640217
:10D9D00076051743240B760D1D4000212403230BED
:10D9E0000C0D7E4A24051C431440330523435B0081
:10D9F000ED075B082B43380019001CBC9046994684
:10DA0000A246F0BD012543466207FF081743E4081C
:10DA10001D40704B9E4236D024037605240B760DB4
:10DA2000DBE76346F31A002B00DC94E06046002835
:10DA300035D068488642B1D080273F043943382B1F
:10DA400000DCFDE00A43170000217A1E974157448D
:10DA500057458041091944420C1923023AD55D4BC0
:10DA600001369E4200D14BE101225B4B1C407B08FA
:10DA700017401F43E207174364088FE7080010436D
:10DA800000D024E721E723003B4300D1B9E1802205
:10DA9000120314432403240B9FE72E007EE70800A3
:10DAA000104300D1CAE0581E8446002800D0E7E0A9
:10DAB0005244524580416418404224181700012600
:10DAC000230207D50226CFE764462C4300D1B3E1F9
:10DAD0002C0067467B0700D062E76307FF081F43FF
:10DAE00001254346E4081D4093E7002D78D1751CBD
:10DAF0006D056D0D012D00DCF2E05046801A824567
:10DB0000BF41651A7F42ED1B8446280200D48CE099
:10DB10005046171ABA4292410C1B5542651B984653
:10DB200014E70125434600241D40002755E72A4CF1
:10DB3000F61A2C4032E73D0028388540002717E7C9
:10DB4000380000F02DFB203006E70A4317000021C3
:10DB50007A1E9741EEE6002B00D0E5E0731C9C4650
:10DB60005B055B0D012B00DC9FE01A4B9C4500D14F
:10DB7000C5E0524452458041641840422418E707EA
:10DB8000520817436408664608E71248854200D1E8
:10DB900085E01D00BCE629001F3EF140202B00D18E
:10DBA0007FE04022D31A9D402F437D1EAF410024C9
:10DBB0000F4300268EE72B000F00203BDF40202D77
:10DBC00071D040235D1BA9400A43511E8A410021A8
:10DBD0001743AFE6FF070000FFFF7FFFFFFF0F8047
:10DBE000002E3ED0B34EB44545D0802636046D425B
:10DBF0003443382D00DDA8E01F2D00DD1FE1202675
:10DC000027005046761BB740E84007435046B040D7
:10DC1000461EB041EC403843171ABA4292410C1BE1
:10DC20005242A41A664698468BE6644667462C43E1
:10DC300000D08BE6002500260027EAE61E00ADE6B0
:10DC40001F2B60DC2027F81A0F0084468740100045
:10DC5000D840074360468240501E8241D940174356
:10DC6000F5E626005046064305D0ED43002DD3D0FF
:10DC7000904EB445BDD10C001700664698468DE61F
:10DC80008C4883420BD06346D9E6002D00D096E045
:10DC90000800104300D1E2E00C0017009846854EC2
:10DCA0007CE6002580E700218EE7230050460343F1
:10DCB000002E00D0A8E0002B00D1DEE00B001343C3
:10DCC00000D16BE65244524580416418404224180A
:10DCD0001700230200D4FDE6774B66461C405DE644
:10DCE000250050460543002ECFD1002D4FD10C000A
:10DCF000144300D1A0E00C00170098464EE666469B
:10DD00000024002785E61F000800203FF840070098
:10DD1000202B00D18EE04020C31A99400A43511EA7
:10DD20008A410021174392E6002E14D12600504666
:10DD3000064362D0DB43002B5CD1871897429241A7
:10DD400064185242A418664687E650462043441E93
:10DD5000A041002460E7574EB4454ED080263604DB
:10DD60005B423443382B00DD7FE01F2B00DD8BE06E
:10DD7000202627005046F61AB740D84007435046A1
:10DD8000B040461EB0410743DC40BF18D6E70D0047
:10DD9000154300D102E65046801A8245BF41651AFC
:10DDA0007F42ED1B8446280200D48DE65046171AA8
:10DDB000BA4292410C1B5242A41A9846EEE50D005D
:10DDC000154300D16BE750466707C0080743802022
:10DDD000E4080003044207D0CD08054204D12C001A
:10DDE0009846D70849070F437B0FE4001C43FF0008
:10DDF000304ED3E52F4EB445B4D10C001700664623
:10DE0000CCE500270024E8E5002B39D00B001343B4
:10DE100000D144E7C008670707438020E4080003F7
:10DE20000442E1D0CB080342DED1D70849070F43B3
:10DE30001C00D9E7002171E700250027E9E52E0045
:10DE40002700203EF740202D2FD04026751BAC40E8
:10DE500050462043441EA04100243843DCE6802481
:10DE600000252403134E0027D3E550462043070026
:10DE7000781E87410024BF1860E70C0017008DE56D
:10DE80000C0017000B4E89E51E002700203EF740CE
:10DE9000202B0CD04026F31A9C4050462043441EB1
:10DEA000A04107430024BF1848E70024D0E700241E
:10DEB000F3E7C046FF070000FFFF7FFF70B50E4E7F
:10DEC0000D031C0349005B002D0B490D240B5B0D5A
:10DED000B14204D0084900208B4208D070BD0543F0
:10DEE0000120002DFAD1044900208B42F6D11443C1
:10DEF0002000441EA041F1E7FF07000030B5134D9C
:10DF00000A034B00120B5B0DC90F0024AB4210DD5E
:10DF10000F4CA3420FDC80240E4D64032243ED1A04
:10DF20001F2D0BDD0C48C31ADA405442002900D1E2
:10DF30001400200030BD094BCC18FAE7084CE8402B
:10DF4000A44663449A400243EFE7C046FE03000044
:10DF50001D0400003304000013040000FFFFFF7FD6
:10DF6000EDFBFFFF70B5002830D0C317C4185C402C
:10DF7000C50F200000F014F9174B184A1B1AD21ACB
:10DF80001F2A18DD164AD21A9440002224035B058A
:10DF9000240B5B0D0021100024030A0D240B120535
:10DFA0002243104C1B05224013435B00ED075B0826
:10DFB0002B43190070BD210091400A000B21081A63
:10DFC000C4405B052403240B5B0DE3E7002500231D
:10DFD00000240022DEE7C0461E04000033040000D7
:10DFE00013040000FFFF0F804100090E4B1C70B5A9
:10DFF000DBB24602750AC40F012B14DDE0239B003F
:10E000006D07360BCB1800210A0D280012051C4D98
:10E0100032435B052A405B0813435B00E4075B085F
:10E020002343190070BD002914D1002D1ED02800F3
:10E0300000F0B6F80A281CDC0B232A001B1ADA4071
:10E04000030015339D400F4B12031B1A5B05160B83
:10E050005B0DD8E7002D06D0320B802636036D0706
:10E060001643094BCFE7084B0026CCE700230026D8
:10E07000C9E703002A000B3B9A400025E3E7C046AE
:10E08000FFFF0F8089030000FF070000F0B54C0080
:10E09000640D0B03621C450F5B0A52052B43C90F2D
:10E0A000C500520D012A28DD3A4AA618FE2E1BDCB7
:10E0B000002E3EDD80010200501E82416D0F2A437A
:10E0C000DB0013435A0704D00F221A40042A00D061
:10E0D00004338022D2041A405AD00136FF2E03D0D6
:10E0E0009B015B0AF4B201E0FF2400235802E4051F
:10E0F000400AC90720430843F0BD002C07D01D4348
:10E10000F2D08020DB0080040343FF26DAE72B43B4
:10E1100003D00523DB08FF2C03D05B025B0AE4B2CB
:10E12000E4E7002B32D08020C00303435B025B0A8C
:10E13000DCE73200173214DB80221E27120413435F
:10E14000BF1B1F2F0FDC144A944664442A00A540CD
:10E150002E00A340751EAE41FA4033431343002600
:10E16000B0E70024D5E702225242961B1A00F24083
:10E17000202F09D0094884466444A3402B435D1EE8
:10E18000AB41002613439DE70023F7E70023ADE7EB
:10E190003400BFE780FCFFFF82FCFFFFA2FCFFFF13
:10E1A0001C2101231B04984201D3000C10391B0AC7
:10E1B000984201D3000A08391B09984201D300098B
:10E1C000043902A2105C40187047C04604030202E2
:10E1D000010101010000000000000000F0B54E4602
:10E1E0005746DE464546E0B5060000200F0083B0E6
:10E1F00019008146002F00DA8CE0002900DA80E067
:10E2000034003D0092469846BB4269D866D04146EC
:10E21000504600F0BFF883463900300000F0BAF8ED
:10E220005B461B1A9C46203B9B4600D587E0514627
:10E23000584681400B005146604681400A00BB426F
:10E2400000D972E06ED034003D005946A41A9D41B9
:10E25000002900DA8AE000210020012600900191C7
:10E2600059468E400196614601268E4061460096D1
:10E27000002961D0D90756080E435F086146012284
:10E2800000230CE0AF4201D1A6420AD8A41BBD4135
:10E2900024196D410139A4185D41002906D0AF420F
:10E2A000F0D9013924196D410029F8D15B46009855
:10E2B000019900196941002B4DDB2E00DE406346B9
:10E2C0002C00DC405B46002B5BDB34009C402300D1
:10E2D0006446A6403200801A994103E0B24296D9C2
:10E2E000002000214B46002B04D003000C0000212D
:10E2F0005842A14103B03CBC90469946A246AB4669
:10E30000F0BD4946C9431000894619000023424226
:10E310008B4175E734003D00013800276642AF416C
:10E3200081466AE7B14200D88DE7002100200090C5
:10E330000191614600299DD100980199D2E762467A
:10E3400040462023514690409B1AD940030000913B
:10E3500000990B436FE7624620239B1A2A009A40DC
:10E36000260013006246D6401E43A8E761462026D9
:10E370000127761A00200021F740009001910197B3
:10E3800071E762462023350094409B1ADD4023004C
:10E390002B439DE710B5002903D1FFF701FF203083
:10E3A00002E0081CFFF7FCFE10BDC046F4F762F85F
:10E3B000002103E00A4B5B584350043109480A4BE3
:10E3C00042189A42F6D3094A02E00023136004324D
:10E3D000074B9A42F9D300F00DF8804770470000D0
:10E3E0004400010000F0FF1F8CF0FF1F90F0FF1FA2
:10E3F000A0000020F8B5F4F787FCF4F70DF9F4F766
:10E4000027F9F4F78DF9F4F773FAF4F7BDFCF6F792
:10E410002DFEF6F75FFEF4F713FEF5F719F8F4F7A3
:10E420007BF9F4F717FCF4F737FC00283FD1254CB3
:10E43000FA252078F5F748F8E078F5F727F922690A
:10E44000A1686079F4F7B6FCAD00FBF7D5F80027BA
:10E45000F6F79EFE0126F9F73BFCFAF7FBFFF4F70F
:10E4600083F9194C0BE0F4F7D7FA2671F4F796FC10
:10E470002060F4F793FCFCF7C5FCF4F7E9FBFCF72C
:10E48000E7FCF9F745F8FAF77FFCFAF7E5FFF4F750
:10E4900085FC2368C01AC317C0185840A842E8DD9D
:10E4A0002379002BDFD0F4F7B5FA2771DEE7F4F714
:10E4B000F3FBFF25034C6070A570F4F7EDFBE560FE
:10E4C000A060B5E74CF9FF1F64F1FF1F030082183D
:10E4D000934200D1704719700133F9E7F0B5C64691
:10E4E00000B58CB004000D0000F080F83A4B060037
:10E4F0001B780F005BB2984601330FD022002B002F
:10E5000020002900FFF7DAFC002807D100220023B1
:10E5100020002900FDF72EF9002805D03000390031
:10E520000CB004BC9046F0BD2C4B0A9003934346BC
:10E530000494059506940795002B1AD1E022284BE8
:10E540001206089209932000002200232900FDF7FB
:10E55000F7F8002838D00223029302A800F048FA06
:10E56000002817D00A9B0193002B18D1089E099F01
:10E57000D4E700221B4B20000892099329000022B7
:10E580000023FDF7DDF800280FD002230293434655
:10E59000022BE2D100F034FA22230360E2E700F01C
:10E5A0002FFA0A9B01930360E0E70123029343469D
:10E5B000022B0BD100F024FA212303600A4800F05B
:10E5C00019FA08900991CDE70123029302A800F0FF
:10E5D0000FFA0028F2D1EDE784F0FF1F18000100C8
:10E5E000FFFFEFC70000F0FF14000100F0B5D646B2
:10E5F0004F464646C0B5DA4A88B00B00914255DC1A
:10E600004A005208024300D1EFE0002900DA79E124
:10E61000D44B0022FEF7BCFE3625D34C0B006D42D6
:10E62000A34247DC1A15D14C1B031B0B9846A4468A
:10E630008024CF4B640343442340CE4C62445219A0
:10E640005C4045461B1599462543CA4B2900914419
:10E650000022FFF71DF9434602331B0306000F009B
:10E660001B0B0022022B2FDC0023FDF769F800288A
:10E6700000D1C1E04B46002B00D14CE14846FFF7EA
:10E6800071FCBD4ABD4B04000D00FEF781FEBC4A83
:10E6900006000F00BB4B20002900FEF779FE0200A8
:10E6A0000B0030003900FDF72FFF07E0AE4C0025CE
:10E6B000A342B7DD02000B00FDF726FF08B01CBC2B
:10E6C00090469946A246F0BD8023DB05FDF71CFF6E
:10E6D00002000B0030003900FEF726FA040048461D
:10E6E0000D00FFF73FFC2200029003912B00200059
:10E6F000290004940595FEF74BFE04000D00A24B83
:10E70000020043449A460B0000940195FEF740FE38
:10E7100004000D009D4A9E4BFEF73AFE9D4A9E4B1B
:10E72000FDF7F2FE22002B00FEF732FE9B4A9C4BC7
:10E73000FDF7EAFE22002B00FEF72AFE994A9A4BCB
:10E74000FDF7E2FE009A019BFEF722FE974A009039
:10E750000191974B20002900FEF71AFE954A964B2F
:10E76000FDF7D2FE22002B00FEF712FE934A944BD7
:10E77000FDF7CAFE22002B00FEF70AFE0B00020086
:10E7800000980199FDF7C0FE0D0041468D4B040035
:10E790005B1A51460B43002B54DD00228A4B30009C
:10E7A0003900FEF7F5FD32003B00FEF7F1FD4B4668
:10E7B0000A00010000910192002B72D11300290080
:10E7C00002002000FDF7A0FE049A059BFEF7E0FD85
:10E7D00002000B0000980199FFF75AF802000B00A5
:10E7E00030003900FFF754F868E7002200230020CA
:10E7F0007649FEF799F961E7754A764B30003900A2
:10E80000FEF7C6FD02000B0000206F49FFF740F83D
:10E81000320004000D003B0030003900FEF7B8FD67
:10E820000B00020029002000FEF7B2FD4B46040059
:10E830000D00002B72D102000B0030003900FFF7F1
:10E8400027F83BE74B46002B00D1C5E0029803991F
:10E85000494A4A4BFEF79CFD2200009001912B0093
:10E8600030003900FFF714F8049A059BFEF790FD7D
:10E87000434A04000D0002980399424BFEF788FDBD
:10E8800002000B0020002900FFF702F832003B00D5
:10E89000FEF7FEFF02000B0000980199FEF7F8FF5B
:10E8A0000CE7354A354B02980399FEF771FD009A43
:10E8B000019B0690079120002900FDF725FE049A90
:10E8C000059BFEF765FD2E4A04000D000298039992
:10E8D0002C4BFEF75DFD02000B0020002900FDF728
:10E8E00013FE02000B0000980199FEF7D1FF3200E1
:10E8F0003B00FEF7CDFF02000B0006980799FEF7DC
:10E90000C7FFDBE602000B00FEF7C2FF0022002378
:10E91000FEF70AF9D2E600200021CFE64846FFF7CD
:10E9200021FB154A154B00900191FEF731FD144A69
:10E930000290039100980199124BFEF729FD020005
:10E940000B0020002900FEF7A3FF32003B00FEF77A
:10E950009FFF02000B0002980399FEF799FFADE6B6
:10E96000FFFF0F0000005043FFFFEF7F01FCFFFFA0
:10E97000645F09000000F03F0000E0FE422EE63F29
:10E98000763C7935EF39EA3D86EBF9FF44523EDFBC
:10E9900012F1C23FDE03CB966446C73F59932294DF
:10E9A0002449D23F935555555555E53F9FC678D0DC
:10E9B000099AC33FAF788E1DC571CC3F04FA979971
:10E9C0009999D93F51B806000000E03F000050C3BC
:10E9D000555555555555D53F22002B00300039006F
:10E9E000FEF756FF049A059BFEF7D2FCF6E6C046FA
:10E9F00000207047002001497047C0460000F87FA2
:10EA0000014B18687047C04620F0FF1FE62A00003F
:10EA1000F42A0000022B00000A2B0000142B000037
:10EA2000142B0000142B0000142B0000142B0000EA
:10EA3000142B0000DC2A0000DC2B0000E42B00007B
:10EA4000EC2B0000F42B00002E2C0000FC2B00000F
:10EA5000182C00002E2C0000C82B0000EA2D00000E
:10EA6000EA2D00004E2E00005A2E0000662E0000F7
:10EA7000722E0000EA2D0000422E00007E2E0000C3
:10EA80008025000040380000004B0000807000002E
:10EA90000096000000E10000002C010000C201000F
:10EAA000D2380000E0380000EC380000F8380000F0
:10EAB0000839000016390000223900002E39000004
:10EAC000B2380000CA38000090390000A0390000B8
:10EAD000AE390000BC390000CE390000DE3900003C
:10EAE000EC390000FA390000083A00006A390000E9
:10EAF000823900005E3A0000683A0000723A000075
:10EB00007C3A0000543A00004A3A00004A3C0000B7
:10EB1000363C0000403C0000543C00005E3C0000DD
:10EB2000683C0000743C00007E3C0000883C000013
:10EB3000923C00009C3C00002C3C00001C3C00006F
:10EB4000E8410000D6410000C4410000B04100008F
:10EB50009C4100008A4100007841000066410000AD
:10EB60005641000048410000364100000E410000BF
:10EB7000864200009A420000AC420000BE42000003
:10EB8000D2420000E6420000F84200000A430000C2
:10EB90001C4300002C430000504200006242000071
:10EBA000DE430000F64300000C4400002244000055
:10EBB0003C440000544400006A44000080440000CB
:10EBC00096440000AA44000094430000B6430000AD
:10EBD000564500006A4500007C4500008E45000057
:10EBE000A2450000B6450000C8450000DA45000017
:10EBF000EC450000FC4500002045000032450000C7
:10EC00009A460000AE460000C0460000D246000012
:10EC1000E6460000FA4600000C4700001E470000D0
:10EC20003047000040470000644600007646000080
:10EC3000C8470000DA470000EA470000FA47000032
:10EC40000C4800001E4800002E4800003E4800000E
:10EC50004E4800005C48000068480000A6470000DD
:10EC6000AC4A0000A24A0000984A00008E4A000008
:10EC7000844A0000784A00006E4A0000644A00009E
:10EC80005A4A0000504A0000464A00002A4A000042
:10EC9000B64A00009E4C0000E84B0000F84B000014
:10ECA000024C0000364C0000B44B0000664C0000E3
:10ECB000584C0000864C0000784C00004A4C000084
:10ECC0003C4C0000944C0000F64D0000DC4D000070
:10ECD000C84D0000824D00007A4D00004E4D0000EE
:10ECE000A84F00004A4F00005C4F0000684F000032
:10ECF000A04F0000104F00004254000038540000A4
:10ED00002C5400002454000014540000045400004B
:10ED1000F8530000EE530000E4530000CE5300000F
:10ED2000C2530000AE530000945300004A54000048
:10ED30004A5400004A5400004A5400004A5400005B
:10ED40004A5400004A5400004A5400004A5400004B
:10ED50004A5400004A5400004A5400004A5400003B
:10ED60004A5400004A5400004A5400004A5400002B
:10ED70004A5400004A5400004A5400004A5400001B
:10ED80004A5400004A5400004A5400004A5400000B
:10ED90004A5400004A5400004A5400004A540000FB
:10EDA0004A5400004A5400004A5400004A540000EB
:10EDB0004A5400004A5400004A5400004A540000DB
:10EDC000885300007C5300004A5300004653000063
:10EDD000425300003E5300000C530000F25200006A
:10EDE000EE5400000C5500002A5500003E5500006E
:10EDF000EE5500004655000070550000A66000006A
:10EE0000A6600000A66000009A550000C4550000EE
:10EE10001056000046570000EE5600001A5700003A
:10EE2000A0560000F45700009E570000A6600000A6
:10EE3000205800003C560000A6600000A6600000BC
:10EE4000A6600000725700005A560000A66000003D
:10EE5000A6600000A660000086560000B2560000C2
:10EE6000C2560000DC560000A6600000A66000004C
:10EE7000A6600000A6600000A6600000A66000007A
:10EE8000065800002E58000040580000525800005C
:10EE90007E580000AA580000AE5B0000A66000008B
:10EEA000A6600000A6600000D6580000F0580000E0
:10EEB000BA5A00004E5F0000B45E00007A5F0000A6
:10EEC000D05D0000A6600000A6600000A660000003
:10EED000A6600000A6600000A6600000A66000001A
:10EEE000A6600000A6600000A6600000A66000000A
:10EEF000A6600000A6600000FC5D0000285E000027
:10EF0000545E000096590000D05C0000C259000019
:10EF1000E05900006A5C0000945C0000A85C0000FE
:10EF2000BC5C0000FE5A0000A6600000A660000065
:10EF3000A6600000A6600000A6600000A6600000B9
:10EF4000A6600000A6600000865D0000125B000065
:10EF50003C5B0000FC5C0000B45D0000A6600000AB
:10EF6000A6600000A6600000A6600000A660000089
:10EF70002A5D0000585D0000025900002E59000073
:10EF8000405900006C590000085C0000046000005B
:10EF9000325C0000505C0000D45A00006260000047
:10EFA000A6600000A6600000A6600000A660000049
:10EFB000A6600000A6600000A6600000A660000039
:10EFC000A6600000A6600000A6600000A660000029
:10EFD000A6600000A6600000A6600000A660000019
:10EFE000A6600000A6600000A6600000A660000009
:10EFF000A6600000A6600000A6600000A6600000F9
:10F00000A6600000A6600000A6600000A6600000E8
:10F01000A6600000A6600000A6600000A6600000D8
:10F02000A6600000A6600000A6600000A6600000C8
:10F03000A6600000A6600000A6600000A6600000B8
:10F04000A6600000A6600000A6600000A6600000A8
:10F0500022600000A6600000A6600000A66000001C
:10F06000A6600000A6600000A6600000A660000088
:10F07000A6600000A6600000A6600000A660000078
:10F08000A6600000A6600000A6600000A660000068
:10F09000A6600000A6600000A6600000A660000058
:10F0A000A6600000A6600000A6600000A660000048
:10F0B000A6600000A6600000A6600000A660000038
:10F0C000A6600000A6600000A6600000A660000028
:10F0D000A6600000A6600000A6600000A660000018
:10F0E000A6600000A6600000A6600000A660000008
:10F0F000A6600000A6600000A6600000A6600000F8
:10F10000A6600000A6600000A6600000A6600000E7
:10F11000A6600000A6600000A6600000A6600000D7
:10F12000A66000007A600000E05E00003860000029
:10F13000985400000C5F0000F4590000A660000025
:10F14000A6600000A6600000A6600000A6600000A7
:10F15000125A0000225A0000A6600000A6600000BB
:10F16000A6600000A6600000A6600000A660000087
:10F17000A6600000A6600000345A0000445A000057
:10F18000625A0000A6600000A6600000A6600000B1
:10F19000A6600000A6600000A6600000A660000057
:10F1A000725A00008A5A0000A25A00009A5E0000BB
:10F1B000805E0000AA5F0000665B0000905F0000B8
:10F1C0007E5B0000965B0000A6600000A660000069
:10F1D000A6600000A6600000A6600000DA540000EF
:10F1E000C66B0000FA6B0000766C0000026E000037
:10F1F0003E6C0000A66C0000DA6B0000806D000021
:10F20000026E0000C46C0000026E0000B86D0000C9
:10F210005C6C0000506D0000026E0000026E000089
:10F22000026E00000A6D0000326D0000126C0000DA
:10F23000026E00009C6D0000026E0000026E000075
:10F24000026E0000026E0000026E0000026E0000FE
:10F25000026E0000026E0000026E0000026E0000EE
:10F26000026E0000026E0000026E0000026E0000DE
:10F27000026E0000026E0000026E0000026E0000CE
:10F28000026E0000026E0000026E0000026E0000BE
:10F29000026E0000026E0000026E0000026E0000AE
:10F2A000026E0000026E0000026E0000026E00009E
:10F2B000026E0000026E0000026E0000026E00008E
:10F2C000026E0000026E0000026E0000026E00007E
:10F2D000026E0000026E0000026E0000026E00006E
:10F2E000E46C0000F46C0000966C0000D86D000027
:10F2F0006A6D0000026E0000026E0000026E0000E7
:10F30000026E0000026E0000026E0000026E00003D
:10F31000026E0000026E0000026E0000026E00002D
:10F32000026E0000026E0000026E0000026E00001D
:10F33000026E0000026E0000026E0000026E00000D
:10F34000026E0000026E0000026E0000026E0000FD
:10F35000026E0000026E0000026E0000026E0000ED
:10F36000026E0000026E0000026E0000026E0000DD
:10F37000026E0000026E0000026E0000026E0000CD
:10F38000026E0000026E0000026E0000026E0000BD
:10F39000026E0000026E0000026E0000026E0000AD
:10F3A000026E0000026E0000026E0000026E00009D
:10F3B000026E0000026E0000026E0000026E00008D
:10F3C000026E0000026E0000026E0000026E00007D
:10F3D000026E0000026E0000026E0000026E00006D
:10F3E000026E0000026E0000026E0000026E00005D
:10F3F000026E0000026E0000026E0000026E00004D
:10F40000026E0000026E0000026E0000026E00003C
:10F41000026E0000026E0000026E0000026E00002C
:10F42000026E0000026E0000026E0000026E00001C
:10F43000026E0000026E0000026E0000026E00000C
:10F44000026E0000026E0000026E0000026E0000FC
:10F45000026E0000026E0000026E0000026E0000EC
:10F46000026E0000026E0000026E0000026E0000DC
:10F47000026E0000026E0000026E0000026E0000CC
:10F48000026E0000026E0000026E0000026E0000BC
:10F49000026E0000026E0000026E0000026E0000AC
:10F4A000B86B0000026E0000026E0000026E0000E9
:10F4B000026E0000026E0000026E0000026E00008C
:10F4C000026E0000026E0000026E0000026E00007C
:10F4D000026E0000026E0000B86B0000EE6D0000CE
:10F4E000E46E0000A06E0000786F0000026E000065
:10F4F000026E0000026E0000026E0000026E00004C
:10F50000026E0000026E0000026E0000026E00003B
:10F51000026E0000026E0000026E0000026E00002B
:10F52000026E0000026E0000026E0000026E00001B
:10F53000026E0000026E0000026E0000026E00000B
:10F54000026E0000026E0000026E0000286F0000D4
:10F55000506F0000006F0000646F0000026E00003A
:10F56000026E0000026E0000026E0000026E0000DB
:10F57000026E0000026E0000026E0000146F0000B8
:10F580003C6F0000D06E00008C6E0000786E0000B2
:10F59000646E0000506E0000BC6E0000E474000059
:10F5A000DA740000D0740000C6740000BE7400005D
:10F5B000A6740000A6740000A6740000A6740000E3
:10F5C000A0740000A0740000A0740000A0740000EB
:10F5D000E47400009A74000094740000E474000065
:10F5E000E4740000E47400008E740000887400006D
:10F5F000827400007C740000767400007074000057
:10F600006A740000647400005E74000058740000A6
:10F61000E4740000527400004C7400004674000052
:10F62000407400003A740000347400002E7400002E
:10F6300028740000227400001C740000167400007E
:10F64000107400000A74000004740000FE730000CF
:10F65000F8730000F2730000E4740000EC73000023
:10F66000E6730000E0730000DA730000E474000049
:10F67000E4740000E4740000D4730000CE73000052
:10F68000C8730000E4740000E4740000E474000037
:10F69000E4740000E4740000E474000026730000C9
:10F6A000E4740000E4740000E4740000E4740000FA
:10F6B000E4740000E4740000E4740000E4740000EA
:10F6C000E4740000E4740000E4740000E4740000DA
:10F6D000E4740000E4740000E4740000C2730000ED
:10F6E000E4740000E4740000E4740000E4740000BA
:10F6F000E4740000E4740000E4740000E4740000AA
:10F70000E4740000E4740000E4740000E474000099
:10F71000E4740000E4740000E4740000E474000089
:10F72000E4740000E4740000E4740000E474000079
:10F73000E4740000E4740000E4740000E474000069
:10F74000E4740000E4740000E4740000E474000059
:10F75000E4740000E4740000E4740000E474000049
:10F76000E4740000E4740000E4740000E474000039
:10F77000E4740000E4740000E4740000E474000029
:10F78000E4740000E4740000E4740000E474000019
:10F79000E4740000E4740000E4740000BC73000032
:10F7A000B6730000B0730000AA730000A0730000DD
:10F7B0008C730000807300007A7300007473000083
:10F7C0006E730000E4740000E474000068730000CD
:10F7D000627300004E730000E4740000E4740000E3
:10F7E000E474000044730000E47400003873000007
:10F7F000E4740000E4740000E4740000E4740000A9
:10F80000E4740000E4740000E4740000E474000098
:10F81000E4740000E4740000E4740000E474000088
:10F82000E4740000E4740000E4740000E474000078
:10F83000E4740000E4740000E4740000E474000068
:10F84000E4740000E4740000E4740000E474000058
:10F85000E4740000E4740000E4740000E474000048
:10F86000E4740000E4740000E4740000E474000038
:10F87000E4740000E4740000E4740000E474000028
:10F88000E4740000E4740000E4740000E474000018
:10F89000E4740000E4740000E4740000E474000008
:10F8A000E4740000E4740000E4740000E4740000F8
:10F8B000E4740000E4740000E4740000E4740000E8
:10F8C000E4740000E4740000E4740000E4740000D8
:10F8D000E4740000E4740000E4740000E4740000C8
:10F8E000E4740000E4740000E4740000E4740000B8
:10F8F000E4740000E4740000E4740000E4740000A8
:10F90000E4740000E4740000E4740000E474000097
:10F91000E4740000E4740000E4740000E474000087
:10F92000E4740000E4740000E4740000E474000077
:10F93000E4740000E4740000E4740000E474000067
:10F94000E4740000E4740000E4740000E474000057
:10F95000E4740000E4740000E4740000E474000047
:10F96000E474000010730000E4740000E47400000C
:10F97000E4740000E4740000E4740000E474000027
:10F98000E4740000E4740000E4740000E474000017
:10F99000E4740000E47400002A730000D8860000BC
:10F9A0000087000014870000708600009E8600001B
:10F9B0005097000064970000789700008E97000031
:10F9C000A4970000D49700003897000038970000F3
:10F9D00038970000089800001E9800002C9800003E
:10F9E0003A980000509800005E980000749800005B
:10F9F00082980000969800003C970000269700002F
:10FA0000E0970000F49700004E990000369900003E
:10FA10001C99000002990000F2980000E69800008E
:10FA2000E2980000E2980000E2980000329A00009C
:10FA3000249A0000169A0000FC990000EE9900003C
:10FA4000D4990000C6990000AE9900009699000074
:10FA50007E99000066990000CE9800004C9A000044
:10FA6000E2980000E2980000E2980000E2980000AE
:10FA7000E29800000010161B2023272A2D30323573
:10FA800037393B3D4041434547494B4C4E5051531C
:10FA9000545657595A5B5D5E60616263656667687C
:10FAA0006A6B6C6D6E707172737475767778797A33
:10FAB0007B7C7D7E80808182838485868788898A1D
:10FAC0008B8C8D8E8F90909192939495969697981B
:10FAD000999A9B9B9C9D9E9FA0A0A1A2A3A3A4A535
:10FAE000A6A7A7A8A9AAAAABACADADAEAFB0B0B15E
:10FAF000B2B2B3B4B5B5B6B7B7B8B9B9BABBBBBC97
:10FB0000BDBDBEBFC0C0C1C1C2C3C3C4C5C5C6C7D9
:10FB1000C7C8C9C9CACBCBCCCCCDCECECFD0D0D123
:10FB2000D1D2D3D3D4D4D5D6D6D7D7D8D9D9DADA77
:10FB3000DBDBDCDDDDDEDEDFE0E0E1E1E2E2E3E3D2
:10FB4000E4E5E5E6E6E7E7E8E8E9EAEAEBEBECEC32
:10FB5000EDEDEEEEEFF0F0F1F1F2F2F3F3F4F4F597
:10FB6000F5F6F6F7F7F8F8F9F9FAFAFBFBFCFCFD05
:10FB7000FDFEFEFF22AC0000F2AA00008EAB0000EA
:10FB800030AC00005EAC000028AC0000430303036F
:10FB900003034343030343430303230103034303D7
:10FBA00003030303030303034303034303030101A9
:10FBB00003030303030303030303030303430303D5
:10FBC00003031303030303030303030303030303F5
:10FBD0000303030303030303030303030313134296
:10FBE00013024242420313130213020202024202B0
:10FBF00000010102020201010202010142424242ED
:10FC000042424242421301131302420153000000D8
:10FC1000FFFFFFFF56000000A000A00057000000FB
:10FC20000000F00058000000900100006200000099
:10FC3000FFFFFF007000000054B5AAAA7100000089
:10FC4000AA54954A72000000292949247300000033
:10FC50002242101074000000FFFFFFFB750000003F
:10FC60007D77BBB576000000565529497700000026
:10FC700022424000780000005680FFFF7E00000016
:10FC80000000F70044B100005AB1000062B100006A
:10FC90004CB1000054B1000054B1000044B1000068
:10FCA00044B1000044B1000044B1000054B1000070
:10FCB000B0B10000C8B10000D0B10000D8B1000060
:10FCC000E0B10000BAB10000AAB100000010161B9C
:10FCD0002023272A2D30323537393B3D40414345DB
:10FCE00047494B4C4E505153545657595A5B5D5EE1
:10FCF00060616263656667686A6B6C6D6E70717275
:10FD0000737475767778797A7B7C7D7E808081824A
:10FD1000838485868788898A8B8C8D8E8F9090913D
:10FD20009293949596969798999A9B9B9C9D9E9F4B
:10FD3000A0A0A1A2A3A3A4A5A6A7A7A8A9AAAAAB6D
:10FD4000ACADADAEAFB0B0B1B2B2B3B4B5B5B6B79D
:10FD5000B7B8B9B9BABBBBBCBDBDBEBFC0C0C1C1DD
:10FD6000C2C3C3C4C5C5C6C7C7C8C9C9CACBCBCC23
:10FD7000CCCDCECECFD0D0D1D1D2D3D3D4D4D5D672
:10FD8000D6D7D7D8D9D9DADADBDBDCDDDDDEDEDFCA
:10FD9000E0E0E1E1E2E2E3E3E4E5E5E6E6E7E7E827
:10FDA000E8E9EAEAEBEBECECEDEDEEEEEFF0F0F18A
:10FDB000F1F2F2F3F3F4F4F5F5F6F6F7F7F8F8F9F3
:10FDC000F9FAFAFBFBFCFCFDFDFEFEFF0002030559
:10FDD0000608090B0D0E101113141617191B1C1E03
:10FDE0001F2122242527292A2C2D2F303233353666
:10FDF00038393B3C3E3F4143444647494A4C4D4FCE
:10FE0000505153545657595A5C5D5F606263646643
:10FE100067696A6C6D6E707173747577787A7B7CC4
:10FE20007E7F808283848687888A8B8C8E8F909257
:10FE30009394959798999A9C9D9E9FA1A2A3A4A5FF
:10FE4000A7A8A9AAABACAEAFB0B1B2B3B4B5B7B8BE
:10FE5000B9BABBBCBDBEBFC0C1C2C3C4C5C6C7C89A
:10FE6000C9CACBCCCDCECFD0D0D1D2D3D4D5D6D792
:10FE7000D7D8D9DADBDCDCDDDEDFDFE0E1E2E2E3AC
:10FE8000E4E4E5E6E7E7E8E8E9EAEAEBECECEDEDE7
:10FE9000EEEEEFF0F0F1F1F2F2F3F3F4F4F4F5F545
:10FEA000F6F6F7F7F7F8F8F8F9F9F9FAFAFAFBFBCA
:10FEB000FBFCFCFCFCFCFDFDFDFDFDFEFEFEFEFE74
:10FEC000FEFEFFFFFFFFFFFFFFFFFFFF20BD000063
:10FED000F0BC000002BD000044BC000002BD0000F8
:10FEE000E6BC000002BD000044BC0000F0BC000005
:10FEF000F0BC0000E6BC000044BC00004CBC0000AC
:10FF00004CBC00004CBC000008BD0000F0BC000070
:10FF1000F0BC0000C4BC0000A8BD0000C4BC0000D0
:10FF2000E6BC0000C4BC0000A8BD0000F0BC00009E
:10FF3000F0BC0000E6BC0000A8BD00004CBC000006
:10FF40004CBC00004CBC0000B2BD000050BF000023
:10FF5000A0BE0000A0BE00009EBE000042BF000088
:10FF600042BF000038BF00009EBE000042BF00003C
:10FF700038BF000042BF00009EBE000048BF000026
:10FF800048BF000048BF0000D8BF000020CD0000DF
:10FF900002CD0000BCCC0000DACB0000BCCC0000DD
:10FFA000F4CC0000BCCC0000DACB000002CD000095
:10FFB00002CD0000F4CC0000DACB0000D2CB000070
:10FFC000D2CB0000D2CB000038CF000080D500009B
:10FFD00040D4000040D400003CD4000058D50000BC
:10FFE00058D500004AD500003CD4000058D5000088
:10FFF0004AD5000058D500003CD4000060D5000070
:020000021000EC
:1000000060D5000060D5000064D70000313633377A
:1000100056313039000000006C6F6700F8B5C046FB
:10002000F8BC08BC9E467047F8B5C046F8BC08BC92
:040030009E46704731
:08003400A8E1FF7F01000000BC
:04003C003924000063
:040040001124000087
:100044000024F40003020000C000000010000000BF
:100054000C0001000100000001000000010000008C
:1000640024F0FF1F0000000000000000000000005A
:10007400000000000000000000000000000000007C
:10008400000000000000000000000000000000006C
:10009400000000000000000000000000000000005C
:1000A400000000000000000000000000000000004C
:1000B400000000000000000000000000000000003C
:0C00C4000000000001000000000000002F
:040000030000E3AD69
:00000001FF
